:020000040800F2
:1080000000800120D9840208614402086344020808
:108010006544020867440208694402080000000041
:108020000000000000000000000000006B44020897
:108030006D440208000000006F440208C5B6010844
:108040001D8502081D8502081D8502081D85020880
:108050001D8502081D85020895D80108EDD8010884
:108060001D8502081D8502081D8502081D85020860
:108070001D8502081D8502081D8502081D85020850
:108080001D8502081D8502081D8502081D85020840
:108090001D8502081D8502081D8502081D85020830
:1080A0001D8502081D8502081D8502081D85020820
:1080B00069E601081D8502081D8502081D85020864
:1080C0001D8502081D8502081D8502081D85020800
:1080D0001D8502081D8502086DCB010841C80108F5
:1080E0001D8502081D8502081D8502081D850208E0
:1080F0001D8502081D8502081D8502081D850208D0
:108100001D8502081D85020845D901081D85020844
:108110001D8502081D8502081D8502081D850208AF
:108120001D8502081D8502081D8502081D8502089F
:108130001D8502081D8502081D8502081D8502088F
:108140001D8502081D8502081D850208B1C10108B0
:108150001D8502081D8502081D850208D5C5010878
:108160001D8502081D8502081D8502081D8502085F
:108170001D8502081D8502081D8502081D8502084F
:048180001D8502084F
:1081880010B5054C237833B9044B13B10448AFF349
:1081980000800123237010BDE80F002000000000BC
:1081A80014B7020808B5034B1BB103490348AFF3E2
:1081B800008008BD00000000EC0F002014B7020882
:1081C80010B515F0E1FB0022054B1A70054B1B6832
:1081D8009847BDE81040044B9B695B69184700BF8E
:1081E800D40A0020AC01002070A30208431E2DE928
:1081F800F0471446052B00F22881DFE813F006004B
:108208000C000C004E007800D200FFF7D9FF47F6AB
:10821800A85323603FE0924B924D02280ABFA9461B
:1082280099461D464FF0FF364FF000084FF0010AFF
:108238008D4BA9F10409DF68043D3B68D9F80400B7
:108248001B6998473B686868DB6898473B6855F83E
:10825800040F5B6998473B6859F8040F5B6A9847B5
:1082680018B90AFA08F326EA03063B6828689B69E6
:1082780098473B68D9F800005B6A984718B10AFA32
:1082880008F326EA030608F10108B8F1110FD4D162
:10829800C6F310062660002031E0216003292DD89E
:1082A800DFE801F0021A1E226F4BDB691B68188891
:1082B8001FF014FA66A3D3E900231FF0A3FB66A3FB
:1082C800D3E900231FF074FA0022684B1FF070FAFC
:1082D8001FF080FC2060DEE7634BDB695B68E6E744
:1082E800614BDB699B68E2E7614B1B6991E70129F8
:1082F800216022D04CB224B1022937D00220BDE837
:10830800F087594BDD68D5E900309B6824309847E1
:10831800D5E90030DB6840309847D5E90030DB68A4
:108328005C309847D5E900305B6940309847D5E91B
:1083380000305B695C309847ADE74B4BDC68D4E9AB
:1083480000309B6840309847D4E90030DB6824301F
:108358009847D4E90030DB685C309847D4E90030AE
:108368005B6924309847D4E90030E2E73E4BDC688B
:10837800D4E900309B685C309847D4E90030DB686A
:1083880024309847D4E90030DB6840309847D4E976
:1083980000305B6924309847D4E900305B6940308D
:1083A800C9E70129216037D04CB2DCB10229A5D137
:1083B8002D4BDC68D4E900309B685C309847D4E9E1
:1083C8000030DB6824309847D4E90030DB6840305F
:1083D8009847D4E900305B6924309847D4E90030E5
:1083E8009B69DCE7204BDD68D5E900309B682430C9
:1083F8009847D5E90030DB6840309847D5E9003028
:10840800DB685C309847D5E900305B6940309847B5
:10841800D5E900309B698DE7134BDC68D4E900305F
:108428009B6840309847D4E90030DB68243098478F
:10843800D4E90030DB685C309847D4E900305B69E8
:1084480024309847D4E90030E4E7042057E700BF18
:108458000000000000FEAF40AAF1D24D62101440A7
:10846800586400209465002070A30208000024408E
:10847800D40A002038B5064C05462368C31AB3F55C
:10848800FA7F04D3034B9B699B699847256038BDE5
:108498000410002070A302083B4B3C4ADB685B6871
:1084A80003F5BA71116003F1B001516003F1E801FD
:1084B800916003F59071D16003F5AC71116103F51A
:1084C800D671516103F5F271916103F50771D161BC
:1084D80003F51571116203F52371516203F53171CA
:1084E800916203F53F71D16203F54D71116303F594
:1084F8005B71516303F56971916303F57771D1631A
:1085080003F214411164224A03F17801116003F166
:108518009401516003F1CC01916003F58271D1603F
:1085280003F59E71116103F5C871516103F5E4719A
:10853800916103F50071D16103F50E71116203F5C4
:108548001C71516203F52A71916203F53871D16289
:1085580003F54671116303F55471516303F56271B4
:10856800916303F5707103F57E731364D16301227F
:10857800084B1A70084B094A5A65094ADA65094ACC
:108588009A651BF0E7BD00BF70A30208586400207D
:1085980094650020D40A00209C640020F58100081E
:1085A800C98100087D8400087047022070470220B6
:1085B80070477047704702207047022070470220BA
:1085C80070470120704770470220704770478369E1
:1085D800124A10B5C3E98122114B1249C365124BE7
:1085E800124AC0E90A131249C361C0E90C130362B5
:1085F800104B114C8364114B8265C364104BC463E8
:108608008363C0E910330F4BC0E914144366002399
:10861800C3660D4B0266C0E91C3310BDCB8500084C
:10862800B1850008B3850008B7850008D58500081E
:10863800BF850008BB850008C7850008BD85000800
:10864800C3850008CF850008D1850008704700BFA2
:108658000022012110B44FF0FF340848084B80F87D
:108668008C201A8083F81012C0E92141C0F890309C
:10867800C0F8802010BC7830FFF7A9BF9C640020A8
:108688001410002000234FF0FF314FF0010C064A70
:108698000648138082F810328261C0E9031C037512
:1086A8008360FFF794BF00BF341200209C64002051
:1086B80000231846054911F8012B02F003029A40DD
:1086C80002330E2B40EA0200F5D170475414002003
:1086D8000549431E063011F8012B02F0030203F886
:1086E800012F8342F7D1704754140020074B1A78A2
:1086F80002705A7842709A788270DA78C2701A7961
:1087080002715A7942719B79837170475414002021
:10871800F8B50024084B094D094FDE6815F8011B10
:108728007A6C33681059DB6901F003010434984707
:108738001C2CF3D1F8BD00BF70A30208541400200C
:10874800000000200723064A013B00F0030113F054
:10875800FF0302F8011B4FEA9000F5D1D8E700BFEC
:1087680054140020014B586AECE700BF00000020B9
:108778000549431E063013F8012F02F00302834215
:1087880001F8012BF7D1C3E7541400200278074BF6
:108798001A7042785A7082789A70C278DA700279C0
:1087A8001A7142795A7182799A71B1E7541400208A
:1087B8000022024BC3F88020704700BF9C64002051
:1087C80010B50348144616F0F4FC206010BD00BF35
:1087D8008414002010B50F4C0146204616F055FDB4
:1087E800002015F08DFE6F21204616F0E2FCC0F344
:1087F8000061002015F024FF012015F081FE7F2183
:10880800204616F0D6FCBDE81040C0F300610120F8
:1088180015F016BF84140020014816F0BCBC00BF38
:1088280084140020012808B503D815F053FE002051
:1088380008BD0820FCE7012808B503D815F028FE74
:10884800002008BD0820FCE70021F4E74942F2E7D0
:10885800F1E70129F8B506461D46084600F2CA8226
:10886800A32A00F0938143D8072A00F0EC8022D88D
:10887800032A00F0C1800AD8012A00F0B18040F232
:10888800A480002E40F0B48015F0CAFFA0E0052AAD
:1088980000F0C38040F2B68020248C4044F01004DD
:1088A800E4B22146B848002E40F0BF8016F081FCA3
:1088B800C0F304208CE0322A00F0FC800AD81C2A7D
:1088C80000F0DE801D2A00F0F080082A00F0D08039
:1088D80004267EE08C2A00F0F980A22A00F03E816E
:1088E800332AF5D1002E40F0ED8015F0DFFF6FE060
:1088F800AB2A00F0008232D8A72A4FEA011000F014
:10890800BE811AD8A52A00F06A8140F2548140F04D
:108918006C00C4B221469C4816F04BFC214600F47A
:1089280080479948002E40F09F81002F00F09681E3
:1089380016F03FFCC0F302104AE0A92A00F0BE81FD
:1089480040F2A98140F06D00C4B221468E48002E45
:1089580040F0C88116F02DFCC0F3032038E0B32A9C
:1089680000F009821BD8AD2A00F0E781C0F0D88159
:10897800AE2AADD10C0144F06D04E4B22146824820
:10898800002E40F0EF8116F014FC001400F07F0375
:1089980010F0400018BF6FF07F00184318E0B52AA8
:1089A80000F00B82C0F0FC81B82A00F00E82CE2ABB
:1089B8008ED1002E8CD1080140F06F01C9B27248E7
:1089C80016F0F7FBC0F3090002E026B915F00CFF1A
:1089D80028603046F8BD196815F07CFD0026F8E7D8
:1089E80016B915F0F3FEF3E7196815F095FEF5E7EB
:1089F800196815F04DFDF1E7002E7FF469AF15F009
:108A080001FFE5E716B915F027FFE1E71968002926
:108A1800B8BF494215F09AFEE0E716B915F00EFF07
:108A2800D6E7196816F015F8D8E716F0C2FB2B68D8
:108A380020F4F8521B0203F4F8531A432146524813
:108A480016F0A9FBCAE720248C4044F01004E4B2D5
:108A580021464D4826B916F0ACFB00F01F00B7E7D9
:108A680016F0A7FB2B6820F01F0203F01F03E4E7B2
:108A7800002E7FF42DAF15F089FDC0F30010A7E795
:108A88000C0144F06C04E4B221463F4826B916F0C4
:108A980090FBC0F380409BE716F08BFB2B6820F41B
:108AA80080229B0403F48023C7E7002E7FF410AFD5
:108AB8000020A4E716B915F0EBFE89E7197815F040
:108AC8005FFE8BE7196815F06BFE87E756B908015A
:108AD80040F06C0101F0FC012B4816F06AFBC0F372
:108AE800036075E71B68102B32D00EDC022B2BD0ED
:108AF80005DC012B17D04FF0FF332B606EE7042BFA
:108B080024D0082BF7D105230EE0402B22D003DC1C
:108B1800202BF0D1032307E0802B1DD0B3F5807FF5
:108B2800E9D1002300E00823040144F06C04E4B216
:108B38002B602146144816F03CFB2B6820F070622D
:108B48001B0603F0706378E70723EDE70623EBE7DE
:108B58000423E9E70223E7E70123E5E70C0144F0F2
:108B68006C04E4B22146084826B916F022FBC0F38B
:108B7800C1302DE716F01DFB2B6820F4C032DB0353
:108B880003F4C03359E700BF841400200C0144F0FB
:108B98006C04E4B22146984826B916F00AFBC0F3E3
:108BA800803015E716F005FB2B6820F480429B0304
:108BB80003F4804341E740F06C00C4B221468E487C
:108BC80026B916F0F6FAC0F3003001E716F0F1FA0C
:108BD8002B6820F480521B0303F480532DE740F0E8
:108BE8006C00C4B22146844816F0E3FA21460746D1
:108BF80000F4804380487EB923B116F0DAFAC0F356
:108C0800C310E5E616F0D5FAC0F3021317F40060B6
:108C180018BF43F0080370E743B116F0CAFA2B688F
:108C280020F4F062DB0103F4F06306E716F0C1FA02
:108C38002A6820F07000120102F0700202432146F7
:108C48006D4816F0A8FA21466B4816F0B2FA2B6860
:108C580020F400621B0203F40063EEE616F0A9FAA2
:108C6800C0F3C3102860B9E6002FD6D016F0A1FAD9
:108C78002B6820F070021B0103F07003DDE640F062
:108C88006C00C4B221465C48002E4ED116F091FA11
:108C980000F00F009CE640F06D00C4B22146564833
:108CA80026B916F086FAC0F3C03091E616F081FABC
:108CB8002B6820F40042DB039BB2BEE640F06D0057
:108CC800C4B221464C4826B916F073FAC0F34130B5
:108CD8007EE616F06EFA2B6820F4C0425B0303F4BC
:108CE800C043AAE616F065FA2B6820F470621B02EE
:108CF80003F47063A1E60C0144F06D04E4B221466C
:108D08003D4826B916F055FAC0F3411060E616F052
:108D180050FA2B6820F060025B0103F060038CE6D8
:108D28000C0144F06D04E4B2ACE716F042FA2B688B
:108D380020F00F0203F00F037FE60C0144F06D04EE
:108D4800E4B221462C4826B916F033FAC0F3006085
:108D58003EE616F02EFA2B6820F080721B0603F010
:108D680080736AE616F025FA2B6820F4FE021B04CD
:108D780003F4FE0361E60C0144F06C04E4B22146FE
:108D88001D4826B916F015FAC0F3404020E616F043
:108D980010FA2B6820F400325B0403F400334CE62D
:108DA800002E7FF495AD080140F06F01C9B212485A
:108DB80016F0FFF9C0F304400AE616B915F05AFD9B
:108DC80006E6196815F0CEFC08E60C0144F06C04C0
:108DD800E4B22146084826B916F0EBF9C0F3403052
:108DE800F6E516F0E6F92B6820F400525B0303F46D
:108DF800005322E60826ECE58414002007B501920A
:108E080001AB02460120FFF724FD03B05DF804FB27
:108E18001346024600201CE5014816F01EBA00BFA2
:108E280084140020022804BF0C4B93F8F00038B9D2
:108E38000B4BDB681B685B690A4AD2F89402184737
:108E4800012809D1054B93F8F030012B04D1044BCC
:108E5800DB681B689B69EFE7704700BF9C640020D4
:108E680070A302088414002070B50020FFF7DAFF11
:108E78000C4B0D4CDD68D4F894022B689B6898471E
:108E88002B68D4F8A4029B6898472B68D4F8A802EA
:108E98009B68984715F0B6FDBDE87040034B5B68CA
:108EA800184700BF70A3020884140020800A00201D
:108EB8000346052B10B5084614460BD006D8022BDE
:108EC80006D315F0F3FC2060002010BD182BF8D055
:108ED8000420FAE715F004FDF5E738B50D46044619
:108EE80020B915F08FFC2860204638BD0820FCE723
:108EF800022810B5144611D0032817D0012819D11B
:108F08000D4B0E4ADB68D2F8A4021B685B6A9847CF
:108F1800003018BF01202060002010BD064B074A12
:108F2800DB68D2F8A8021B685B6AF0E7084615F010
:108F38002DFBF0E70420F0E770A30208841400205A
:108F4800012838B504460D4608D815F03FFC2B68B3
:108F5800C11829602046BDE8384063E4082038BDC0
:108F680038B5002015F04EFC08B1002038BD0120AE
:108F780015F048FC05460028F7D10C4C204616F0A1
:108F880059F90B4815F0C2FC2B46D4F88C22D4F8BA
:108F98008412284615F01EFB01202B46D4F8902297
:108FA800D4F8881215F016FB0120DFE7841400209E
:108FB800A0860100022806D3052801D9182802D165
:108FC80000201060704704207047034B0846D3F810
:108FD800B0321146DB681847841400202DE9F041AF
:108FE8005A4C5B4D5B4F0121D4F8902028465A4BD0
:108FF80016F003F9FE68736803F1CC02C5F89422F1
:1090080003F59E72C5F8A82203F5AC72C5F8A42230
:1090180003F5C872C5F88C2203F5D67203F5BA7049
:10902800C5F8882203F5E47203F50E73C5F8AC326F
:109038003368C5F89022DB68C5F88402984733681E
:10904800D5F88C02DB6898473368D5F88802DB6866
:1090580098473368D5F89002DB6898473368D5F8A5
:109068009402DB6898473368D5F8AC02DB68984708
:109078003B693A4803F11402C5F8B022D5F8AC228E
:109088009A6115F043FC0023D5F88C22D5F8841298
:10909800184615F09FFAD5F88812D5F890220023C3
:1090A800012015F097FAD4F890302D4A0220C3F821
:1090B80004222C4AC3F8082201221A802A4B3222A1
:1090C800C4F89C30294B84F88C00C4F89830284B9D
:1090D800C4F89430274BC4F8A030274BC4F8B430F8
:1090E800264BC4F8B030264BC4F8A430254BC4F83E
:1090F800A830254BC4F8C430244BC4F8C030244BE6
:10910800C4F8D030234BC4F8CC30234BC4F8C83053
:10911800224BC4F8DC30224BC4F8D8304FF48F739C
:10912800C4E921321F4BC4F8D4301F4BC4F8E830CF
:109138001E4BC4F8EC301E4CFFF774FE23689847AA
:109148000021A3680846BDE8F04118479C64002048
:109158008414002070A3020848870208A086010032
:10916800698F0008218E00083F8800085988000888
:109178005588000851880008198E0008058E0008D7
:109188002D880008498F000821880008C987000831
:10919800DD870008F98E0008E38E00082D8E000890
:1091A800B9870008718E0008BD8F0008B98E0008C5
:1091B800800A0020014B1046DB6B18470000002096
:1091C800034B10B51B6C14469847206010BD00BFB8
:1091D80000000020062873B504460E467BD8404D93
:1091E80068462B6B013C98472B46042C04D8DFE8D3
:1091F80004F00866696C6F009DF800303360002049
:109208000BE09DF80120E978914208D19DF8020011
:10921800297B884203D10020306002B070BD1979E3
:10922800914206D19DF80200597B884201D1012361
:10923800E4E75979914206D19DF80200997B88426A
:1092480001D10223DAE79979914206D19DF802000B
:10925800D97B884201D10323D0E7D979914206D13D
:109268009DF80200197C884201D10423C6E7597A87
:10927800914206D19DF80200997C884201D10523CC
:10928800BCE7997A914206D19DF80200D97C8842C0
:1092980001D10623B2E7197A914206D19DF802005E
:1092A800597C884201D10723A8E7D97A914214D181
:1092B8009DF802201B7D9A420FD108239EE79DF856
:1092C80003309BE79DF8043098E79DF8053095E753
:1092D8009DF8063092E704209FE710209DE700BF25
:1092E8000000002007B5034B68461B6B984703B086
:1092F8005DF804FB0000002070B50020FFF7F2FFC6
:109308001E4B1F4CDD68206B2B689B6898472B68A9
:10931800E06A9B6898472B68E0689B6898472B68C9
:10932800A0689B6898472B6860689B6898472B687B
:1093380020689B6898472B68A0699B6898472B68AA
:10934800E0699B6898472B68A06A9B6898472B68D8
:1093580060699B6898472B68206A9B6898472B68C8
:10936800606A9B6898472B6820699B68984715F046
:1093780049FBBDE87040034B5B68184770A30208BF
:1093880044170020800A002010B5044618B915F0CB
:10939800A1F8204610BD0820FCE710B5044618B90E
:1093A80015F076F8204610BD0820FCE70021F4E708
:1093B8004942F2E7F1E7062873B505460C465DD841
:1093C800022903D901285BD10F2959DC2D4E6846A3
:1093D800336B98473346052D06D8DFE805F0030BB5
:1093E8004346494C8DF800406846DB6A98470020A0
:1093F80002B070BD082CF7D8DFE804F0050C111690
:109408001B20252A2F00F2788DF80120327B8DF859
:109418000220E9E732798DF80120727BF7E772794B
:109428008DF80120B27BF2E7B2798DF80120F27B4A
:10943800EDE7F2798DF80120327CE8E7727A8DF851
:109448000120B27CE3E7B27A8DF80120F27CDEE7F6
:10945800327A8DF80120727CD9E7F27A8DF80120F2
:10946800327DD4E78DF80340BEE78DF80440BBE7B2
:109478008DF80540B8E78DF80640B5E70420B7E752
:109488001020B5E700000020002015F039B838B5E5
:10949800154618B1012807D0042038BD084615F034
:1094A80075F828600020F8E7094B0A4DDC680A4B7C
:1094B800606800F5BA70D8616B6C58612368DB6826
:1094C80098476A6C236850699B699847EAE700BF28
:1094D80070A30208000000204417002038B50D468C
:1094E800044648B915F072F92B68C118296020465E
:1094F80014F0F0FF204638BD0820FCE770B505469B
:1095080016460C4600295DD10B2810D806283CD2F7
:1095180002282ED004D808B3012825D0042421E03D
:1095280004282ED029D9084615F088F91FE01328F9
:109538000CD80E283CD20C282FD00D28EED1224B67
:10954800224ADB68106B1B685B6A2CE0322835D036
:109558003328E3D1084615F0A9F908E015F044F9D5
:109568002C463060204670BD084615F02FF9306053
:10957800F8E7084615F054F9F9E7084615F042F9F6
:10958800F5E7084615F068F9F1E70828C6D1084656
:1095980014F0FCFFC0F30010E9E70B4B0B4ADB6843
:1095A800D06A1B685B6A9847003018BF0120DEE765
:1095B8000E381146C0B2FFF70DFED3E7084615F086
:1095C80067F9D4E70824CDE770A302084417002000
:1095D80030B585B0054601920C4600296ED10B289E
:1095E80012D8062846D2022837D004D848B3012812
:1095F8002CD004242EE0042834D00528F9D11146B3
:10960800204615F026FA25E013280FD80E2845D253
:109618000C2836D00D28ECD142F210739A42E8D8C3
:10962800274B91B29B682046984713E0332837D0E0
:109638008C283AD03228DCD1D1B2204615F0A0F8D7
:1096480008E0114614F046FF2C4603E01146204678
:1096580015F062F8204605B030BD1146204614F0DA
:1096680017FFF7E782EAE271A1EBE271204615F0F5
:109678006DF8EFE706381146C0B2FFF79CFE0446C6
:10968800E8E7104B1049DB68C86A1B68154612B139
:109698005B699847DEE79B699847D5E70E38EAE7A4
:1096A8001146204615F07CF8D4E701A90120FFF700
:1096B80091FD064B04469B6B02A8EAE70824C9E71C
:1096C800800A002070A30208441700200000002030
:1096D8006F4B2DE9F041DE686E4C7068002500F58F
:1096E8000073236300F5F273E36200F52A73E36005
:1096F80000F53173A36000F52373636000F50E7302
:10970800236000F55B73A36100F55473E36100F116
:10971800CC03A36200F5C873636100F56973236223
:1097280000F570736362336800F5BA70DB68206116
:10973800984733686069DB6898473368206BDB6853
:1097480098473368E06ADB6898473368206A1B6982
:1097580098473368504F1B69606A98477B6CE2688A
:109768001A60A2685A6062689A602268DA60A26920
:109778001A61E2695A61A26A9A617A6C336850592F
:10978800DB6898477A6C336850599B690435984769
:109798001C2DF2D14FF00008404D4FF40030D5F8A1
:1097A800903083F8008015F0B1F8D4E904124346EC
:1097B800404614F00FFF44F62061404614F0C6FFFF
:1097C80046F2A811404615F044F9354B0220C5F879
:1097D8009C30344BC5F89830334BC5F89430334B34
:1097E800C5F8A030324BC5F8B430324BC5F8B030AC
:1097F800314BC5F8A430314BC5F8A830304BC5F80B
:10980800C430304BC5F8C0302F4BC5F8CC302F4B87
:10981800C5F8D0302E4BC5F8DC30012385F88C30E4
:109828002C4BC5F8D430FFF75DFD404614F0EAFF35
:1098380010B1294B9B78ABB1BB6A98474FF4003005
:1098480015F064F8D4E904120023184614F0C2FE97
:1098580044F62061002014F079FF46F2A811002098
:1098680015F0F7F80222236B197C5A741868012244
:109878001AF0DFFD3368206B184C1B689847236883
:1098880098470021A3680846BDE8F041184700BF83
:1098980070A3020844170020000000209C640020E8
:1098A800A3930008BD930008B9930008B593000876
:1098B80005950008D995000891930008E5940008DB
:1098C800BD910008C9910008979400089194000878
:1098D800ED92000801930008D40A0020800A0020B5
:1098E8001B4B70B5DD681B4C2B68A0685B699847FB
:1098F8002B6820689B6898472B6860689B68984726
:109908002B68206A9B6898472B68606A9B68984711
:109918002B68E0689B6898472B6820699B68984784
:109928002B6860699B6898472B68A0699B68984773
:109938002B68E0699B6898472B68A0689B689847E4
:1099480015F060F8BDE87040034B5B68184700BF2E
:1099580070A3020884170020800A002010B514465E
:10996800062805D8DFE800F00626243540454F00D4
:10997800042010BD44F6206314689C424FD842F27C
:109988001071284B284ADB688C421B6898BF00215D
:10999800DB6988BF0121106A984742F21173B4FB52
:1099A800F3F103FB1141214B89B29B6800209847D2
:1099B8000020DEE71B4B2468DA68D2E9003000F5A6
:1099C80007701CB10021DB699847F1E79B6898474D
:1099D800EEE7144B1168DB68134A1B680031DB693A
:1099E80018BF01211069EFE7084614F0CFFD206089
:1099F800DEE70C4B0C4ADB6858681B6800F5BA7048
:109A08001061DB68E3E7074B074ADB6858681B68A7
:109A180000F22471D1605B6900F55470D7E710201B
:109A2800A7E700BF70A3020884170020800A00205F
:109A380010B50348144615F0A6FC206010BD00BF01
:109A4800D865002010B5094C0146204615F039FDAF
:109A5800002014F055FD6F21204615F094FCBDE858
:109A68001040C0F30061002014F0EABDD865002062
:109A7800014815F07ABC00BFD865002010B504462F
:109A880018B914F027FD204610BD0820FCE710B5D2
:109A9800044618B914F0FCFC204610BD0820FCE769
:109AA8000021F4E74942F2E7F1E770B504461D46A4
:109AB8000E46002940F04E85A52A00F08F8256D820
:109AC800172A00F0478126D8042A00F0E8800ED82B
:109AD800012A00F0AD80002A00F09E80022A00F0E2
:109AE800B280032A00F0BA800424204670BD072AF9
:109AF80000F0068107D8052A00F0DF80062A00F06A
:109B0800E7800424F1E7082A00F01181152A00F003
:109B180017810424E9E7322A00F0B28113D81B2AFE
:109B280000F0638107D8182A00F039811A2A00F05A
:109B380044810424D9E71C2A00F06F811D2A00F013
:109B480086810424D1E7A22A00F0008207D8332AAC
:109B580000F0A1818C2A00F0A9810424C5E7A32A7A
:109B680000F00C82A42A00F021820424BDE7B42A64
:109B780000F0B58324D8AA2A00F018830CD8A72AA5
:109B880000F0CE82C0F08682A82A00F0E082A92ADE
:109B980000F0F4820424A8E7AD2A00F0518307D826
:109BA800AB2A00F01B83AC2A00F0308304249CE726
:109BB800AE2A00F05D83B32A00F07983042494E789
:109BC800BB2A00F0278413D8B82A00F0C88307D826
:109BD800B52A00F09083B62A00F09A83042484E71B
:109BE800B92A00F0D683BA2A00F0ED8304247CE772
:109BF800C02A00F06C8407D8BC2A00F03384BF2A3E
:109C080000F04684042470E7CC2A00F07B84CE2A36
:109C180000F09684042468E720B9002014F0E4FDDD
:109C2800286062E71968002014F054FC00245CE7FF
:109C380018B914F0CBFD286057E71968304614F0BE
:109C48006BFD344651E718B914F0EAFD28604CE77B
:109C58001968002014F01CFC002446E7002840F096
:109C68007C8414F015FE18B914F0CCFD28603CE78C
:109C7800204614F01BFE12210646B14815F083FB5E
:109C8800C0F313027A20D317A6FB00011EF066FA70
:109C980000F11303262B98BF0020286025E718B988
:109CA80014F0DAFD286020E7196830460029B8BFAB
:109CB800494214F04BFD344617E718B914F0BEFDBD
:109CC800286012E71968002014F0C3FE00240CE78E
:109CD80010219B482CB915F056FBC0F304202860CE
:109CE80003E715F050FB2B6820F4F8521B0203F42D
:109CF800F8531A431021924815F037FB0024F4E674
:109D080010218F482CB915F03EFB00F01F00286089
:109D1800EBE615F038FB2B6820F01F0203F01F0359
:109D28001A431021864815F020FB3446DDE600284A
:109D380040F0168414F02AFCC0F300102860D4E622
:109D4800002800F010841A6811217D4815F00DFBD9
:109D58000024CAE67B4E80B91521794815F013FB1B
:109D680048B14FF0807393FBF0F0B042A8BF304683
:109D780028600024B9E63046FAE71B686BB14FF05B
:109D8800807292FBF3F2B242A8BF32462A601521D4
:109D98006B4815F0EAFA0024A7E63246F6E728B938
:109DA8003321674815F0EFFA28609EE61A683321D8
:109DB800634815F0DAFA002497E66C2160482CB95C
:109DC80015F0E1FAC0F3804028608EE615F0DBFA62
:109DD8002B6820F480229B0403F480231A436C210F
:109DE800574815F0C2FA00247FE66C2154482CB974
:109DF80015F0C9FAC0F3C040286076E615F0C3FA3A
:109E08002B6820F40022DB0403F400231A436C219E
:109E18004B4815F0AAFA344667E638B9014648486F
:109E280015F0B1FAC0F3400028605EE6002144480E
:109E380015F0A9FA2B6820F002025B0003F0020378
:109E48001A4300213E4815F090FA00244DE60028F8
:109E580040F08C8314F02AFD12210646384815F08C
:109E680092FAC0F313027A20D317A6FB00011EF062
:109E780075F900F11303262B98BF0020286034E6FB
:109E880018B914F005FD28602FE61978304614F04B
:109E980077FC344629E618B914F008FD286024E652
:109EA8001968002014F07CFC00241EE650B96C21CF
:109EB800234815F068FA4FF48073C0F30360034138
:109EC8002B6012E61B68102B35D00FDC022B2ED02E
:109ED80006DC012B18D04FF0FF3310242B6004E66A
:109EE800042B26D0082BF6D105230EE0402B24D0D6
:109EF80003DC202BEFD1032307E0802B24D0B3F51C
:109F0800807FE8D1002300E008232B606C210C48F7
:109F180015F039FA2B6820F070621B0603F07063A5
:109F28001A436C21064815F020FA0024DDE50723C2
:109F3800EBE70623E9E70423E7E70223E5E700BFA9
:109F4800D8650020FFFF0F000123DEE76C21BB4826
:109F58002CB915F018FAC0F3C1302860C5E515F022
:109F680012FA2B6820F4C032DB0303F4C0331A431F
:109F78006C21B24815F0F9F93446B6E56C21AF48C2
:109F88002CB915F000FAC0F380302860ADE515F063
:109F9800FAF92B6820F480429B0303F480431A43A8
:109FA8006C21A64815F0E1F900249EE56C21A34830
:109FB8002CB915F0E8F9C0F30030286095E515F0E4
:109FC800E2F92B6820F480521B0303F480531A43F0
:109FD8006C219A4815F0C9F9002486E56C21974848
:109FE80004BB15F0D0F910F480464FF06C0193488B
:109FF80005D015F0C8F9C0F3C310286075E515F051
:10A00800C2F96C2104468D4815F0BDF92205C0F34C
:10A01800021002D42860002467E540F00800286098
:10A02800344662E515F0AFF910F480444FF06C0146
:10A0380082480ED015F0A7F92B6820F4F062DB01F6
:10A0480003F4F0631A436C217C4815F08EF934460A
:10A058004BE515F098F96C21784815F094F92A68C1
:10A0680020F40060120202F4006202436C2173487B
:10A0780015F07BF96C21714815F085F92B6820F0F3
:10A0880070021B0103F070031A436C216B4815F032
:10A098006CF92AE56C216948ECB915F074F910F4EB
:10A0A80080444FF06C01654806D015F06CF9C0F398
:10A0B80002102860002418E515F065F96C210646A1
:10A0C8005E4815F060F93305C0F3C310A2D540F01F
:10A0D8000800286009E515F056F910F480444FF09F
:10A0E8006C0156480ED015F04EF92B6820F070021E
:10A0F8001B0103F070031A436C21504815F035F921
:10A108000024F2E415F03FF92B6820F4F062DB013B
:10A1180003F4F0631A436C21484815F026F9E4E487
:10A128006C2146482CB915F02EF900F00F00286074
:10A13800DBE415F028F92B6820F00F0203F00F0379
:10A148001A436C213D4815F010F93446CDE46D21D1
:10A158003A482CB915F017F9C0F3C0302860C4E4A8
:10A1680015F011F92B6820F40042DB039BB21A4367
:10A178006D21324815F0F9F80024B6E46D212F4816
:10A188002CB915F000F9C0F341302860ADE415F0A2
:10A19800FAF82B6820F4C0425B0303F4C0431A4367
:10A1A8006D21264815F0E1F800249EE46D2123482E
:10A1B8002CB915F0E8F8C0F30320286095E415F0F1
:10A1C800E2F82B6820F470621B0203F470631A43F0
:10A1D8006D211A4815F0C9F8344686E46D211748F0
:10A1E8002CB915F0D0F8C0F3411028607DE415F0C3
:10A1F800CAF82B6820F060025B0103F060031A4381
:10A208006D210E4815F0B1F800246EE46D210B485D
:10A218002CB915F0B8F800F00F00286065E415F0C7
:10A22800B2F82B6820F00F0203F00F031A436D21D8
:10A23800024815F09AF8002457E400BFD8650020BA
:10A248006D21BD482CB915F09EF8C0F30060286058
:10A258004BE415F098F82B6820F080721B0603F089
:10A2680080731A436D21B44815F07FF834463CE4F6
:10A278006D21B14864B915F086F8001400F07F0329
:10A2880010F0400018BF6FF07F00184328602CE4DE
:10A2980015F079F82B6820F4FE021B0403F4FE0382
:10A2A8001A436D21A44815F060F800241DE46C21C0
:10A2B800A1482CB915F067F8C0F34040286014E4B1
:10A2C80015F061F82B6820F400325B0403F40033C6
:10A2D8001A436C21984815F048F8002405E4002832
:10A2E80040F047816F21944815F04DF8C0F30440C1
:10A2F8002860FFF7FABB20B914F0BCFA2860FFF712
:10A30800F4BB1968002014F02DFA0024FFF7EDBB08
:10A318008A4E88B91421884815F035F850B14FF0A5
:10A32800807393FBF0F0B042A8BF30462860002449
:10A33800FFF7DBBB3046F9E71B6873B14FF080725B
:10A3480092FBF3F2B242A8BF32462A6014217A483F
:10A3580015F00BF80024FFF7C8BB3246F5E76C216F
:10A36800754834B915F00FF8C0F340302860FFF78E
:10A37800BCBB15F008F82B6820F400525B0303F40B
:10A3880000531A436C216C4814F0EFFF3446FFF772
:10A39800ACBB6C21684834B914F0F5FFC0F3035026
:10A3A8002860FFF7A2BB14F0EEFF2B6820F47002C0
:10A3B8001B0503F470031A436C215F4814F0D5FFA2
:10A3C8000024FFF792BB5D4E88B913215A4814F058
:10A3D800DAFF50B14FF0807393FBF0F0B042A8BFA2
:10A3E800304628600024FFF780BB3046F9E71B6839
:10A3F80073B14FF0807292FBF3F2B242A8BF3246BB
:10A408002A6013214C4814F0B0FF0024FFF76DBBFD
:10A418003246F5E77021484834B914F0B4FFC0F368
:10A4280007202860FFF761BB14F0ADFF2A6820F40D
:10A438007F40120292B2024370213F4814F095FF08
:10A4480031463D4814F09FFF2B6820F00402002B92
:10A4580018BF042331461A43374814F086FF3446A0
:10A46800FFF743BB702134482CB914F08CFFC0B2FD
:10A478002860FFF73ABB14F086FF2A7820F0FF0027
:10A48800024370212C4814F070FF0024FFF72DBB05
:10A4980040B97021284814F076FFC0F301402860C5
:10A4A800FFF723BB1B68032B66D87021224814F0E2
:10A4B8006AFF2B6820F440321B0403F440331A432C
:10A4C80070211D4814F051FF0024FFF70EBB7021C6
:10A4D800194834B914F057FFC0F380402860FFF7DB
:10A4E80004BB14F050FF2B6820F48022002B18BF07
:10A4F8004FF4802370211A430F4814F036FF344676
:10A50800FFF7F3BA70210C4834B914F03CFFC0F3DC
:10A5180001502860FFF7E9BA14F035FF2B6820F4E2
:10A5280040121B0503F440131A437021024814F02B
:10A538001CFF0024FFF7D9BAD8650020FFFF0F00E1
:10A54800E8B96F210F4814F01EFFC0F30900286016
:10A55800FFF7CBBA0824FFF7C8BA0424FFF7C5BA37
:10A568000424FFF7C2BA0424FFF7BFBA0424FFF794
:10A57800BCBA0424FFF7B9BA1024FFF7B6BA04240A
:10A58800FFF7B3BAD865002007B5019201AB0246C0
:10A598000120FFF78AFA03B05DF804FB1346024670
:10A5A8000020FFF782BA014814F073BFD865002075
:10A5B80008B5002014F026F910B1094B987868B155
:10A5C800084814F04FFF4FF4003014F09FF90023AF
:10A5D8000549184606C913F0FDFF012008BD00BF54
:10A5E800D40A0020D865002084170020022804BF60
:10A5F8000B4B93F8F00030B90A4BDB681B685B69BA
:10A60800094A90681847012809D1054B93F8F0309A
:10A61800012B04D1034BDB681B689B69F0E770478B
:10A628009C64002070A30208841700200346052BB1
:10A6380010B5084614460BD006D8022B06D314F0E2
:10A6480035F92060002010BD182BF8D00420FAE757
:10A6580014F046F9F5E738B50D46044620B914F06C
:10A66800D1F82860204638BD0820FCE7012910B53C
:10A67800044608D1044A702114F077FE2046BDE84C
:10A68800104014F0C5BE10BDC804050038B50D460D
:10A69800044648B914F09AF82B68C1182960204676
:10A6A80013F018FF204638BD0820FCE7022806D31F
:10A6B800052801D9182802D100201060704704200D
:10A6C8007047054B0846DB6E114603B11847034B2C
:10A6D8001B68DB68FAE700BF9C6400205C68002008
:10A6E8002DE9F0416C4D6D4FD5F890206C4B3846F4
:10A6F800DFF80C82012114F06EFE6A49384614F026
:10A70800DCFED8F80C60684C736803F1CC02A260D8
:10A7180003F5BA72226003F5C872626003F5F2723B
:10A72800226203F50072626203F55472E26003F577
:10A738005B7203F56970226103F5627203F5707349
:10A74800E361336862611B69A06198473368E06917
:10A758001B699847336860691B69984733682068A4
:10A76800DB68984733686068DB6898473368A06897
:10A77800DB68984733682069DB6898473368E06886
:10A78800DB6898473368606ADB6898473368206AF3
:10A79800DB6898473368606A9B6998473368206A22
:10A7A8009B699847336860699B6998473368E06894
:10A7B8009B699847D8F810203C4B02F114011960A6
:10A7C80073684FF4003003F50E73936114F09EF82C
:10A7D800D4E900120023184613F0FCFEAF670127E6
:10A7E800D5F89030324A1F80C3F80422314A02203B
:10A7F800C3F80822304B3222C5F89C302F4B85F81D
:10A808008C70C5F898302E4BC5F894302D4BC5F890
:10A81800A0302D4BC5F8B4302C4BC5F8B0302C4BBC
:10A82800C5F8A4302B4BC5F8A8302B4BC5F8C4305D
:10A838002A4BC5F8C0302A4BC5F8D030294BC5F88B
:10A84800CC30294BC5F8C830284BC5F8DC304FF45C
:10A85800F073C5E92132264BC5F8D430254BC5F82D
:10A86800E830254BC5F8EC30FFF7C0FE0222636ADA
:10A87800197C5A7418683A4619F0DBFD3368606A27
:10A888001E4C1B689847236898470021A368084610
:10A89800BDE8F041184700BF9C640020D86500203F
:10A8A8004889020875A60008841700205C68002003
:10A8B800B9A50008AFA50008979A0008B19A000842
:10A8C800AD9A0008A99A0008A5A5000891A5000856
:10A8D800859A000895A60008799A0008399A000810
:10A8E8004D9A0008659900085FA60008F5A50008BC
:10A8F800E9980008B5A6000835A60008800A0020D7
:10A9080070A3020838B5184B184CDD6820682B680E
:10A918005B6998472B6860689B6898472B68A068B4
:10A928009B6898472B68E0689B6898472B68206964
:10A938009B6898472B6860699B6898472B68A06953
:10A948009B6898472B68E0699B6898472B68206A42
:10A958009B68984714F056F8054B5B6898470023A6
:10A9680084F8243038BD00BF70A30208B81700204F
:10A97800800A002010B50348144614F020FE206019
:10A9880010BD00BF64680020014814F00ABE00BF73
:10A998006468002010B5044618B913F09BFD2046E2
:10A9A80010BD0820FCE710B5044618B913F070FD77
:10A9B800204610BD0820FCE70021F4E74942F2E7F1
:10A9C800F1E770B504461D460E46002940F04E8555
:10A9D800A52A00F08F8256D8172A00F0478126D87A
:10A9E800042A00F0E8800ED8012A00F0AD80002A81
:10A9F80000F09E80022A00F0B280032A00F0BA809C
:10AA08000424204670BD072A00F0068107D8052ACD
:10AA180000F0DF80062A00F0E7800424F1E7082A26
:10AA280000F01181152A00F017810424E9E7322A81
:10AA380000F0B28113D81B2A00F0638107D8182AC6
:10AA480000F039811A2A00F044810424D9E71C2A2D
:10AA580000F06F811D2A00F086810424D1E7A22A24
:10AA680000F0008207D8332A00F0A1818C2A00F078
:10AA7800A9810424C5E7A32A00F00C82A42A00F0C7
:10AA880021820424BDE7B42A00F0B58324D8AA2A79
:10AA980000F018830CD8A72A00F0CE82C0F0868276
:10AAA800A82A00F0E082A92A00F0F4820424A8E78A
:10AAB800AD2A00F0518307D8AB2A00F01B83AC2ADB
:10AAC80000F0308304249CE7AE2A00F05D83B32AAB
:10AAD80000F07983042494E7BB2A00F0278413D874
:10AAE800B82A00F0C88307D8B52A00F09083B62AA0
:10AAF80000F09A83042484E7B92A00F0D683BA2A9E
:10AB080000F0ED8304247CE7C02A00F06C8407D8A9
:10AB1800BC2A00F03384BF2A00F04684042470E77E
:10AB2800CC2A00F07B84CE2A00F09684042468E7BF
:10AB380020B9002013F058FE286062E71968002049
:10AB480013F0C8FC00245CE718B913F03FFE286036
:10AB580057E71968304613F0DFFD344651E718B956
:10AB680013F05EFE28604CE71968002013F090FC93
:10AB7800002446E7002840F07C8413F089FE18B9C9
:10AB880013F040FE28603CE7204613F08FFE1221A8
:10AB98000646B14814F013FDC0F313027A20D31708
:10ABA800A6FB00011DF0DAFA00F11303262B98BF6B
:10ABB8000020286025E718B913F04EFE286020E72A
:10ABC800196830460029B8BF494213F0BFFD344622
:10ABD80017E718B913F032FE286012E71968002049
:10ABE80013F037FF00240CE710219B482CB914F010
:10ABF800E6FCC0F30420286003E714F0E0FC2B68AF
:10AC080020F4F8521B0203F4F8531A431021924817
:10AC180014F0C7FC0024F4E610218F482CB914F076
:10AC2800CEFC00F01F002860EBE614F0C8FC2B688F
:10AC380020F01F0203F01F031A431021864814F066
:10AC4800B0FC3446DDE6002840F0168413F09EFC84
:10AC5800C0F300102860D4E6002800F010841A68B9
:10AC680011217D4814F09DFC0024CAE67B4E80B972
:10AC78001521794814F0A3FC48B14FF0807393FB79
:10AC8800F0F0B042A8BF304628600024B9E630464C
:10AC9800FAE71B686BB14FF0807292FBF3F2B24295
:10ACA800A8BF32462A6015216B4814F07AFC0024AC
:10ACB800A7E63246F6E728B93321674814F07FFC47
:10ACC80028609EE61A683321634814F06AFC002461
:10ACD80097E66C2160482CB914F071FCC0F38040F1
:10ACE80028608EE614F06BFC2B6820F480229B040D
:10ACF80003F480231A436C21574814F052FC0024B3
:10AD08007FE66C2154482CB914F059FCC0F3C040BC
:10AD1800286076E614F053FC2B6820F40022DB044C
:10AD280003F400231A436C214B4814F03AFC3446D0
:10AD380067E638B90146484814F041FCC0F34000C2
:10AD480028605EE60021444814F039FC2B6820F0A6
:10AD580002025B0003F002031A4300213E4814F08C
:10AD680020FC00244DE6002840F08C8313F09EFD63
:10AD780012210646384814F022FCC0F313027A2048
:10AD8800D317A6FB00011DF0E9F900F11303262BE8
:10AD980098BF0020286034E618B913F079FD2860C0
:10ADA8002FE61978304613F0EBFC344629E618B93B
:10ADB80013F07CFD286024E61968002013F0F0FCED
:10ADC80000241EE650B96C21234814F0F8FB4FF418
:10ADD8008073C0F3036003412B6012E61B68102BDD
:10ADE80035D00FDC022B2ED006DC012B18D04FF00B
:10ADF800FF3310242B6004E6042B26D0082BF6D151
:10AE080005230EE0402B24D003DC202BEFD10323B5
:10AE180007E0802B24D0B3F5807FE8D1002300E041
:10AE280008232B606C210C4814F0C9FB2B6820F018
:10AE380070621B0603F070631A436C21064814F015
:10AE4800B0FB0024DDE50723EBE70623E9E704234D
:10AE5800E7E70223E5E700BF64680020FFFF0F0073
:10AE68000123DEE76C21BB482CB914F0A8FBC0F322
:10AE7800C1302860C5E514F0A2FB2B6820F4C0326D
:10AE8800DB0303F4C0331A436C21B24814F089FB86
:10AE98003446B6E56C21AF482CB914F090FBC0F3EA
:10AEA80080302860ADE514F08AFB2B6820F48042DE
:10AEB8009B0303F480431A436C21A64814F071FBEA
:10AEC80000249EE56C21A3482CB914F078FBC0F34C
:10AED8000030286095E514F072FB2B6820F480524E
:10AEE8001B0303F480531A436C219A4814F059FB4E
:10AEF800002486E56C21974804BB14F060FB10F42D
:10AF080080464FF06C01934805D014F058FBC0F30D
:10AF1800C310286075E514F052FB6C2104468D4877
:10AF280014F04DFB2205C0F3021002D4286000245F
:10AF380067E540F008002860344662E514F03FFBFE
:10AF480010F480444FF06C0182480ED014F037FBA7
:10AF58002B6820F4F062DB0103F4F0631A436C21E0
:10AF68007C4814F01EFB34464BE514F028FB6C219A
:10AF7800784814F024FB2A6820F40060120202F4D6
:10AF8800006202436C21734814F00BFB6C2171487A
:10AF980014F015FB2B6820F070021B0103F07003FE
:10AFA8001A436C216B4814F0FCFA2AE56C216948B5
:10AFB800ECB914F004FB10F480444FF06C016548C0
:10AFC80006D014F0FCFAC0F302102860002418E53B
:10AFD80014F0F5FA6C2106465E4814F0F0FA3305D1
:10AFE800C0F3C310A2D540F00800286009E514F0AA
:10AFF800E6FA10F480444FF06C0156480ED014F075
:10B00800DEFA2B6820F070021B0103F070031A436C
:10B018006C21504814F0C5FA0024F2E414F0CFFA79
:10B028002B6820F4F062DB0103F4F0631A436C210F
:10B03800484814F0B6FAE4E46C2146482CB914F0F8
:10B04800BEFA00F00F002860DBE414F0B8FA2B68B1
:10B0580020F00F0203F00F031A436C213D4814F04F
:10B06800A0FA3446CDE46D213A482CB914F0A7FA79
:10B07800C0F3C0302860C4E414F0A1FA2B6820F4AF
:10B088000042DB039BB21A436D21324814F089FA5F
:10B098000024B6E46D212F482CB914F090FAC0F3BF
:10B0A80041302860ADE414F08AFA2B6820F4C042DD
:10B0B8005B0303F4C0431A436D21264814F071FA68
:10B0C80000249EE46D2123482CB914F078FAC0F3CB
:10B0D8000320286095E414F072FA2B6820F470625B
:10B0E8001B0203F470631A436D211A4814F059FACD
:10B0F800344686E46D2117482CB914F060FAC0F381
:10B10800411028607DE414F05AFA2B6820F06002A0
:10B118005B0103F060031A436D210E4814F041FAF5
:10B1280000246EE46D210B482CB914F048FA00F0A5
:10B138000F00286065E414F042FA2B6820F00F0233
:10B1480003F00F031A436D21024814F02AFA002471
:10B1580057E400BF646800206D21BD482CB914F085
:10B168002EFAC0F3006028604BE414F028FA2B682C
:10B1780020F080721B0603F080731A436D21B448D7
:10B1880014F00FFA34463CE46D21B14864B914F068
:10B1980016FA001400F07F0310F0400018BF6FF09B
:10B1A8007F00184328602CE414F009FA2B6820F477
:10B1B800FE021B0403F4FE031A436D21A44814F095
:10B1C800F0F900241DE46C21A1482CB914F0F7F91A
:10B1D800C0F34040286014E414F0F1F92B6820F41F
:10B1E80000325B0403F400331A436C21984814F0CE
:10B1F800D8F9002405E4002840F047816F219448DD
:10B2080014F0DDF9C0F304402860FFF7FABB20B959
:10B2180013F030FB2860FFF7F4BB1968002013F027
:10B22800A1FA0024FFF7EDBB8A4E88B9142188489B
:10B2380014F0C5F950B14FF0807393FBF0F0B042B1
:10B24800A8BF304628600024FFF7DBBB3046F9E78B
:10B258001B6873B14FF0807292FBF3F2B242A8BF41
:10B2680032462A6014217A4814F09BF90024FFF72B
:10B27800C8BB3246F5E76C21754834B914F09FF91C
:10B28800C0F340302860FFF7BCBB14F098F92B6876
:10B2980020F400525B0303F400531A436C216C48FA
:10B2A80014F07FF93446FFF7ACBB6C21684834B919
:10B2B80014F085F9C0F303502860FFF7A2BB14F01F
:10B2C8007EF92B6820F470021B0503F470031A43FF
:10B2D8006C215F4814F065F90024FFF792BB5D4EBE
:10B2E80088B913215A4814F06AF950B14FF08073A5
:10B2F80093FBF0F0B042A8BF304628600024FFF767
:10B3080080BB3046F9E71B6873B14FF0807292FB3F
:10B31800F3F2B242A8BF32462A6013214C4814F017
:10B3280040F90024FFF76DBB3246F5E77021484825
:10B3380034B914F044F9C0F307202860FFF761BB63
:10B3480014F03DF92A6820F47F40120292B20243B9
:10B3580070213F4814F025F931463D4814F02FF983
:10B368002B6820F00402002B18BF042331461A432F
:10B37800374814F016F93446FFF743BB70213448B8
:10B388002CB914F01CF9C0B22860FFF73ABB14F0CE
:10B3980016F92A7820F0FF00024370212C4814F097
:10B3A80000F90024FFF72DBB40B97021284814F09C
:10B3B80006F9C0F301402860FFF723BB1B68032B85
:10B3C80066D87021224814F0FAF82B6820F440322D
:10B3D8001B0403F440331A4370211D4814F0E1F8AC
:10B3E8000024FFF70EBB7021194834B914F0E7F8B0
:10B3F800C0F380402860FFF704BB14F0E0F82B6826
:10B4080020F48022002B18BF4FF4802370211A43A8
:10B418000F4814F0C6F83446FFF7F3BA70210C4809
:10B4280034B914F0CCF8C0F301502860FFF7E9BA3A
:10B4380014F0C5F82B6820F440121B0503F44013E0
:10B448001A437021024814F0ACF80024FFF7D9BA67
:10B4580064680020FFFF0F00E8B96F210F4814F05F
:10B46800AEF8C0F309002860FFF7CBBA0824FFF74D
:10B47800C8BA0424FFF7C5BA0424FFF7C2BA0424E3
:10B48800FFF7BFBA0424FFF7BCBA0424FFF7B9BA20
:10B498001024FFF7B6BA0424FFF7B3BA6468002093
:10B4A80007B5019201AB02460120FFF78AFA03B003
:10B4B8005DF804FB134602460020FFF782BA0148F4
:10B4C80014F0F5B86468002008B5002013F09AF964
:10B4D80010B1094B987870B1084814F0D5F84FF4BA
:10B4E800003013F013FA0023054918468A684968A2
:10B4F80013F070F8012008BDD40A00206468002009
:10B50800B8170020022804BF0B4B93F8F00030B99D
:10B518000A4BDB681B685B69094A106818470128F1
:10B5280009D1054B93F8F030012B04D1034BDB68AC
:10B538001B689B69F0E770479C64002070A30208B1
:10B54800B817002010B51446062805D8DFE800F023
:10B558000618162732374100042010BD136844F638
:10B568002062934239D842F21172B3FBF2F102FB26
:10B5780011311B4B89B29B68002098470020ECE7EB
:10B58800184B2468DA68D2E9003000F507701CB15E
:10B598000021DB699847F1E79B689847EEE7114B74
:10B5A8001168DB68104A1B680031DB6918BF01218C
:10B5B8005069EFE7084612F0E9FF2060DEE7094B23
:10B5C800094ADB6858681B6800F5BA705061DB6887
:10B5D800E3E70220FFF796FFD0E71020BDE700BFA2
:10B5E800800A002070A30208B81700200346052B24
:10B5F80010B5084614460BD006D8022B06D313F014
:10B6080055F92060002010BD182BF8D00420FAE767
:10B6180013F066F9F5E738B50D46044620B913F07E
:10B62800F1F82860204638BD0820FCE738B5194CE9
:10B63800054694F8240001281CD002281FD029466A
:10B64800154814F04CF8002012F05AFF002012F0B0
:10B658009DFF10F008041BD1820619D56F210E48F2
:10B6680013F0ADFFC30113D52046BDE838400221D1
:10B6780012F066BF0223A56284F82430DFE7A36ACC
:10B68800EB1AB3F5FA6FDAD9FFF73CFF0323F3E7B8
:10B6980038BD00BFB817002064680020012910B524
:10B6A80004460DD1074A702113F07BFF2046064A55
:10B6B8000A2113F076FF2046BDE8104013F0C0BF02
:10B6C80010BD00BF1E000CC40004080038B50D46AC
:10B6D800044648B913F07AF82B68C1182960204647
:10B6E80012F0F8FE204638BD0820FCE7022806D3F1
:10B6F800052801D9182802D10020106070470420BD
:10B708007047054B0846DB6E114603B11847034BDB
:10B718001B68DB68FAE700BF9C64002060680020B3
:10B728002DE9F0415C4C5D4FD4F890205C4B3846D5
:10B73800DFF8CC81012113F066FF5A49384613F02F
:10B74800CAFFD8F80C60584D736803F1CC022A6020
:10B7580003F5BA726A6003F5C872AA6003F500724D
:10B76800EA6003F554722A6103F55B7203F56270AF
:10B778006A6103F5697203F570732B623368EA61D5
:10B788001B69A861984733682868DB68984733685D
:10B798006868DB6898473368A868DB689847336847
:10B7A800E868DB68984733686869DB6898473368F6
:10B7B8002869DB6898473368E8685B6998473368A5
:10B7C800A8699B699847336828699B699847D8F89E
:10B7D8001020364B02F11401196073684FF40030E1
:10B7E80003F50E73936113F091F8D5E90112002364
:10B7F800184612F0EFFED4F890202D4BA767C2F838
:10B8080004322C4B3221C2F80832012313802A4A11
:10B8180084F88C30C4F89C20284A85F82430C4F871
:10B828009820274AC4F89420264AC4F8A020264A1B
:10B83800C4F8B420254AC4F8B020254AC4F8A42086
:10B84800244AC4F8A820244AC4F8C420234AC4F8C7
:10B85800C020234AC4F8D020224AC4F8CC20224A67
:10B86800C4F8C820214AC4F8DC204FF4F072C4E9B7
:10B8780021211F4AC4F8D4201E4AC4F8E8201E4AD1
:10B88800C4F8EC201D4C236898470021A36808469B
:10B89800BDE8F041184700BF9C64002064680020A0
:10B8A800488B0208A5B60008B81700206068002079
:10B8B800D1B40008C7B40008AFA90008C9A9000896
:10B8C800C5A90008C1A90008BDB40008A9B40008AA
:10B8D8009DA90008D5B6000891A900087DA900080F
:10B8E80035B600084DB500081FB600080DB50008AC
:10B8F8000DA90008F5B60008F5B50008800A002073
:10B9080070A302080022024BC3F88020704700BFD2
:10B918009C640020014813F01FBF00BFF0170020EF
:10B9280010B50348144613F04AFF206010BD00BF4D
:10B93800F017002038B51546044628B9084612F015
:10B9480025FE2860204638BD0420FCE710B50446D3
:10B9580018B912F0BFFD204610BD0820FCE710B54D
:10B96800044618B912F094FD204610BD0820FCE7E3
:10B978000021F4E74942F2E7F1E7014813F0DCBFA0
:10B98800F017002010B54FF4003012F0BFFF00236D
:10B99800054C1846D4E9A21212F01CFE2046BDE858
:10B9A800104013F0B2BF00BFF0170020022804BFF8
:10B9B8000C4B93F8F00038B90B4BDB681B685B69DC
:10B9C8000A4AD2F884021847012809D1054B93F88E
:10B9D800F030012B04D1044BDB681B689B69EFE74F
:10B9E800704700BF9C64002070A30208F017002075
:10B9F80038B50020FFF7DAFF144B154CDD68D4F892
:10BA080084022B689B6898472B68D4F888029B6847
:10BA180098472B68D4F88C029B6898472B68D4F811
:10BA280090029B6898472B68D4F894029B689847C3
:10BA38002B68D4F898029B6898472B68D4F89C0226
:10BA48009B689847BDE8384012F0DCBF70A3020835
:10BA5800F017002008B50146034813F00BFFBDE8B6
:10BA68000840002012F04CBDF017002038B50D46F4
:10BA7800044648B912F0AAFE2B68C118296020466E
:10BA880012F028FD204638BD0820FCE708B519BB90
:10BA9800052823D8DFE800F003090E22131B1146FE
:10BAA800002012F017FD002008BD1146002012F0FA
:10BAB80033FEF8E71146002012F0EAFCF3E782EAC9
:10BAC800E271A1EBE271002012F040FEEBE71146B3
:10BAD800002012F0BEFFE6E70820E5E70420E3E7D0
:10BAE80010B5144629BB062825D8DFE800F0040A5B
:10BAF8000E12161A1E00002012F076FE206000209A
:10BB080010BD002012F062FEF8E7002012F088FE57
:10BB1800F4E7002012F076FEF0E7002012F09CFE19
:10BB2800ECE7002012F08AFEE8E7044813F00DFF66
:10BB3800E4E70820E4E70420E2E700BFF01700206C
:10BB48000248DBB2D0F8A00211F05CB8F017002070
:10BB5800012213F0E5B8012270B5544E11460720B2
:10BB680013F082F8F568524C6B6803F5BA72C4F8A2
:10BB7800882203F5C872C4F88C2203F59072C4F8C1
:10BB8800902203F59E7203F1CC00C4F8942203F1CD
:10BB9800E80203F58273C4F89C322B68C4F8982233
:10BBA800DB68C4F8840298472B68D4F88802DB68FD
:10BBB80098472B68D4F88C02DB6898472B68D4F830
:10BBC8009002DB6898472B68D4F89402DB689847A2
:10BBD8002B68D4F898021B6998472B680025D4F87D
:10BBE8009C021B699847F36A0126C4F8A0321D70AD
:10BBF8005B6898472F4B3049D3F890203220C2F821
:10BC080004122E491680C2F808122D4983F88C6058
:10BC1800C3F89C102B49C3F898102B49C3F894100B
:10BC28002A49C3F8A0102A49C3F8B4102949C3F80F
:10BC3800B0102949C3F8A4102849C3F8A810284906
:10BC4800C3F8C4102749C3F8C0102749C3F8CC105B
:10BC58002649C3F8DC102649C3F8D8104FF4C3713D
:10BC6800C3E9211023492046C3F8D4102249C3F858
:10BC7800D0102946214B13F0E1FD4FF4003012F0AB
:10BC880045FED4E9A2122B46284612F0A3FC28460A
:10BC98004FF4484112F05AFD28464FF4484112F03B
:10BCA800D8FE3046BDE8704080E600BF70A30208A9
:10BCB800F01700209C6400208DB9000883B90008A3
:10BCC80067B9000881B900087DB9000879B900088A
:10BCD800E9BA000895BA000855B9000875BA00080D
:10BCE8001DB9000829B900083DB90008B5B9000810
:10BCF8000DB90008F9B900085DBA0008488D0208B6
:10BD08000022024BC3F88020704700BF9C640020CB
:10BD1800074870B550F8044B0D46164613F074FEEC
:10BD280033462A4601462046BDE8704010F0D5BF8C
:10BD3800A01A0020074870B550F8044B0D46164667
:10BD480013F062FE33462A4601462046BDE870409D
:10BD580010F07CBFA01A002038B51546044628B953
:10BD6800084612F013FC2860204638BD0420FCE782
:10BD780010B5044618B912F0ADFB204610BD0820D6
:10BD8800FCE710B5044618B912F082FB204610BD36
:10BD98000820FCE70021F4E74942F2E7F1E7024B0B
:10BDA800D3F8940213F028BEA01A002010B54FF45F
:10BDB800003012F0ABFD0023054C1846D4E9A71259
:10BDC80012F008FCD4F89402BDE8104013F00CBE41
:10BDD800A01A0020022804BF0C4B93F8F00038B9D1
:10BDE8000B4BDB681B685B690A4AD2F89802184754
:10BDF800012809D1054B93F8F030012B04D1044BED
:10BE0800DB681B689B69EFE7704700BF9C640020F4
:10BE180070A30208A01A002038B50020FFF7DAFF47
:10BE2800164B174CDD68D4F898022B689B68984726
:10BE38002B68D4F89C029B6898472B68D4F8A0021A
:10BE48009B6898472B68D4F8A4029B6898472B688E
:10BE5800D4F8A8029B6898472B68D4F8AC029B6872
:10BE680098472B68D4F8B0029B68984723689B686A
:10BE78009847BDE8384012F0C5BD00BF70A302085E
:10BE8800A01A002008B5064A0146D2F894320020CC
:10BE9800043213F09AFDBDE80840002012F030BBD0
:10BEA800A01A002038B50D46044648B912F08EFC99
:10BEB8002B68C1182960204612F00CFB204638BDBB
:10BEC8000820FCE708B549BB062829D8DFE800F0B8
:10BED800040A0F28141C21001146002012F0FAFA57
:10BEE800002008BD1146002012F016FCF8E71146A4
:10BEF800002012F0CDFAF3E782EAE271A1EBE271D9
:10BF0800002012F023FCEBE71146002012F0A1FDFF
:10BF1800E6E7D1B2034813F07AFDE1E70820E0E74D
:10BF28000420DEE7A41A002010B5144629BB062811
:10BF380025D8DFE800F0040A0E12161A1E000020A9
:10BF480012F052FC2060002010BD002012F03EFCD0
:10BF5800F8E7002012F064FCF4E7002012F052FC2D
:10BF6800F0E7002012F078FCECE7002012F066FC05
:10BF7800E8E7044813F048FDE4E70820E4E7042074
:10BF8800E2E700BFA41A0020012270B5524C114606
:10BF9800524E072012F068FE201D13F0D9FCF568F8
:10BFA8006B6803F5BA72C4F89C2203F5C872C4F82A
:10BFB800A02203F59072C4F8A42203F59E7203F13F
:10BFC800CC00C4F8A82203F1E80203F58273C4F890
:10BFD800B0322B68C4F8AC22DB68C4F898029847E2
:10BFE8002B68D4F89C02DB6898472B68D4F8A00229
:10BFF800DB6898472B68D4F8A402DB6898472B685D
:10C00800D4F8A802DB6898472B68D4F8AC021B69FF
:10C0180098472B680125D4F8B0021B699847F36A42
:10C0280023605B6898472E4B2E49D3F890204FF435
:10C038000030C2F804122C491580C4F89422C2F8C2
:10C0480008122A4A3221C3F89C20294A83F88C50C6
:10C05800C3F89820274AC3F89420274AC3F8A02099
:10C06800264AC3F8B420264AC3F8B020254AC3F8A4
:10C07800A420254AC3F8A820244AC3F8C420244A87
:10C08800C3F8C020234AC3F8CC20234AC3F8DC20D5
:10C09800224AC3F8D8204FF4C372C3E92121204AA9
:10C0A800C3F8D4201F4AC3F8D02012F02FFCD4E9DB
:10C0B800A7120023184612F08DFA4FF448410020C9
:10C0C80012F044FB00204FF4484112F0C2FC28460D
:10C0D800BDE870407EE600BFA01A002070A30208E9
:10C0E8009C640020B5BD0008A7BD00088BBD0008F2
:10C0F800A5BD0008A1BD00089DBD000831BF00080E
:10C10800CDBE000879BD0008ADBE000819BD000805
:10C118003DBD000861BD0008DDBD000809BD00087F
:10C1280021BE00088DBE00080022024BC3F8802003
:10C13800704700BF9C640020014813F06BBC00BF2F
:10C14800601D002010B50348144613F096FC2060CB
:10C1580010BD00BF601D002010B5044618B912F0CC
:10C16800B9F9204610BD0820FCE710B5044618B9F7
:10C1780012F08EF9204610BD0820FCE70021F4E7F4
:10C188004942F2E7F1E7F8B506461D460C46002994
:10C1980040F06E82332A00F0228140D8052A00F050
:10C1A800C08017D8022A00F0A58007D8002A00F01E
:10C1B8008C80012A00F09480042624E1032A00F0F0
:10C1C800A280042AF8D1002840F0A380002012F0B1
:10C1D80043FB7DE0082A00F0CB800ED8062A00F049
:10C1E800A980072AE8D11021BA48002E40F0B8806B
:10C1F80013F043FC00F01F006AE01D2A00F0CD8018
:10C20800322A00F0E2801C2AD6D1002840F0B880FB
:10C218000146B04813F031FCC0F3400058E0B42A9E
:10C2280000F0AE8123D8A52A00F033810ED88C2ADD
:10C2380000F0DE80A22ABFD16C21A648002E40F073
:10C248001F8113F01AFCC0F3C13041E0A72A00F0A7
:10C258007E81C0F04381B32AAED16C219D48002E67
:10C2680040F0858113F009FCC0F3404030E0BB2A60
:10C2780000F0AA8117D8B52A00F08C81BA2A9BD180
:10C28800002840F092811321924813F0F6FB002811
:10C2980000F089814FF0807393FBF0F08E4B984249
:10C2A800A8BF184614E1C02A00F0BF81CC2A00F0CC
:10C2B800CE81BF2A80D1002840F0A6817021854810
:10C2C80013F0DBFBC0F3014002E018B912F08CFA5E
:10C2D800286098E01968104612F0FCF8002692E0F1
:10C2E80018B9002012F072FAF2E71968002012F06B
:10C2F80013FAF3E710B912F093FAE9E71968204640
:10C3080012F0C6F8EAE700287FF456AF12F07AFA7E
:10C31800DEE7196800200029B8BF494212F016FA72
:10C32800DCE710B912F08AFAD2E71968204612F051
:10C3380090FBD3E71021674826B913F09EFBC0F3A2
:10C348000420C5E713F099FB2B6820F4F8521B0270
:10C3580003F4F85310211A435E4813F05BFBBDE762
:10C3680013F08BFB2B6820F01F0203F01F03F1E78B
:10C3780000287FF421AF12F009F9C0F30010A7E7F5
:10C388000021544813F079FB2B6820F002025B006F
:10C3980003F002031A430021DEE700287FF40CAF04
:10C3A80012F084FA122104464A4813F066FBC0F3DF
:10C3B80013027A20D317A4FB00011BF0CFFE00F173
:10C3C8001303262B98BF002082E718B9002012F02B
:10C3D8005FFA7DE71978002012F0D2F97EE710B9EC
:10C3E80012F064FA74E71968204612F0D9F975E773
:10C3F80058B96C21374813F040FB4FF48073C0F3F1
:10C40800036003412B603046F8BD1B68102B31D008
:10C418000FDC022B2AD006DC012B18D04FF0FF339B
:10C428002B601026EFE7042B22D0082BF6D105232A
:10C438000EE0402B20D003DC202BEFD1032307E0B4
:10C44800802B1BD0B3F5807FE8D1002300E00823C0
:10C458002B606C211F4813F010FB2B6820F07062D2
:10C468001B0603F070631A436C2175E70723EFE797
:10C478000623EDE70423EBE70223E9E70123E7E7D7
:10C4880013F0FBFA2B6820F4C032DB0303F4C0334B
:10C49800E9E700287FF490AE6C210E4813F0EDFA1E
:10C4A80010F480444FF06C010A4804D013F0E5FA08
:10C4B800C0F3C3100CE713F0E0FA6C2106460548F8
:10C4C80013F0DBFAC0F30210330548BF40F0080050
:10C4D800286003E7601D0020FFFF0F006C216548FE
:10C4E800B6B913F0CAFA10F480444FF06C016148F1
:10C4F80004D013F0C2FAC0F30210E9E613F0BDFA53
:10C508006C2106465B4813F0B8FAC0F3C310DBE7AA
:10C5180013F0B3FA10F480464FF06C01554808D078
:10C5280013F0ABFA2B6820F070021B0103F07003C4
:10C5380099E713F0A2FA2B6820F4F062DB0103F408
:10C54800F0631A436C214B4813F064FA5BE76C21E3
:10C55800484826B913F091FA00F00F00B8E613F036
:10C568008CFA2B6820F00F0203F00F037BE713F01F
:10C5780084FA2B6820F400325B0403F4003372E77A
:10C5880000287FF419AE6F213A4813F076FAC0F309
:10C5980004409DE610B912F06DF999E61968204635
:10C5A80012F0E0F89AE6344892E71B6853B14FF06E
:10C5B800807292FBF3F2304B9A42A8BF1A462A6067
:10C5C8001321C9E62C4AFAE770212A4826B913F044
:10C5D80054FAC0F307207BE613F04FFA2A6820F4D8
:10C5E8007F40120292B202437021224813F012FADD
:10C5F8002146204813F041FA2B6820F00402002B52
:10C60800D4BF04230023C5E61B68032B3FF609AFFC
:10C618007021184813F031FA2B6820F440321B04BB
:10C6280003F440331A43702196E67021114826B965
:10C6380013F023FAC0F380404AE613F01EFA2B6881
:10C6480020F48022002B18BF4FF48023EAE77021E2
:10C65800084826B913F011FAC0F3015038E613F070
:10C668000CFA2B6820F440121B0503F44013D9E799
:10C678000826C8E6601D0020FFFF0F0007B50192DD
:10C6880001AB02460120FFF77EFD03B05DF804FB15
:10C6980013460246002076E5014813F0ABBA00BF06
:10C6A800601D002010B54FF4003012F02FF9002360
:10C6B800054C1846D4E9A31211F08CFF2046BDE8BA
:10C6C800104013F080BA00BF601D0020022804BF8C
:10C6D8000C4B93F8F00038B90B4BDB681B685B69AF
:10C6E8000A4AD2F888021847012809D1054B93F85D
:10C6F800F030012B04D1044BDB681B689B69EFE722
:10C70800704700BF9C64002070A30208601D0020D1
:10C7180038B50020FFF7DAFF144B154CDD68D4F864
:10C7280088022B689B6898472B68D4F88C029B6812
:10C7380098472B68D4F890029B6898472B68D4F8E0
:10C7480094029B6898472B68D4F898029B6898478E
:10C758002B68D4F89C029B6898472B68D4F8A002F1
:10C768009B689847BDE8384012F04CB970A302089E
:10C77800601D002008B50146034813F0D9F9BDE84B
:10C788000840002011F0BCBE601D002010B5144602
:10C79800042828D8DFE800F003080E121A0008461B
:10C7A80011F0F4FE206003E01178104813F02BFA22
:10C7B800002010BD0D4813F029FAF3E70C4B0220B6
:10C7C800DB6898476423B0FBF3F0EBE742F21071A3
:10C7D8001368022059436423B1FBF3F1044B89B277
:10C7E8009B689847E4E70420E3E700BF601D00204A
:10C7F800800A002038B50D46044648B911F0E6FF16
:10C808002B68C1182960204611F064FE204638BD07
:10C818000820FCE70248DBB2D0F8A80210F0F2B911
:10C82800601D0020012212F07BBA0122F8B5604E8B
:10C838001146072012F018FAF5685E4C6B6802275B
:10C8480003F5BA72C4F88C2203F5C872C4F89022B2
:10C8580003F59072C4F8942203F59E72C4F89822E6
:10C8680003F1E80203F1CC00C4F89C2203F58272BC
:10C8780003F5E473C4F8A4322B68C4F8A022DB687B
:10C88800C4F8880298472B68D4F88C02DB6898476C
:10C898002B68D4F89002DB6898472B68D4F8940288
:10C8A800DB6898472B68D4F89802DB6898472B68B0
:10C8B800D4F89C021B6998472B68D4F8A0021B691E
:10C8C8009847F36A0126C4F8A8321E705B68984737
:10C8D800394B3A49D3F890203220C2F8041238492B
:10C8E8001680C2F80812374983F88C60C3F89C1088
:10C8F8003549C3F898103549C3F894103449C3F83A
:10C90800A0103449C3F8B4103349C3F8B010334900
:10C91800C3F8A4103249C3F8A8103249C3F8C410A8
:10C928003149C3F8C0103149C3F8CC103049C3F8B5
:10C93800DC103049C3F8D8104FF4C371C3E9211093
:10C948002D492046C3F8D4102C49C3F8D0102C4BDD
:10C95800002113F0D1F84FF4003011F0D7FFD4E9DB
:10C96800A3120023184611F035FE4FF44841002069
:10C9780011F0ECFE4FF44841002012F06AF8D4F8A8
:10C98800A4323246197C5F74186817F052FD2B6880
:10C99800D4F8A4021B4C1B6898472368984738466C
:10C9A800A36841F64C5198473046BDE8F8408DE6FB
:10C9B80070A30208601D00209C640020ADC600081A
:10C9C800A1C6000873C100088DC1000889C100080C
:10C9D80085C1000899C6000885C6000861C100081D
:10C9E800FDC7000841C100084DC1000895C70008EF
:10C9F800D5C6000831C1000819C700087DC700085E
:10CA0800488F0208800A0020012810B514460DD06E
:10CA180043B21BB1022810D0042010BD1268094986
:10CA2800B2FA82F252090A710020F6E71368064A40
:10CA3800B3FA83F35B091360F6E7084611F0A6FD25
:10CA48002060F1E7182000206400002010B503489A
:10CA5800144613F027F9206010BD00BF18200020ED
:10CA680070B5164C0146204613F066F9002011F007
:10CA780047FD002011F0C6FEA3680028B8BF404259
:10CA8800984234BF0026012694F84020B24213D0C1
:10CA980098424FF0050109482CBFA579657913F034
:10CAA80001F905F00F0520F00F022A43052103487C
:10CAB80013F0E6F884F8406070BD00BF182000202D
:10CAC800014813F0DDB800BF1820002010B5044657
:10CAD80018B911F0FFFC204610BD0820FCE710B57E
:10CAE800044618B911F0D4FC204610BD0820FCE714
:10CAF8000021F4E74942F2E7F1E770B504461D4624
:10CB08000E46002940F03283A72A00F0148267D825
:10CB18001D2A00F0028122D8042A00F005810DD8D0
:10CB2800012A00F0E880002A00F0D980022A00F0EB
:10CB3800EB80032A00F0F18004245EE1062A00F06D
:10CB48000981C0F0FD80072A00F01A81082AF3D174
:10CB58000028F1D111F01AFDC0F30010C3E0A12A9A
:10CB680000F086811AD8332A00F0278107D8322AA4
:10CB7800E2D1002840F01C8111F08AFEB3E08C2A33
:10CB880000F02481A02AD7D1002840F06481082130
:10CB9800B64813F087F8C0F34020A4E0A42A00F0B8
:10CBA80099810ED8A22A00F07581A32AC4D1002841
:10CBB80040F085810C21AD4813F074F8C0F3803043
:10CBC80091E0A52A00F09981A62AB5D1002840F065
:10CBD800A7810C21A54813F065F8C0F3021082E084
:10CBE800B22A00F0458241D8AC2A00F0F48113D86B
:10CBF800A92A00F0C581C0F0B081AA2A00F0D1812D
:10CC0800AB2A99D105219948002C40F0DB8113F01B
:10CC180049F8C0F3411066E0AF2A00F0FD8115D84D
:10CC2800AD2A00F0DF81AE2A86D106218F48002C7C
:10CC380040F0E98113F036F8000A00F07F0310F0A5
:10CC4800400018BF6FF07F0018434CE0B02A00F096
:10CC5800F581B12A7FF470AF07218448002C40F099
:10CC6800FE8113F01FF8C0F380203CE0B72A00F0E3
:10CC7800378210D8B42A00F01D82C0F00A82B52A83
:10CC880000F02282B62A7FF457AF784B002840F094
:10CC980024829B6861E0CE2A00F0468213D8B82A25
:10CCA80000F02E82B92A7FF447AF07216F48002C85
:10CCB80000F09B8112F0F6FF2B6820F480321B04F1
:10CCC80003F48033B7E1D02A00F04482D62A7FF4F7
:10CCD80033AF664B002840F046821B693DE020B91F
:10CCE800002011F081FD286087E01968002011F00C
:10CCF800F1FB002481E010B911F068FDF3E7196831
:10CD0800304611F009FDF4E710B911F089FDEAE7A2
:10CD18001968002011F0BCFBEBE7002C7FF40CAF86
:10CD2800204611F06FFDDEE710B911F095FDDAE746
:10CD3800196830460029B8BF494211F007FDD8E705
:10CD480018B9002011F07AFDCDE71968002011F01C
:10CD580080FECEE7454E10B9737B2B604DE01B6813
:10CD68007373337B002BC4D10621404812F09AFF1D
:10CD7800737B20F01F0203F01F031A430621FDE016
:10CD88003A4E08B9B37BE8E71B68B373337B012BD2
:10CD9800AFD10621304612F085FF062120F01F0290
:10CDA8003046B37B03F01F031A4312F069FFA0E774
:10CDB8001978002011F0E4FC9BE710B911F076FD1A
:10CDC80091E71968304611F0EBFC92E740B9082169
:10CDD800264812F067FF00F00F00C0F1080082E754
:10CDE8001B68102B31D010DC022B2AD007DC012B5A
:10CDF80019D04FF0FF3310242B60204670BD042B50
:10CE080021D0082BF5D105230EE0402B1FD003DCE1
:10CE1800202BEED1032307E0802B1AD0B3F5807FB7
:10CE2800E7D1002300E008232B6000210F4812F00F
:10CE380039FF2B6820F00F0203F00F031A4300217B
:10CE48009CE00723F0E70623EEE70423ECE7022340
:10CE5800EAE70123E8E70021044812F023FF2B68E2
:10CE680020F400725B0203F40073E7E71820002047
:10CE780030B90821AB4812F015FFC0F3002032E7A3
:10CE8800A84812F00FFF2B6820F480721B0203F4ED
:10CE98008073D3E730B90C21A24812F003FFC0F326
:10CEA800C13020E704219F4812F0FCFE2B6820F4D3
:10CEB800C032DB0303F4C0331A4304215EE00421CB
:10CEC800984812F0EFFE2B6820F480429B0303F48D
:10CED8008043F1E730B90C21924812F0E3FEC0F329
:10CEE800C12000E704218F4812F0DCFE2B6820F4F3
:10CEF800C052DB0203F4C053DEE730B90C21894885
:10CF080012F0D0FEC0F3C310EDE60421854812F0FC
:10CF1800C9FE2B6820F4F062DB0103F4F063CBE771
:10CF28000421804812F0BEFE2B6820F070021B011D
:10CF380003F07003C0E730B90C217A4812F0B2FE52
:10CF480000F00F00CFE60421764812F0ABFE2B6804
:10CF580020F00F0203F00F03AEE70521714824B952
:10CF680012F0A0FEC0F3C030BDE612F09BFE2B68A5
:10CF780020F40042DB039BB205211A43694814E7F9
:10CF88000521684824B912F08DFEC0F34130AAE6A5
:10CF980012F088FE2B6820F4C0425B0303F4C04300
:10CFA800EAE705215F4824B912F07CFEC0F30320AC
:10CFB80099E612F077FE2B6820F470621B0203F4E6
:10CFC8007063D9E712F06EFE2B6820F060025B01F7
:10CFD80003F06003D0E7534B08B99B79BDE62A6894
:10CFE8009A7186E606214F4824B912F05BFEC0F319
:10CFF800004078E612F056FE2B6820F480321B04BD
:10D0080003F48033B9E612F04DFE2B6820F4FE429B
:10D018001B0203F4FE43B0E60721424824B912F08C
:10D0280041FEC0F381305EE612F03CFE2B6820F42E
:10D0380040429B039BB21A4307219FE707213948C7
:10D0480024B912F02FFEC0F301304CE612F02AFE8C
:10D058002B6820F440521B0303F44053EBE712F013
:10D0680021FE2B6820F480629B0203F48063E2E7D0
:10D0780007212C4824B912F015FEC0F3012032E62E
:10D0880012F010FE2B6820F440721B0203F4407368
:10D09800D1E70721234824B912F004FEC0F3801019
:10D0A80021E612F0FFFD2B6820F040029B0103F0FF
:10D0B8004003C0E700287FF43FAD0221194812F071
:10D0C800F1FDC0F384200EE610B911F0D3FB0AE697
:10D0D8001968002011F046FB0BE62A689A6008E6FA
:10D0E8000721104824B912F0DDFDC0F3C010FAE59D
:10D0F80012F0D8FD2B6820F08002DB01DBB29AE742
:10D108000421084824B912F0CDFDC0F34030EAE507
:10D1180012F0C8FD2B6820F400525B0303F400539F
:10D12800CAE600BF1820002000287FF405AD104B88
:10D138001B6843B102210F4812F0B4FD800A00F4C5
:10D1480078702860D5E501210A4812F0ABFDC0F3DC
:10D158008920F6E700287FF4EFAC0321054812F098
:10D16800A1FDC0B2BFE52A681A61C2E5082444E6F9
:10D17800640000201820002007B5019201AB024688
:10D188000120FFF7BAFC03B05DF804FB1346024622
:10D198000020B2E4014812F041BE00BF1820002070
:10D1A800022804BF0B4B93F8F00030B90A4BDB6838
:10D1B8001B685B69094A106D1847012809D1054B9E
:10D1C80093F8F030012B04D1034BDB681B689B6993
:10D1D800F0E770479C64002070A302081820002024
:10D1E80038B50020FFF7DCFF0F4B104CDD68206DD1
:10D1F8002B685B6998472B68606C9B6898472B681D
:10D20800E06C9B6898472B68206D9B6898472B6853
:10D21800606D9B6898472B68A06C9B689847BDE831
:10D22800384011F0EFBB00BF70A30208182000209F
:10D238000346052B10B5084614460BD006D8022B1A
:10D2480006D311F033FB2060002010BD182BF8D056
:10D258000420FAE711F044FBF5E738B50D4604461B
:10D2680020B911F0CFFA2860204638BD0820FCE725
:10D2780070B5002011F0C6FA0646A8B901240B4D76
:10D28800284612F0AFFD0A4B02201C60FFF788FF0A
:10D298004FF4003011F03AFBD5E9121230466B6DAD
:10D2A80011F098F9204670BD0020FCE718200020F6
:10D2B8006400002038B50D46044648B911F086FAD6
:10D2C8002B68C1182960204611F004F9204638BDA2
:10D2D8000820FCE7022806D3052801D9182802D11E
:10D2E80000201060704704207047054B0846DB6E2D
:10D2F800114603B11847034BDB6DDB68FAE700BF43
:10D308009C640020182000202DE9F0410127474C9B
:10D31800474D484BDFF8708100211F60D4F89020FA
:10D328002846454B12F0E3FCD8F80C60736803F10B
:10D33800CC022A6503F1E80203F5BA706A6503F5C1
:10D34800C87203F50E736B643368EA64DB68A8641B
:10D3580098473368E86CDB6898473368286DDB6862
:10D3680098473368686D1B6998473368686CDB6851
:10D3780098477068336824309B68A8659847D8F840
:10D3880010304FF4003003F11402EA656A6C9A61B8
:10D3980011F0BCFAD5E912126B6D002011F01AF9E0
:10D3A800D4F89030254A84F88C70C3F80822244AAF
:10D3B8000220C3F80422234B3222C4F89C30224BAB
:10D3C800C4F89830214BC4F89430214BC4F8A030ED
:10D3D800204BC4F8B430204BC4F8B0301F4BC4F80D
:10D3E800A4301F4BC4F8A8301E4BC4F8C4301E4BE1
:10D3F800C4F8C0301D4BC4F8D0301D4BC4F8CC3035
:10D408001C4BC4F8C8301C4BC4F8DC304FF41673FE
:10D41800C4E92132194BC4F8D430194BC4F8E830A8
:10D42800184BC4F8EC30BDE8F041B9E69C64002024
:10D438001820002064000020489102089DD10008AF
:10D4480079D20008E7CA000801CB0008FDCA000825
:10D45800F9CA000895D1000881D10008D5CA00088A
:10D46800BDD20008C9CA000855CA000869CA000820
:10D4780011CA000863D20008A9D10008E9D1000840
:10D48800DDD2000839D2000870A30208012810B5BF
:10D4980014460DD043B21BB1022810D0042010BD91
:10D4A80012680949B2FA82F252098A720020F6E734
:10D4B8001368064AB3FA83F35B091360F6E7084674
:10D4C80011F064F82060F1E7842000206800002053
:10D4D80010B5044618B910F0FDFF204610BD08200D
:10D4E800FCE7024B986C12F050BD00BF842000206E
:10D4F800022804BF0B4B93F8F00030B90A4BDB68E5
:10D508001B685B69094A906D1847012809D1054BCA
:10D5180093F8F030012B04D1034BDB681B689B693F
:10D52800F0E770479C64002070A302088420002064
:10D5380038B50020FFF7DCFF0F4B104CDD68A06DFD
:10D548002B685B6998472B68E06C9B6898472B6849
:10D55800606D9B6898472B68A06D9B6898472B68FF
:10D56800E06D9B6898472B68206D9B689847BDE8DD
:10D57800384011F047BA00BF70A302088420002089
:10D5880038B50D46044620B911F03CF9286020460C
:10D5980038BD0820FCE710B5044628B9034B1881AC
:10D5A80010F076FF204610BD0820FCE784200020FC
:10D5B8000021F0E74942EEE7EDE770B5002011F0F1
:10D5C80021F90646B0B901240B4DA96C284612F082
:10D5D800BFFC0A4B02201C60FFF78AFF4FF40030A3
:10D5E80011F094F9D5E914123046EB6D10F0F2FF02
:10D5F800204670BD0020FCE7842000206800002041
:10D6080038B50D46044648B911F0E0F82B68C11842
:10D618002960204610F05EFF204638BD0820FCE750
:10D6280038B51F4C0546636E00219B68C0F3074060
:10D63800984794F86820A36C000203EB82035860B3
:10D64800636E00219B68C5F30720984794F86830FB
:10D65800A26C012102EB830253681843636E000237
:10D6680050609B68E8B29847A26C94F8681002EB87
:10D6780081014B6818430011AB0C486010610AD057
:10D68800C5F34243072B03D1C5F3011184F8681091
:10D6980043F0080300E0082302EB83035D6038BD14
:10D6A8008420002010B40A4C00F07702A36C42F0EA
:10D6B800080203EB8203C1F313015960A37A23B96B
:10D6C80041EA404010BCFFF7ABBF10BC704700BF39
:10D6D8008420002008461146E4E738B504460F20A8
:10D6E80000F013F80323B4FBF3F3054603EB4303FD
:10D6F800E41AE4B220F0300040EA0410FFF790FF8B
:10D708002846BDE83840FFF78BBF38B5084D00F014
:10D718000802A97A044651EA020301D1FFF7DDFFA6
:10D72800AB6C04F07F0403EB8404606838BD00BF71
:10D738008420002070B504461D460E46002940F09E
:10D748002E83A72A00F0028264D81D2A00F0F380F5
:10D7580022D8042A00F0F6800DD8012A00F0D980DA
:10D76800002A00F0CA80022A00F0DC80032A00F0B8
:10D77800E280042418E1062A00F0FA80C0F0EE8066
:10D78800072A00F02081082AF3D10028F1D110F0EF
:10D79800FDFEC0F30010B4E0A12A00F0838119D87F
:10D7A800332A00F02B8107D8322AE2D1002840F032
:10D7B800208111F06DF8A4E08C2A00F02881A02ABD
:10D7C800D7D10820002C40F06481FFF79EFFC0F3FA
:10D7D800402096E0A42A00F090810DD8A22A00F0FB
:10D7E8007181A32AC5D10C20002C40F07D81FFF760
:10D7F8008CFFC0F3803084E0A52A00F08E81A62A31
:10D80800B7D10C20002C40F09881FFF77EFFC0F3C1
:10D81800021076E0B22A00F041823ED8AC2A00F02D
:10D82800E98112D8A92A00F0B981C0F0A381AA2AF7
:10D8380000F0C581AB2A9CD1002840F0D181052099
:10D84800FFF763FFC0F341105BE0AF2A00F0F981F6
:10D8580014D8AD2A00F0DA81AE2A8AD1002840F027
:10D86800E6810620FFF751FF000A00F07F0310F061
:10D87800400018BF6FF07F00184342E0B02A00F064
:10D88800F281B12A7FF475AF002840F0FD810720AE
:10D89800FFF73BFFC0F3802033E0B72A00F0358262
:10D8A80010D8B42A00F01C82C0F00982B52A00F012
:10D8B8002082B62A7FF45DAFAC4B002840F022826C
:10D8C8001B6958E0CE2A00F04B820AD8B82A00F02B
:10D8D8002C82B92A7FF44DAF002840F03782072008
:10D8E80096E1D02A00F05082D62A7FF442AF9F4BAF
:10D8F800002840F051825B683DE020B9002010F01C
:10D9080073FF286050E01968002010F0E3FD002440
:10D918004AE010B910F05AFFF3E71968304610F0E2
:10D92800FBFEF4E710B910F07BFFEAE71968002066
:10D9380010F0AEFDEBE7002C7FF41BAF204610F093
:10D9480061FFDEE710B910F087FFDAE719683046A3
:10D958000029B8BF494210F0F9FED8E718B90020ED
:10D9680010F06CFFCDE71968002011F072F8CEE7CF
:10D978007E4E10B9F37A2B6016E01B68F3727C4B6D
:10D98800DB6E9BB90020FFF7C0FE10F08004BED10B
:10D998000E20FFF7BAFEF37A20F01F0103F01F03F1
:10D9A80019430E20FFF77EFE204670BD2B680E201F
:10D9B8003370FFF7AAFEF37A20F01F0103F01F036C
:10D9C80019430E20E7E0694E08B93378D3E71B689E
:10D9D8003370674BDC6E4CB92046FFF796FE0306A2
:10D9E80095D50E20FFF791FE3378D5E72B68F372B3
:10D9F8008DE71978002010F0C3FE88E710B910F001
:10DA080055FF7EE71968304610F0CAFE7FE738B93F
:10DA18000820FFF77AFE00F00F00C0F1080070E759
:10DA28001B68102B2FD00FDC022B28D006DC012B13
:10DA380018D04FF0FF3310242B60B5E7042B20D00B
:10DA4800082BF6D105230EE0402B1ED003DC202B3B
:10DA5800EFD1032307E0802B19D0B3F5807FE8D1FD
:10DA6800002300E008232B600820FFF74EFE2B68F8
:10DA780020F00F0103F00F03194308208BE0072360
:10DA8800F1E70623EFE70423EDE70223EBE70123A1
:10DA9800E9E7FFF73AFE2B6820F400715B0203F414
:10DAA8000073E9E7082024B9FFF72FFEC0F3002030
:10DAB80027E7FFF72AFE2B6820F480711B0203F486
:10DAC8008073D9E70C2024B9FFF71FFEC0F3C130DB
:10DAD80017E7FFF71AFE2B6820F4C031DB0303F4C5
:10DAE800C03319430C2056E0FFF70FFE2B6820F4D3
:10DAF80080419B0303F48043F3E70C2024B9FFF72C
:10DB080004FEC0F3C120FCE6FFF7FFFD2B6820F4FC
:10DB1800C051DB0203F4C053E3E70C2024B9FFF73C
:10DB2800F4FDC0F3C310ECE6FFF7EFFD2B6820F41B
:10DB3800F061DB0103F4F063D3E7FFF7E6FD2B6840
:10DB480020F070011B0103F07003CAE70C2024B910
:10DB5800FFF7DBFD00F00F00D3E6FFF7D6FD2B68DB
:10DB680020F00F0103F00F03BBE700BF8420002063
:10DB78009C64002028B90520FFF7C7FDC0F3C0301A
:10DB8800BFE60D20FFF7C1FD2B6820F40041DB0341
:10DB98009BB20D201943FFF785FDB8E628B905208B
:10DBA800FFF7B3FDC0F34130ABE60D20FFF7ADFD45
:10DBB8002B6820F4C0415B0303F4C043E9E728B9AC
:10DBC8000520FFF7A2FDC0F303209AE60D20FFF71A
:10DBD8009CFD2B6820F470611B0203F47063D8E786
:10DBE8000D20FFF792FD2B6820F060015B0103F028
:10DBF8006003CEE708B90520AAE70D20FFF785FDE9
:10DC08002B6820F00F0103F00F03C2E728B90620A4
:10DC1800FFF77BFDC0F3004073E60E20FFF775FDAC
:10DC28002B6820F480311B0403F48033C8E60E20EF
:10DC3800FFF76BFD2B6820F4FE411B0203F4FE4343
:10DC4800BEE628B90720FFF760FDC0F3813058E62B
:10DC58000F20FFF75AFD2B6820F440419B039BB22D
:10DC680019430F2097E728B90720FFF74EFDC0F3A7
:10DC7800013046E60F20FFF748FD2B6820F440519D
:10DC88001B0303F44053EBE70F20FFF73EFD2B681F
:10DC980020F480619B0203F48063E1E728B9072040
:10DCA800FFF733FDC0F301202BE60F20FFF72DFD12
:10DCB8002B6820F440711B0203F44073D0E728B9A5
:10DCC8000720FFF722FDC0F380101AE60F20FFF7A8
:10DCD8001CFD2B6820F040019B0103F04003BFE7C7
:10DCE80000287FF446AD0220FFF70FFDC0F3842023
:10DCF80007E610B910F0BEFD03E61968002010F021
:10DD080031FD04E62A681A6101E628B90720FFF701
:10DD1800FCFCC0F3C010F4E50F20FFF7F6FC2B68FD
:10DD280020F08001DB01DBB29AE728B90420FFF775
:10DD3800ECFCC0F34030E4E50C20FFF7E6FC2B6870
:10DD480020F400515B0303F40053CAE60F20FFF7E9
:10DD5800DCFC2B6820F480311B0403F480337FE75C
:10DD680000287FF406AD0F4B1B683BB10220FFF77C
:10DD7800CCFC800A00F478702860C8E50120FFF721
:10DD8800C4FCC0F38920F7E700287FF4F2AC032035
:10DD9800FFF7BBFCC0B2B4E52A685A60B7E50824AF
:10DDA80002E600BF6800002007B5019201AB0246F9
:10DDB8000120FFF7BFFC03B05DF804FB13460246E1
:10DDC8000020B7E410B508461446FFF79EFC206013
:10DDD80010BDF8B5364D0646E86E364CE8B9FFF783
:10DDE80094FC94F86930C0F3C017BB4215D00E20DC
:10DDF800002F4CD0FFF789FC00F01F00E0720E20C6
:10DE0800FFF783FC237803F01F0320F01F01194359
:10DE18000E20FFF747FC84F86970227AD5F8803025
:10DE2800002A3ED043F00103627A002A3CD043F036
:10DE380002030020C5F8803010F0E4FC23690028B4
:10DE4800B8BF4042984234BF0027012794F86A209F
:10DE5800BA4211D098424FF00D002CBF657B257B4C
:10DE6800FFF753FC05F00F0520F00F0129430D20A3
:10DE7800FFF718FC84F86A70A36C314600200D4A3D
:10DE880012F011F8BDE8F840002010F039BBFFF798
:10DE98003CFC00F01F0020700E20FFF736FCE37AF0
:10DEA800B1E723F00103BFE723F00203C1E700BF96
:10DEB8009C640020842000200A4810B4836C01F080
:10DEC800770444F0080403EB8403C2F313025A6096
:10DED800837A23B942EA414010BCFFF7A1BB10BCCA
:10DEE800704700BF8420002038B5094D01F00802B2
:10DEF8000C46A97A51EA020302D12046FFF7EDFB4E
:10DF0800A96C04F07F0401EB8404606838BD00BF8D
:10DF18008420002038B50D461E4C0021636EC5F3E1
:10DF280007409B68984794F86B20A36C000203EBAA
:10DF380082035860636E00219B68C5F307209847E9
:10DF480094F86B30A26C012102EB830253681843EA
:10DF5800636E000250609B68E8B29847A26C94F820
:10DF68006B1002EB81014B6818430011AB0C486041
:10DF780010610AD0C5F34243072B03D1C5F3011141
:10DF880084F86B1043F0080300E0082302EB8303D6
:10DF98005D6038BD84200020F8B50126454C464B0D
:10DFA800464F20461E6011F05BFFFD686B6803F169
:10DFB800CC02A26503F1E80203F5BA70E26503F545
:10DFC800C87203F50E73E3642B686265DB6820652D
:10DFD80098472B68606DDB6898472B68A06DDB68F5
:10DFE80098472B68E06D1B6998472B68E06CDB68E5
:10DFF800984768682B6824309B68206698473B6977
:10E008004FF4003003F114026266E26C9A61052352
:10E0180023704FF47A73636010F078FCD4E914121B
:10E02800E36D002010F0D6FA254B2649D3F890204E
:10E038000220C2F808122449A264C2F8041200217E
:10E048001180224A3221C3F89C20214A83F88C602F
:10E05800C3F898201F4AC3F894201F4AC3F8A02089
:10E068001E4AC3F8B4201E4AC3F8B0201D4AC3F89C
:10E07800A4201D4AC3F8A8201C4AC3F8C4201C4A7F
:10E08800C3F8C0201B4AC3F8D0201B4AC3F8CC20D1
:10E098001A4AC3F8C8201A4AC3F8DC204FF416728B
:10E0A800C3E92121174AC3F8D420BDE8F840FFF797
:10E0B8001FBA00BF842000206800002070A3020857
:10E0C8009C640020EBD40008C3D500089FD5000845
:10E0D800C1D50008BDD50008B9D50008C5DD0008C0
:10E0E800B1DD0008D9D4000809D60008DDD600083B
:10E0F800CDDD0008DBDD000895D4000889D50008CF
:10E10800F9D4000839D500080022014B9A607047FD
:10E118009C64002070B5184E184CF56860682B6830
:10E128009B6998472B68A0699B6898472B6860692A
:10E138009B6898472B6820699B6898472B68E0681C
:10E148009B6898472B68A0689B6898472B68206A4B
:10E158009B6898472B68E0699B6898472B682068FC
:10E168009B6898472B6860689B6898473369BDE847
:10E1780070405B6A184700BF70A30208FC200020AB
:10E18800022870B5144648D005D898B1012835D072
:10E198000424204670BD03284DD0FF28F8D12A4C0E
:10E1A800D4F89030D3F804329847A369D3F80432EE
:10E1B800984714E0126832F0030310D1234B244D22
:10E1C800DE68D207686933680BD51B6998472468ED
:10E1D800326814F00204A86909D01369984700242A
:10E1E800D7E7DB689847336868699B69EEE7D368C7
:10E1F80098473368A8699B699847CAE7134B144D39
:10E20800DE681468286933680CB11B69E6E7DB68C7
:10E218009847336828699B69EEE70C4B0C4DDE681C
:10E2280014683368A868002CEFD1DB689847336816
:10E23800A8689B69E0E70121064811F0D9FF206032
:10E248000028CCD12024A4E79C64002070A30208F5
:10E25800FC200020202100200146014812F086B849
:10E268002021002010B50348144611F0F0FE20606C
:10E2780010BD00BF20210020014811F0DABE00BF08
:10E288002021002008B50448D0F8B822243011F025
:10E298009FFF002008BD00BFFC20002008B50448EF
:10E2A800D0F8B822243011F077FF002008BD00BF55
:10E2B800FC20002070B504461D460E46002940F09B
:10E2C800CA836E2A00F02C825CD8122A00F0718171
:10E2D8002CD8052A00F0058114D8022A00F0CA803B
:10E2E80008D8002A00F0AA80012A00F0B58004248A
:10E2F800204670BD032A00F0CF80042A00F0D580A4
:10E308000424F5E70F2A00F01E8107D8082A00F038
:10E31800FC800E2A00F004810424E9E7102A00F0AA
:10E328002081112A00F031810424E1E7182A00F045
:10E338009F8113D8152A00F06C8107D8132A00F0A2
:10E348004681142A00F057810424D1E7162A00F0E8
:10E358007381172A00F07E810424C9E71B2A00F084
:10E36800B58107D8192A00F091811A2A00F09C81FA
:10E378000424BDE76C2A00F0B7816D2A00F0C28141
:10E388000424B5E77E2A00F0A2822BD8742A00F074
:10E39800398213D8712A00F0FC8107D86F2A00F05F
:10E3A800D481702A00F0E7810424A1E7722A00F0E2
:10E3B8000482732A00F01882042499E7772A00F06F
:10E3C8005C8207D8752A00F02B82762A00F03F82FB
:10E3D80004248DE77C2A00F05E827D2A00F06982A1
:10E3E800042485E7892A00F0DF8213D8852A00F003
:10E3F800A78207D8812A00F08282842A00F09782B7
:10E40800042475E7862A00F0AD82882A00F0B882D5
:10E4180004246DE7D12A00F0F38207D88A2A00F095
:10E42800D982C82A00F0B581042461E7D42A00F013
:10E43800F582D62A00F0FF82042459E728B937214B
:10E44800A04811F004FE286052E71A6837219D4859
:10E4580011F0EFFD00244BE728B92121994811F06C
:10E46800F6FD286044E71A682121964811F0E1FD7D
:10E4780000243DE730B92421924811F0E8FD00124C
:10E48800286035E7186811F056FE242102468D48A9
:10E4980011F0CFFD34462BE7002840F0DE82222120
:10E4A800884811F0D4FD286022E7874E18B9D6F8BD
:10E4B800B8322B601CE71B68202106F12400C6F83F
:10E4C800B83211F0C4FD420740F12482D6F8B802F0
:10E4D80011F031FE24210246701811F0AAFD002423
:10E4E80006E730B92821774811F0B1FD801028607F
:10E4F800FEE61A68940DA405002C40F0B082920044
:10E508002821704811F095FDF2E6002840F0A98214
:10E518000F216C4811F09BFD00F001002860E7E630
:10E5280030B92021674811F092FD40002860DFE6ED
:10E538001B682021002B14BF02220122614811F020
:10E5480078FD0024D4E628B925215E4811F07FFD26
:10E558002860CDE61A6825215A4811F06AFD34462C
:10E56800C6E630B92A21574811F071FD801028609D
:10E57800BEE61A68940DA405002C40F0748292003F
:10E588002A21504811F055FDB2E630B929214D48ED
:10E5980011F05DFD80102860AAE61A68940DA405A4
:10E5A800002C40F0628292002921464811F041FD7A
:10E5B8009EE628B92721434811F049FD286097E6CF
:10E5C8001A6827213F4811F034FD344690E630B9E7
:10E5D8002B213C4811F03BFD8010286088E61A6822
:10E5E800940DA405002C40F0428292002B2135485E
:10E5F80011F01FFD7CE628B92621324811F027FDCD
:10E60800286075E61A6826212E4811F012FD0024AC
:10E618006EE628B92C212B4811F019FD286067E611
:10E628001A68930D9B05002B40F023822C21254866
:10E6380011F0FFFC00245BE628B92D21214811F0D8
:10E6480006FD286054E61A682D211E4811F0F1FCD9
:10E6580000244DE628B92E211A4811F0F8FC28604C
:10E6680046E61A682E21174811F0E3FC00243FE61D
:10E6780028B92F21134811F0EAFC286038E61A68F7
:10E688002F21104811F0D5FC344631E628B9302145
:10E698000C4811F0DCFC28602AE61A683021094889
:10E6A80011F0C7FC002423E628B93321054811F0EE
:10E6B800CEFC28601CE61A683321024811F0B9FC28
:10E6C800002415E620210020FC20002028B9342150
:10E6D800A24811F0BCFC28600AE61A6834219F4859
:10E6E80011F0A7FC344603E628B960219B4811F0D5
:10E6F800AEFC2860FCE51A686021984811F099FC86
:10E708000024F5E528B96121944811F0A0FC28609F
:10E71800EEE51A686121914811F08BFC0024E7E5C9
:10E728001C218E4824B911F092FC00142860DFE502
:10E7380011F08DFC2A68C0F3080040EA02421C214F
:10E74800864811F076FC3446D2E51C21834824B96A
:10E7580011F07DFCC0B22860CAE511F078FC2B6886
:10E7680000F47F02C3F308031A431C217B4811F00D
:10E7780060FC0024BCE528B95921784811F067FCF1
:10E788002860B5E51A685921744811F052FC002434
:10E79800AEE50521714824B911F059FCC0B22860D2
:10E7A800A6E511F054FC2A7820F0FF000243052169
:10E7B8006A4811F03EFC00249AE5052167482CB907
:10E7C80011F045FCC0F30720286091E511F03FFCEB
:10E7D8002B6820F47F421B029BB21A4305215F4835
:10E7E80011F027FC002483E528B95D4B5B6AD3F858
:10E7F8006C312B607CE51A685A21584811F019FCD5
:10E80800002475E528B9564B5B6AD3F870312B6044
:10E818006EE51A685B21514811F00BFC344667E538
:10E828004F48436AD3F870311CB9C3F30E032B6009
:10E838005EE52A6823F4FF4323F07F03C2F30E0248
:10E848001A435B21243011F0F4FB002450E54448BE
:10E85800436AD3F870211CB9C2F307422A6047E51E
:10E868002B6822F47F021B0403F47F031A435B2105
:10E87800243011F0DEFB00243AE528B95E21374840
:10E8880011F0E5FB286033E51A685E21334811F082
:10E89800D0FB34462CE528B95C21304811F0D7FB71
:10E8A800286025E51A685C212C4811F0C2FB002479
:10E8B8001EE528B95F21294811F0C9FB286017E532
:10E8C8001A685F21254811F0B4FB002410E50521E2
:10E8D80022482CB911F0BBFBC0F30740286007E5BC
:10E8E80011F0B5FB2B6820F47F021B0403F47F03AF
:10E8F8001A430521194811F09CFB3446F8E448B145
:10E908001C684CB10121154811F072FC28600028E0
:10E9180000F0B1800024EBE40721104811F097FBC8
:10E92800072120F480020D4811F083FBE0E4002861
:10E9380040F0A3806521094811F089FB2860D7E4DD
:10E948000028E7D10721054811F081FBC0F3815069
:10E95800431E584258412860CAE400BF20210020C5
:10E96800FC20002028B95221454811F070FB28608E
:10E97800BEE41A685221424811F05BFB0024B7E458
:10E988004048436AD3F8902114B9D2B22A60AFE460
:10E998002B6822F0FF0203F00F031A43632124308F
:10E9A80011F047FB0024A3E43648436AD3F89021CA
:10E9B8001CB9C2F303222A609AE42B6822F470621D
:10E9C8001B0203F470631A436321243011F031FBF6
:10E9D80034468DE42B48436AD3F890211CB9C2F31E
:10E9E80007422A6084E42B6822F47F021B0403F4A4
:10E9F8007F031A436321243011F01BFB002477E4C2
:10EA080028B950211E4811F022FB286070E41A68CA
:10EA180050211B4811F00DFB344669E420B9194B0D
:10EA28005B6A9B692B6063E41A685321144811F0F0
:10EA380000FB00245CE428B91521114811F007FBFC
:10EA4800286055E41B68104A15215A430C4811F0F8
:10EA5800F0FA00244CE408244AE4042448E410248E
:10EA680046E4042444E4102442E4102440E410243E
:10EA78003EE410243CE420243AE4042438E400BFB3
:10EA880020210020FC2000200071020007B501921F
:10EA980001AB02460120FFF70DFC03B05DF804FB53
:10EAA80013460246002005E408B50021024811F08B
:10EAB80055FB002008BD00BF2021002008B54942B1
:10EAC800024811F04BFB002008BD00BF20210020A8
:10EAD80008B5024811F042FB002008BD20210020A3
:10EAE80038B50A4B0A4CDD6860682B689B69984703
:10EAF80001200CF00DFE2B6860685B69984704F1F3
:10EB0800240011F000FB012038BD00BF70A30208EB
:10EB1800FC20002038B50A4B0A4CDD6860682B6879
:10EB28009B69984701200CF0F3FD2B6860685B69CE
:10EB3800984704F1240011F0D3FA012038BD00BF32
:10EB480070A30208FC20002008B5024811F006FB5B
:10EB5800002008BD20210020034B0846D3F8BC3212
:10EB68001146DB68184700BFFC200020F8B5484C68
:10EB7800484D494F0021494BAA6904F1240011F07E
:10EB88008EFAFE68736803F59E72226203F5AC7212
:10EB9800E26103F55472A26103F55B72626103F5E9
:10EBA8006272226103F5697203F57770E26003F51A
:10EBB800707203F57E7323603368A260DB6860605F
:10EBC80098473368A069DB68984733686069DB68F1
:10EBD800984733682069DB6898473368E068DB68E2
:10EBE80098473368A068DB689847336860685B6952
:10EBF80098473368A0695B699847336860695B69BF
:10EC08009847336820695B6998473368E0685B69AF
:10EC180098473368A0685B6998473368206A1B691E
:10EC280098473368E0691B699847336820681B690F
:10EC3800984773683A6903F538735360C4F8BC227F
:10EC48000122AB6916491A80C3F8041215492A75BE
:10EC5800C3F80812144B6B62144B2B62144BEB6114
:10EC6800144BAB62144BEB63144BAB63144BEB626A
:10EC7800144B2B63144BEB64144BAB64144BAB6514
:10EC8800144B6B65144B2B66144BEB65F8BD00BF3A
:10EC9800FC2000209C64002070A3020868910208F0
:10ECA8001DEB0008E9EA000851EB0008D9EA000862
:10ECB800C5EA0008B1EA0008A9EA000895EA0008D0
:10ECC800A5E200088DE2000881E200086DE2000874
:10ECD80061E2000889E1000811E100081DE100086F
:10ECE8000022014B9A6070479C640020022870B58E
:10ECF800144646D004D890B1012833D0042070BD02
:10ED080003284CD0FF28F9D1264CD4F89030D3F8FA
:10ED180004329847A369D3F80432984714E012687C
:10ED280032F00303EBD1204B204DDE68D20768692F
:10ED380033680BD51B6998472468326814F00204BD
:10ED4800A86909D0136998470020D8E7DB68984775
:10ED5800336868699B69EEE7D36898473368A869A0
:10ED68009B69F0E7104B114DDE6814682869336819
:10ED78000CB11B69E7E7DB689847336828699B692A
:10ED8800E1E7094B094DDE6814683368A868002C70
:10ED9800EFD1DB6898473368A8689B69D3E72020E0
:10EDA800ADE700BF9C64002070A30208C8230020C0
:10EDB80070B5184E184CF56860682B689B699847C1
:10EDC8002B68A0699B6898472B6860699B6898477F
:10EDD8002B6820699B6898472B68E0689B68984770
:10EDE8002B68A0689B6898472B68206A9B6898479F
:10EDF8002B68E0699B6898472B6820689B68984750
:10EE08002B6860689B6898473369BDE870405B6A07
:10EE1800184700BF70A30208C82300200A4601460D
:10EE2800014811F056BB00BFEC2300200146014801
:10EE380011F0FFBBEC23002010B50348144611F075
:10EE480020FB206010BD00BFEC2300206C2970B5AA
:10EE58000D46144623D06D2917D0062918D1214B09
:10EE680093F87C20032A2DD00B2A11D19E6F1021F4
:10EE7800304610F0A4FBC4F3046220F01F000243E4
:10EE88001021304610F08DFB02E0174BC3F8B82272
:10EE980022462946BDE87040144811F0E4BA1149E9
:10EEA800D1F8C43091F87C10012915BF0E49C2F37E
:10EEB8001302D1F8B812C4F3025118BF01F07F0150
:10EEC8009847E5E79E6F1021304610F05CFAC4F3CE
:10EED800046220F01F0002431021304610F045FA6A
:10EEE800D6E700BF9C640020C8230020EC23002044
:10EEF80008B50448D0F8BC22243011F029FC0020C1
:10EF080008BD00BFC823002008B50448D0F8BC22BB
:10EF1800243011F001FC002008BD00BFC8230020E8
:10EF2800F8B504461D46002940F01E81112A00F05C
:10EF3800D08029D8042A7DD00AD8012A62D057B2B5
:10EF4800002F55D0022A63D0032A6FD0042476E01C
:10EF58000E2A00F09B800DD8052A00F08880082A28
:10EF6800F4D10028F2D10F21814811F08AFA00F07B
:10EF7800010053E00F2A00F09B80102AE6D10028F8
:10EF880040F09C802A2174E0172A00F0CD8017D821
:10EF9800142A00F0B78009D8122A00F0A580132A95
:10EFA800D4D1002840F0A6802B2162E0152A00F079
:10EFB800AF80162ACAD1002840F0B3802D2119E06D
:10EFC8001A2A00F0C08009D8182A00F0B380192A3C
:10EFD800BCD1002840F0B48030210BE01B2A00F09F
:10EFE800B880D62AB2D1002840F0B980152101E0B6
:10EFF80020B937215E4811F044FA0FE037211A682A
:10F008005B4830E008B92121F4E71A682121F7E7C5
:10F0180030B92421564811F034FA001228600EE065
:10F028001A682421002AB8BF5242E9E700288DD186
:10F038002221DFE74F4F20B9D7F8BC322B6020469A
:10F04800F8BD1B68202107F12400C7F8BC3211F075
:10F0580018FA10F00404F2D0D7F8BC0211F02BFB18
:10F0680024210246781811F0FEF90024E7E728B9B0
:10F0780028213F4811F005FA8010CFE71A68930D50
:10F088009B05002B72D192002821B9E748B92021AD
:10F09800374811F0F6F900F00300831E5842584132
:10F0A800BCE71B682021002B14BF02220122A7E71E
:10F0B80008B925219EE71A682521A1E71A68940D49
:10F0C800A405002C52D12A219200294811F0CBF92D
:10F0D800B5E708B92921CCE71A68940DA405002CD6
:10F0E80044D192002921F0E708B9272182E71A685C
:10F0F800272185E71A68940DA405002C36D19200C3
:10F108002B21E2E708B9262174E71A68262177E758
:10F1180008B92C216EE71A68930D9B0533BB2C2187
:10F128006EE71A682D216BE708B92E2162E71A6885
:10F138002E2165E708B92F215CE71A682F215FE7C0
:10F148001A6830215CE708B9332153E71A6833217C
:10F1580056E708B934214DE71A68342150E71B688F
:10F16800054A15215A434BE7082468E7102466E747
:10F17800EC230020C82300200071020007B501928B
:10F1880001AB02460120FFF7CBFE03B05DF804FB9C
:10F19800134602460020C3E608B50021024811F0D4
:10F1A8009DFA002008BD00BFEC23002008B54942A5
:10F1B800024811F093FA002008BD00BFEC2300209C
:10F1C80008B5024811F08AFA002008BDEC23002097
:10F1D80038B50A4B0A4CDD6860682B689B6998470C
:10F1E80001200CF095FA2B6860685B69984704F178
:10F1F800240011F006FA012038BD00BF70A30208F0
:10F20800C823002038B50A4B0A4CDD6860682B68B3
:10F218009B69984701200CF07BFA2B6860685B6952
:10F22800984704F1240011F0D9F9012038BD00BF36
:10F2380070A30208C823002070B5114C0D4694F83D
:10F248007C30012B19D0032B0BBF002328230C2261
:10F258000F2242EA433242F0884242F0401204212F
:10F2680011F001F9D4F89030012D0CBFD3F8043215
:10F27800D3F80832BDE87040184700230B22E8E7AE
:10F288009C640020F8B5334CD4E9B032120240EA4D
:10F29800032042EA136294F8C832C4E9B002D4E900
:10F2A800B4600133050E000240EA1660DBB2360294
:10F2B80084F8C832C4E9B460002949D0042B04D9C1
:10F2C8006D2104F1240011F0CEF8D4F8C0226C218D
:10F2D800214811F0C8F801200CF01AFAD4F8C0221D
:10F2E8006C211D4811F0BFF800230022C4E9B423A3
:10F2F80094F8C832042B08D96F21174811F0C1F8C7
:10F30800D4F8D4321843C4F8D4026E21124811F04C
:10F31800B8F8D4E9B423C717104394F8C8223B437C
:10F32800C2F10802D200A2F12006C2F120019340E6
:10F3380000FA06F620FA01F133430B439040C4E982
:10F34800B40300220023C4E9B023002384F8C832A0
:10F358002846F8BDC8230020EC23002008B5024841
:10F3680011F0BCF9002008BDEC230020034B08462F
:10F37800D3F8D8321146DB68184700BFC8230020ED
:10F38800F8B54C4C4C4D04F124064C4BAA69304658
:10F3980000214B4F11F001F94A49304611F045F967
:10F3A800FE68736803F59E72226203F5AC72E2612F
:10F3B80003F55472A26103F55B72626103F5627230
:10F3C800226103F5697203F57770E26003F57072E4
:10F3D80003F57E7323603368A260DB68606098473A
:10F3E8003368A069DB68984733686069DB689847C9
:10F3F80033682069DB6898473368E068DB689847BA
:10F408003368A068DB689847336860685B69984729
:10F418003368A0695B699847336860695B69984796
:10F42800336820695B6998473368E0685B69984787
:10F438003368A0685B6998473368206A1B699847F6
:10F448003368E0691B699847336820681B699847E7
:10F4580073683A6903F538735360C4F8D8220122F7
:10F46800AB6919491A80C3F8041218492A75C3F8F8
:10F478000812174BAB66174B6B62174B2B62174B77
:10F48800EB61174BAB62174BEB63174BAB63174B37
:10F49800EB62174B2B63174BEB64174BAB64174BA3
:10F4A800AB65174B6B65174B2B66174BEB65174B0B
:10F4B800EB66F8BDC82300209C640020689302080E
:10F4C80070A3020841F200080DF20008D9F1000803
:10F4D8008DF2000865F30008C9F10008B5F10008CD
:10F4E800A1F1000899F1000885F1000811EF000862
:10F4F800F9EE000855EE000841EE000835EE000868
:10F50800F5EC0008E9EC0008B9ED000825EE000864
:10F518000022014B9A6070479C64002070B5184E19
:10F52800184CF56860682B689B6998472B68A06938
:10F538009B6898472B6860699B6898472B68206987
:10F548009B6898472B68E0689B6898472B68A06879
:10F558009B6898472B68206A9B6898472B68E069E6
:10F568009B6898472B6820689B6898472B68606859
:10F578009B6898473369BDE870405B6A184700BFCD
:10F5880070A30208B02600200A460146014811F07F
:10F598005CB900BFD4260020022870B5144648D0B4
:10F5A80005D898B1012835D00424204670BD032819
:10F5B8004DD0FF28F8D12A4CD4F89030D3F8043233
:10F5C8009847A369D3F80432984714E0126832F0D8
:10F5D800030310D1234B244DDE68D20768693368D2
:10F5E8000BD51B6998472468326814F00204A8698F
:10F5F80009D0136998470024D7E7DB689847336830
:10F6080068699B69EEE7D36898473368A8699B697E
:10F618009847CAE7134B144DDE68146828693368A5
:10F628000CB11B69E6E7DB689847336828699B6972
:10F63800EEE70C4B0C4DDE6814683368A868002CA4
:10F64800EFD1DB6898473368A8689B69E0E7012138
:10F65800064811F009FA20600028CCD12024A4E73C
:10F668009C64002070A30208B0260020D426002045
:10F678000146014811F0B6BAD426002010B5034857
:10F68800144611F0BAF8206010BD00BFD42600203F
:10F698006C2970B50D46144623D06D2917D006295C
:10F6A80018D1214B93F87C20032A2DD00B2A11D195
:10F6B8009E6F102130460FF082FFC4F3046220F0E1
:10F6C8001F000243102130460FF06BFF02E0174B7A
:10F6D800C3F8B82222462946BDE87040144811F004
:10F6E8007EB81149D1F8C43091F87C10012915BFB2
:10F6F8000E49C2F31302D1F8B812C4F3025118BF6D
:10F7080001F07F019847E5E79E6F102130460FF022
:10F718003AFEC4F3046220F01F0002431021304671
:10F728000FF023FED6E700BF9C640020B02600201F
:10F73800D426002008B50448D0F8BC22243011F0A3
:10F7480083F9002008BD00BFB026002008B5044892
:10F75800D0F8BC22243011F05BF9002008BD00BFAE
:10F76800B026002070B504461D460E46002940F01C
:10F77800EB836F2A00F047825ED8122A00F0768168
:10F788002CD8052A00F00A8114D8022A00F0CF806C
:10F7980008D8002A00F0AF80012A00F0BA800424BB
:10F7A800204670BD032A00F0D480042A00F0DA80D5
:10F7B8000424F5E70F2A00F0238107D8082A00F06F
:10F7C80001810E2A00F009810424E9E7102A00F0DB
:10F7D8002581112A00F036810424E1E7182A00F077
:10F7E800A48113D8152A00F0718107D8132A00F0D4
:10F7F8004B81142A00F05C810424D1E7162A00F01A
:10F808007881172A00F083810424C9E71B2A00F0B5
:10F81800BB8107D8192A00F096811A2A00F0A18125
:10F828000424BDE76D2A00F0CB8100F2D7816C2A51
:10F8380000F0B8810424B3E77D2A00F0B4822BD805
:10F84800752A00F04B8213D8722A00F0148207D868
:10F85800702A00F0EE81712A00F0F98104249FE7F4
:10F86800732A00F01F82742A00F02A82042497E782
:10F87800782A00F06E8207D8762A00F04682772A26
:10F8880000F0598204248BE7792A00F070827C2AE0
:10F8980000F07B82042483E7882A00F0EA8213D8E8
:10F8A800842A00F0C28207D87E2A00F08A82812A40
:10F8B80000F09F82042473E7852A00F0BF82862A1D
:10F8C80000F0C98204246BE7C82A00F0C08107D879
:10F8D800892A00F0E2828A2A00F0F58204245FE790
:10F8E800D42A00F01483D62A00F01E83D12A00F00F
:10F8F8000083042454E728B93721A14810F07DFF7C
:10F9080028604DE71A6837219D4810F068FF0024E9
:10F9180046E728B921219A4810F06FFF28603FE791
:10F928001A682121964810F05AFF002438E730B9A8
:10F938002421934810F061FF0012286030E718680E
:10F9480011F035F8242102468D4810F048FF34465E
:10F9580026E7002840F0FA822221894810F04DFF5E
:10F9680028601DE7874E18B9D6F8BC322B6017E718
:10F978001B68202106F12400C6F8BC3210F03DFFB8
:10F98800420740F14182D6F8BC0211F010F8242158
:10F998000246701810F023FF002401E730B928212F
:10F9A800774810F02AFF80102860F9E61A68940D4D
:10F9B800A405002C40F0CC8292002821704810F059
:10F9C8000EFFEDE6002840F0C5820F216C4810F0CC
:10F9D80014FF00F001002860E2E630B920216848F1
:10F9E80010F00BFF40002860DAE61B682021002B8E
:10F9F80014BF02220122624810F0F1FE0024CFE673
:10FA080028B925215E4810F0F8FE2860C8E61A6873
:10FA180025215B4810F0E3FE3446C1E630B92A21BF
:10FA2800574810F0EAFE80102860B9E61A68940D6D
:10FA3800A405002C40F0908292002A21504810F032
:10FA4800CEFEADE630B929214D4810F0D6FE801023
:10FA58002860A5E61A68940DA405002C40F07E8263
:10FA680092002921464810F0BAFE99E628B92721C4
:10FA7800434810F0C2FE286092E61A6827214048E1
:10FA880010F0ADFE34468BE630B92B213C4810F01F
:10FA9800B4FE8010286083E61A68940DA405002C33
:10FAA80040F05E8292002B21354810F098FE77E6F0
:10FAB80028B92621324810F0A0FE286070E61A689E
:10FAC80026212F4810F08BFE002469E628B92C2146
:10FAD8002B4810F092FE286062E61A68930D9B0589
:10FAE800002B40F03F822C21254810F078FE00249E
:10FAF80056E628B92D21224810F07FFE28604FE6EF
:10FB08001A682D211E4810F06AFE002448E628B91C
:10FB18002E211B4810F071FE286041E61A682E213C
:10FB2800174810F05CFE00243AE628B92F21144843
:10FB380010F063FE286033E61A682F21104810F091
:10FB48004EFE34462CE628B930210D4810F055FEFB
:10FB5800286025E61A683021094810F040FE002484
:10FB68001EE628B93321064810F047FE286017E63C
:10FB78001A683321024810F032FE002410E600BF54
:10FB8800D4260020B026002028B934219F4810F040
:10FB980034FE286004E61A6834219C4810F01FFEE1
:10FBA8003446FDE528B96021984810F026FE286003
:10FBB800F6E51A686021954810F011FE0024EFE57B
:10FBC80028B96121914810F018FE2860E8E51A6804
:10FBD80061218E4810F003FE0024E1E51C218B48CA
:10FBE80024B910F00AFE00142860D9E510F005FECB
:10FBF8002A68C0F3080040EA02421C21834810F03A
:10FC0800EEFD0024CCE51C21804824B910F0F5FD58
:10FC1800C0B22860C4E510F0F0FD2B6800F47F0244
:10FC2800C3F308031A431C21784810F0D8FD344662
:10FC3800B6E528B95921754810F0DFFD2860AFE511
:10FC48001A685921714810F0CAFD0024A8E5062158
:10FC58006E4824B910F0D1FDC0B22860A0E510F0BC
:10FC6800CCFD2A7820F0FF0002430621674810F0F7
:10FC7800B6FD002494E5062164482CB910F0BDFDBA
:10FC8800C0F3072028608BE510F0B7FD2B6820F43F
:10FC98007F421B029BB21A4306215C4810F09FFD6D
:10FCA80034467DE528B95A4B5B6AD3F86C312B6032
:10FCB80076E51A685A21554810F091FD00246FE541
:10FCC80028B9534B5B6AD3F870312B6068E51A6822
:10FCD8005B214E4810F083FD002461E54C48436ADF
:10FCE800D3F870311CB9C3F30E032B6058E52A68AA
:10FCF80023F4FF4323F07F03C2F30E021A435B2170
:10FD0800243010F06CFD34464AE54148436AD3F884
:10FD180070211CB9C2F307422A6041E52B6822F41E
:10FD28007F021B0403F47F031A435B21243010F085
:10FD380056FD002434E528B95E21344810F05DFDF5
:10FD480028602DE51A685E21304810F048FD00242F
:10FD580026E528B918212D4810F04FFD28601FE529
:10FD68001A681821294810F03AFD344618E528B9D0
:10FD78001921264810F041FD286011E51A6819215B
:10FD8800224810F02CFD00240AE528B95C211F4800
:10FD980010F033FD286003E51A685C211B4810F059
:10FDA8001EFD0024FCE428B95F21184810F025FD49
:10FDB8002860F5E41A685F21144810F010FD3446F5
:10FDC800EEE4062111482CB910F017FDC0F30740E6
:10FDD8002860E5E410F011FD2B6820F47F021B0475
:10FDE80003F47F031A430621084810F0F8FC0024A6
:10FDF800D6E448B11C686CB10121044810F034FE07
:10FE08002860002800F0B0800024C9E4D42600202F
:10FE1800B02600200721564810F0EFFC072120F4F7
:10FE28008002534810F0DBFCBAE4002840F09E80C2
:10FE380065214F4810F0E1FC2860B1E40028E3D1C7
:10FE480007214B4810F0D9FCC0F38150431E58429B
:10FE580058412860A4E428B95221454810F0CDFC47
:10FE680028609DE41A685221414810F0B8FC00242B
:10FE780096E44048436AD3F8902114B9D2B22A6074
:10FE88008EE42B6822F0FF0203F00F031A4363216C
:10FE9800243010F0A4FC344682E43648436AD3F890
:10FEA80090211CB9C2F303222A6079E42B6822F45A
:10FEB80070621B0203F470631A436321243010F04C
:10FEC8008EFC00246CE42B48436AD3F890211CB9BB
:10FED800C2F307422A6063E42B6822F47F021B0402
:10FEE80003F47F031A436321243010F078FC0024C4
:10FEF80056E428B950211E4810F07FFC28604FE4D2
:10FF08001A6850211A4810F06AFC002448E420B905
:10FF1800184B5B6ADB692B6042E41A68532114486A
:10FF280010F05DFC00243BE428B91521104810F0BE
:10FF380064FC286034E41B680F4A15215A430C48B6
:10FF480010F04DFC00242BE4082429E4042427E4C1
:10FF5800102425E4042423E4102421E410241FE4BD
:10FF680010241DE410241BE4202419E4042417E4BD
:10FF7800D4260020B02600200071020007B50192A7
:10FF880001AB02460120FFF7EDFB03B05DF804FB6F
:10FF9800134602460020FFF7E5BB08B500210248DA
:10FFA80010F018FD002008BDD426002008B54942ED
:10FFB800024810F00FFD002008BD00BFD426002025
:10FFC80008B5024810F006FD002008BDD426002020
:10FFD80038B50A4B0A4CDD6860682B689B699847FE
:10FFE80001200BF095FB2B6860685B69984704F16A
:08FFF800240010F0C4FC0120FC
:020000040801F1
:1000000038BD00BF70A30208B026002038B50A4BE7
:100010000A4CDD6860682B689B69984701200BF0EB
:100020007BFB2B6860685B69984704F1240010F043
:1000300097FC012038BD00BF70A30208B026002045
:1000400070B5114C0D4694F87C30012B19D0032B60
:100050000BBF002328230C220F2242EA433242F036
:10006000884242F04012042110F0BDFBD4F89030D9
:10007000012D0CBFD3F80432D3F80832BDE870402C
:10008000184700230B22E8E79C640020F8B5334CA6
:10009000D4E9B032120240EA032042EA136294F833
:1000A000C832C4E9B002D4E9B4600133050E0002DD
:1000B00040EA1660DBB2360284F8C832C4E9B460A4
:1000C000002949D0042B04D96D2104F1240010F03B
:1000D0008AFBD4F8C0226C21214810F084FB012057
:1000E0000BF01AFBD4F8C0226C211D4810F07BFBEA
:1000F00000230022C4E9B42394F8C832042B08D9A1
:100100006F21174810F07DFBD4F8D4321843C4F89F
:10011000D4026E21124810F074FBD4E9B423C7173F
:10012000104394F8C8223B43C2F10802D200A2F166
:100130002006C2F12001934000FA06F620FA01F1F0
:1001400033430B439040C4E9B40300220023C4E9C5
:10015000B023002384F8C8322846F8BDB02600201A
:10016000D426002008B5024810F038FC002008BD55
:10017000D4260020034B0846D3F8D8321146DB685A
:10018000184700BFB0260020F8B54C4C4C4D04F188
:1001900024064C4BAA69304600214B4F10F0BDFBA2
:1001A0004A49304610F003FCFE68736803F59E72FE
:1001B000226203F5AC72E26103F55472A26103F5A9
:1001C0005B72626103F56272226103F5697203F585
:1001D0007770E26003F5707203F57E732360336815
:1001E000A260DB68606098473368A069DB68984765
:1001F00033686069DB68984733682069DB68984733
:100200003368E068DB6898473368A068DB68984724
:10021000336860685B6998473368A0695B69984791
:10022000336860695B699847336820695B69984700
:100230003368E0685B6998473368A0685B699847F2
:100240003368206A1B6998473368E0691B699847DF
:10025000336820681B69984773683A6903F53873F7
:100260005360C4F8D8220122AB6919491A80C3F837
:10027000041218492A75C3F80812174BAB66174BBE
:100280006B62174B2B62174BEB61174BAB62174B33
:10029000EB63174BAB63174BEB62174B2B63174B9F
:1002A000EB64174BAB64174BAB65174B6B65174B88
:1002B0002B66174BEB65174BEB66F8BDB02600209D
:1002C0009C6400206895020870A3020841000108A0
:1002D0000D000108D9FF00088D0001086501010823
:1002E000C9FF0008B5FF0008A3FF000899FF000838
:1002F00085FF000855F700083DF7000899F600084B
:1003000085F6000879F60008A1F5000819F500083F
:1003100025F5000891F500080022014B9A6070470E
:100320009C64002070B5184E184CF56860682B6806
:100330009B6998472B68A0699B6898472B68606900
:100340009B6898472B6820699B6898472B68E068F2
:100350009B6898472B68A0689B6898472B68206A21
:100360009B6898472B68E0699B6898472B682068D2
:100370009B6898472B6860689B6898473369BDE81D
:1003800070405B6A184700BF70A3020898290020DC
:100390000A460146014810F0DCBC00BFBC29002021
:1003A000022870B5144648D005D898B1012835D038
:1003B0000424204670BD03284DD0FF28F8D12A4CD4
:1003C000D4F89030D3F804329847A369D3F80432B4
:1003D000984714E0126832F0030310D1234B244DE8
:1003E000DE68D207686933680BD51B6998472468B3
:1003F000326814F00204A86909D0136998470024F0
:10040000D7E7DB689847336868699B69EEE7D3688C
:1004100098473368A8699B699847CAE7134B144DFE
:10042000DE681468286933680CB11B69E6E7DB688D
:100430009847336828699B69EEE70C4B0C4DDE68E2
:1004400014683368A868002CEFD1DB6898473368DC
:10045000A8689B69E0E70121064810F0AFFD206025
:100460000028CCD12024A4E79C64002070A30208BB
:1004700098290020BC2900200146014810F05CBEEC
:10048000BC29002010B50348144610F03AFC206047
:1004900010BD00BFBC2900206C2970B50D46144664
:1004A00023D06D2917D0062918D1214B93F87C2031
:1004B000032A2DD00B2A11D19E6F102130460FF048
:1004C00082F8C4F3046220F01F000243102130467A
:1004D0000FF06BF802E0174BC3F8BC222246294606
:1004E000BDE87040144810F0FEBB1149D1F8C4308B
:1004F00091F87C10012915BF0E49C2F31302D1F8FF
:10050000BC12C4F3025118BF01F07F019847E5E720
:100510009E6F102130460EF03AFFC4F3046220F0C3
:100520001F000243102130460EF023FFD6E700BF24
:100530009C64002098290020BC29002008B50448AC
:10054000D0F8C022243010F029FD002008BD00BFE3
:100550009829002008B50448D0F8C022243010F0B3
:1005600001FD002008BD00BF9829002070B5044699
:100570001D460E46002940F0EB836F2A00F04782AB
:100580005ED8122A00F076812CD8052A00F00A8164
:1005900014D8022A00F0CF8008D8002A00F0AF80DB
:1005A000012A00F0BA800424204670BD032A00F01E
:1005B000D480042A00F0DA800424F5E70F2A00F042
:1005C000238107D8082A00F001810E2A00F0098152
:1005D0000424E9E7102A00F02581112A00F0368171
:1005E0000424E1E7182A00F0A48113D8152A00F0AA
:1005F000718107D8132A00F04B81142A00F05C8126
:100600000424D1E7162A00F07881172A00F08381AC
:100610000424C9E71B2A00F0BB8107D8192A00F07F
:1006200096811A2A00F0A1810424BDE76D2A00F00A
:10063000CB8100F2D7816C2A00F0B8810424B3E7A3
:100640007D2A00F0B4822BD8752A00F04B8213D893
:10065000722A00F0148207D8702A00F0EE81712A05
:1006600000F0F98104249FE7732A00F01F82742AA6
:1006700000F02A82042497E7782A00F06E8207D8D7
:10068000762A00F04682772A00F0598204248BE70C
:10069000792A00F070827C2A00F07B82042483E7B0
:1006A000882A00F0EA8213D8842A00F0C28207D890
:1006B0007E2A00F08A82812A00F09F82042473E758
:1006C000852A00F0BF82862A00F0C98204246BE7E5
:1006D000C82A00F0C08107D8892A00F0E2828A2A5D
:1006E00000F0F58204245FE7D42A00F01483D62AB0
:1006F00000F01E83D12A00F00083042454E728B9B7
:100700003721A14810F0FDFA28604DE71A6837211B
:100710009D4810F0E8FA002446E728B921219A48BC
:1007200010F0EFFA28603FE71A682121964810F090
:10073000DAFA002438E730B92421934810F0E1FABE
:100740000012286030E7186810F0DBFB2421024615
:100750008D4810F0C8FA344626E7002840F0FA82A7
:100760002221894810F0CDFA28601DE7874E18B97C
:10077000D6F8C0322B6017E71B68202106F1240051
:10078000C6F8C03210F0BDFA420740F14182D6F8F7
:10079000C00210F0B6FB24210246701810F0A3FA34
:1007A000002401E730B92821774810F0AAFA801018
:1007B0002860F9E61A68940DA405002C40F0CC825C
:1007C00092002821704810F08EFAEDE6002840F0E3
:1007D000C5820F216C4810F094FA00F001002860E7
:1007E000E2E630B92021684810F08BFA400028601A
:1007F000DAE61B682021002B14BF02220122624886
:1008000010F071FA0024CFE628B925215E4810F0D7
:1008100078FA2860C8E61A6825215B4810F063FA68
:100820003446C1E630B92A21574810F06AFA8010E0
:100830002860B9E61A68940DA405002C40F0908257
:1008400092002A21504810F04EFAADE630B9292125
:100850004D4810F056FA80102860A5E61A68940DED
:10086000A405002C40F07E8292002921464810F019
:100870003AFA99E628B92721434810F042FA28604D
:1008800092E61A682721404810F02DFA34468BE68C
:1008900030B92B213C4810F034FA8010286083E6F0
:1008A0001A68940DA405002C40F05E8292002B2162
:1008B000354810F018FA77E628B92621324810F0AA
:1008C00020FA286070E61A6826212F4810F00BFAEB
:1008D000002469E628B92C212B4810F012FA286070
:1008E00062E61A68930D9B05002B40F03F822C2195
:1008F000254810F0F8F9002456E628B92D212248A1
:1009000010F0FFF928604FE61A682D211E4810F0FC
:10091000EAF9002448E628B92E211B4810F0F1F925
:10092000286041E61A682E21174810F0DCF90024EF
:100930003AE628B92F21144810F0E3F9286033E68D
:100940001A682F21104810F0CEF934462CE628B949
:1009500030210D4810F0D5F9286025E61A683021BD
:10096000094810F0C0F900241EE628B933210648D2
:1009700010F0C7F9286017E61A683321024810F012
:10098000B2F9002410E600BFBC29002098290020FD
:1009900028B934219F4810F0B4F9286004E61A6899
:1009A00034219C4810F09FF93446FDE528B96021B8
:1009B000984810F0A6F92860F6E51A686021954875
:1009C00010F091F90024EFE528B96121914810F069
:1009D00098F92860E8E51A6861218E4810F083F9DB
:1009E0000024E1E51C218B4824B910F08AF9001499
:1009F0002860D9E510F085F92A68C0F3080040EABC
:100A000002421C21834810F06EF90024CCE51C2121
:100A1000804824B910F075F9C0B22860C4E510F020
:100A200070F92B6800F47F02C3F308031A431C21FA
:100A3000784810F058F93446B6E528B95921754878
:100A400010F05FF92860AFE51A685921714810F07D
:100A50004AF90024A8E506216E4824B910F051F99E
:100A6000C0B22860A0E510F04CF92A7820F0FF0011
:100A700002430621674810F036F9002494E5062168
:100A800064482CB910F03DF9C0F3072028608BE5CD
:100A900010F037F92B6820F47F421B029BB21A43F7
:100AA00006215C4810F01FF934467DE528B95A4B01
:100AB0005B6AD3F86C312B6076E51A685A21554889
:100AC00010F011F900246FE528B9534B5B6AD3F895
:100AD00070312B6068E51A685B214E4810F003F90D
:100AE000002461E54C48436AD3F870311CB9C3F364
:100AF0000E032B6058E52A6823F4FF4323F07F039D
:100B0000C2F30E021A435B21243010F0ECF8344695
:100B10004AE54148436AD3F870211CB9C2F3074241
:100B20002A6041E52B6822F47F021B0403F47F0353
:100B30001A435B21243010F0D6F8002434E528B99C
:100B40005E21344810F0DDF828602DE51A685E213A
:100B5000304810F0C8F8002426E528B918212D489F
:100B600010F0CFF828601FE51A681821294810F006
:100B7000BAF8344618E528B91921264810F0C1F80A
:100B8000286011E51A681921224810F0ACF80024F9
:100B90000AE528B95C211F4810F0B3F8286003E586
:100BA0001A685C211B4810F09EF80024FCE428B968
:100BB0005F21184810F0A5F82860F5E41A685F2155
:100BC000144810F090F83446EEE4062111482CB990
:100BD00010F097F8C0F307402860E5E410F091F8B2
:100BE0002B6820F47F021B0403F47F031A430621C1
:100BF000084810F078F80024D6E448B11C686CB1BD
:100C00000121044810F0DAF92860002800F0B080D3
:100C10000024C9E4BC290020982900200721564857
:100C200010F06FF8072120F48002534810F05BF8B1
:100C3000BAE4002840F09E8065214F4810F061F82A
:100C40002860B1E40028E3D107214B4810F059F89F
:100C5000C0F38150431E584258412860A4E428B98B
:100C60005221454810F04DF828609DE41A68522141
:100C7000414810F038F8002496E44048436AD3F81D
:100C8000902114B9D2B22A608EE42B6822F0FF02C0
:100C900003F00F031A436321243010F024F8344684
:100CA00082E43648436AD3F890211CB9C2F3032288
:100CB0002A6079E42B6822F470621B0203F47063EB
:100CC0001A436321243010F00EF800246CE42B4802
:100CD000436AD3F890211CB9C2F307422A6063E447
:100CE0002B6822F47F021B0403F47F031A43632161
:100CF00024300FF0F8FF002456E428B950211E4894
:100D00000FF0FFFF28604FE41A6850211A480FF0D7
:100D1000EAFF002448E420B9184B5B6ADB692B60CA
:100D200042E41A68532114480FF0DDFF00243BE42D
:100D300028B9152110480FF0E4FF286034E41B683F
:100D40000F4A15215A430C480FF0CDFF00242BE425
:100D5000082429E4042427E4102425E4042423E4BB
:100D6000102421E410241FE410241DE410241BE4AB
:100D7000202419E4042417E4BC2900209829002029
:100D80000071020007B5019201AB02460120FFF796
:100D9000EDFB03B05DF804FB134602460020FFF7AD
:100DA000E5BB08B50021024810F0BEF8002008BDE0
:100DB000BC29002008B54942024810F0B5F80020CF
:100DC00008BD00BFBC29002008B5024810F0ACF8EF
:100DD000002008BDBC29002038B50A4B0A4CDD684C
:100DE00060682B689B69984701200AF095FC2B6886
:100DF00060685B69984704F1240010F06AF80120EC
:100E000038BD00BF70A302089829002038B50A4BEE
:100E10000A4CDD6860682B689B69984701200AF0DE
:100E20007BFC2B6860685B69984704F1240010F034
:100E30003DF8012038BD00BF70A3020898290020AA
:100E4000F8B5334CD4E9B232120240EA032042EA48
:100E5000136294F8D032C4E9B202D4E9B660013327
:100E6000050E000240EA1660DBB2360284F8D0328A
:100E7000C4E9B660002949D0042B04D96D2104F1DE
:100E800024000FF030FFD4F8C8226C2121480FF065
:100E90002AFF01200AF040FCD4F8C8226C211D482A
:100EA0000FF021FF00230022C4E9B62394F8D032CA
:100EB000042B08D96F2117480FF023FFD4F8DC3238
:100EC0001843C4F8DC026E2112480FF01AFFD4E96F
:100ED000B623C717104394F8D0223B43C2F108024F
:100EE000D200A2F12006C2F12001934000FA06F6DA
:100EF00020FA01F133430B439040C4E9B6030022CA
:100F00000023C4E9B223002384F8D0322846F8BD78
:100F100098290020BC29002070B51A4C054694F889
:100F20007C300E46012B25D0032B0BBF002328233A
:100F30000C220F2242EA433242F0884242F0401231
:100F4000042128460FF0CFFE012E16D103220521E1
:100F500028460FF0C8FE0022062128460FF0C3FEE7
:100F600028460FF07BFFD4F89030D3F80432BDE868
:100F70007040184700230B22DCE7D4F89030D3F8F8
:100F80000832F4E79C64002008B502480FF0CCFF5B
:100F9000002008BDBC290020034B0846D3F8E032EE
:100FA0001146DB68184700BF98290020F8B54C4C63
:100FB0004C4D04F124064C4BAA69304600214B4F9E
:100FC0000FF02BFF4A4930460FF097FFFE68736819
:100FD00003F59E72226203F5AC72E26103F554726E
:100FE000A26103F55B72626103F56272226103F52F
:100FF000697203F57770E26003F5707203F57E7332
:1010000023603368A260DB68606098473368A0693A
:10101000DB68984733686069DB6898473368206904
:10102000DB6898473368E068DB6898473368A068F6
:10103000DB689847336860685B6998473368A069E4
:101040005B699847336860695B69984733682069D2
:101050005B6998473368E0685B6998473368A068C4
:101060005B6998473368206A1B6998473368E06971
:101070001B699847336820681B69984773683A6909
:1010800003F538735360C4F8E0220122AB691949B3
:101090001A80C3F8041218492A75C3F80812174BAE
:1010A000AB66174B6B62174B2B62174BEB61174B01
:1010B000AB62174BEB63174BAB63174BEB62174BF2
:1010C0002B63174BEB64174BAB64174BAB65174B9C
:1010D0006B65174B2B66174BEB65174BEB66F8BD33
:1010E000982900209C6400206897020870A30208D9
:1010F000190F01080D0E0108D90D0108410E010854
:10110000890F0108C90D0108B50D0108A30D0108DB
:10111000990D0108850D0108550501083D050108D7
:10112000990401088504010879040108A103010854
:1011300019030108250301089103010800207047E5
:10114000012070470022014B9A6070479C64002088
:1011500010B50020144610F035F8206010BD0020B6
:1011600010F052B810B5044618B910F049F92046ED
:1011700010BD0820FCE710B5044618B910F022F99C
:10118000204610BD0820FCE70021F4E74942F2E7C1
:10119000F1E738B504461D46002940F03C87043A83
:1011A000FA2A00F23B87DFE812F0FB003907390723
:1011B000390739073907390739073907390739072F
:1011C000390739073907390739073907390739071F
:1011D000390739073907390739073907390739070F
:1011E00039073907390739073907390739073907FF
:1011F00039073907390739073907390739073907EF
:101200003907390739070901190139072901390156
:1012100039073907390739073907390739073907CE
:1012200039073907390739073907390739073907BE
:1012300039073907390739073907390739073907AE
:10124000390739073907390739073907390739079E
:10125000390739073907390739073907390739078E
:101260003907390739073907390749015701650136
:10127000730181018F019D01AB01B901C701D50146
:10128000E301F101FF010D021B02290233023D02BD
:101290003907470251025B0265026F027E028D022E
:1012A0009C02A502390739073907AE02B602BE0211
:1012B000C802D202390739073907DA02E202EA0224
:1012C0003907390739073907390739073907F40268
:1012D000FE020803120339073907390739073907AE
:1012E00039071C03260330033A034403390739073F
:1012F0003907390739074E03580368037803800319
:101300008C0396039F03A903B003BB03C803D50353
:10131000E203EF03FC0309041604390723042E0437
:101320003B044804530460046D047A048704940465
:10133000A304B204C104D004DF04EE04FD040D05CF
:101340001F052F053F054F055F056F057F058F05BD
:101350009F05AF05BF05CE0539073907390739079E
:101360003907390739073907390739073907DD05DB
:10137000ED05FD050D061D062D063D064D065D0617
:101380006C067B068A069906A806B706C606D50629
:10139000E306F106FF0639070D07180726072E0793
:1013A00028B960210FF00EFF2860204638BD2A685A
:1013B000602100200FF028FF0024F6E730B9024634
:1013C00008210FF041FF00B22860EEE700222B88D1
:1013D000082110460FF045FF0024E6E730B9024629
:1013E00009210FF031FF00B22860DEE700222B88D0
:1013F000092110460FF035FF0024D6E730B901224D
:1014000008210FF021FF00B22860CEE72B880122CF
:10141000082100200FF025FF0024C6E730B9012283
:1014200009210FF011FF00B22860BEE72B880122CE
:10143000092100200FF015FF0024B6E7002840F036
:10144000F085012203210FF0DFFE22460221204613
:101450000FF0FAFE2860A8E7002840F0E585012299
:1014600003210FF0D1FE0122022120460FF0ECFEF5
:1014700028609AE7002840F0DA85022203210FF065
:10148000C3FE2246022120460FF0DEFE28608CE7D4
:10149000002840F0CF85024603210FF0B5FE22461A
:1014A000022120460FF0D0FE28607EE7002840F0A1
:1014B000C485024603210FF0A7FE01220221204627
:1014C0000FF0C2FE286070E7002840F0B9850322C3
:1014D00011460FF099FE2246022120460FF0B4FE7D
:1014E000286062E7002840F0AE85042203210FF057
:1014F0008BFE2246022120460FF0A6FE286054E70C
:10150000002840F0A385042203210FF07DFE012274
:10151000022120460FF098FE286046E7002840F0A0
:101520009885052203210FF06FFE224602212046F6
:101530000FF08AFE286038E7002840F08D850522EC
:1015400003210FF061FE0122022120460FF07CFEF4
:1015500028602AE7002840F08285062203210FF048
:1015600053FE2246022120460FF06EFE28601CE743
:10157000002840F07785072203210FF045FE224620
:10158000022120460FF060FE28600EE7002840F0A0
:101590006C85072203210FF037FE0122022120462D
:1015A0000FF052FE286000E7002840F06185082215
:1015B00003210FF029FE2246022120460FF044FEAF
:1015C0002860F2E6002840F05685082203210FF03B
:1015D0001BFE0122022120460FF036FE2860E4E6C1
:1015E000002840F04B85092203210FF00DFE224612
:1015F000022120460FF028FE2860D6E6002840F0A1
:101600004085024612210FF01FFE00B22860CCE692
:10161000002840F03985012212210FF015FE00B29A
:101620002860C2E6002840F03285024613210FF000
:101630000BFE00B22860B8E6002840F02B85024679
:1016400015210FF001FE00B22860AEE6002840F040
:101650002485012215210FF0F7FD00B22860A4E6D1
:10166000002840F01D85024616210FF0EDFD00B266
:1016700028609AE6002840F01685012216210FF016
:10168000E3FD00B2286090E6002840F00F850A22B2
:1016900003210FF0B9FD2246022120460FF0D4FDB0
:1016A00000B2286081E6002840F003850A22032169
:1016B0000FF0AAFD0122022120460FF0C5FD00B265
:1016C000286072E6002840F0F7840B2203210FF017
:1016D0009BFD2246022120460FF0B6FD00B2286095
:1016E00063E6002840F0EB84024606210FF0ACFDD3
:1016F00028605AE6002840F0E584012206210FF018
:10170000A3FD286051E6002840F0DF8441210FF05E
:1017100059FD286049E6002840F0DA8442210FF0A4
:1017200051FD286041E6002840F0D5840122462181
:101730000FF08AFD00B2286037E6002840F0CE8422
:10174000024646210FF080FD00B228602DE60028F9
:1017500040F0C78447210FF035FD286025E60028BA
:1017600040F0C28421210FF02DFD28601DE60028E5
:1017700040F0BD8422210FF025FD286015E60028E9
:1017800040F0B884024623210FF05EFD00B22860CD
:101790000BE6002840F0B18427210FF013FD20F064
:1017A0007F40286001E6002840F0AA8428210FF03D
:1017B00009FD20F07F402860F7E5002840F0A38471
:1017C00001222A210FF040FD00B22860EDE500283B
:1017D00040F09C8402462A210FF036FD00B22860BA
:1017E000E3E5002840F09584024639210FF02CFDF6
:1017F00000B22860D9E5002840F08E84012239210A
:101800000FF022FD00B22860CFE5002840F0878469
:1018100002463D210FF018FD00B22860C5E5002802
:1018200040F0808402463F210FF00EFD00B2286098
:10183000BBE5002840F0798402463A210FF004FD10
:1018400000B22860B1E5002840F0728402465321BE
:101850000FF0FAFC00B22860A7E530B9012264213C
:101860000FF0F2FC00B228609FE52B880122642172
:1018700000200FF0F6FC002497E530B90246642101
:101880000FF0E2FC00B228608FE500222B88642173
:1018900010460FF0E6FC002487E5002840F04B845A
:1018A00066210FF08FFC28607FE520B968210FF0DA
:1018B00089FC286079E5296800200FF0A1FD00244B
:1018C00073E5002840F03A84012269210FF0BCFC46
:1018D00000B2286069E5002840F03384C14B598983
:1018E0000FF023FD286060E5002840F02D840246BB
:1018F00069210FF0A9FC00B2286056E5002840F0ED
:1019000026840FF078FD28604FE518B90FF09DFD93
:1019100028604AE5296800200FF093FD002444E583
:10192000002840F0178402466D210FF06DFC6C21F9
:1019300020460FF047FC286037E5002840F00D8472
:1019400001226D210FF060FC6C2120460FF03AFC63
:1019500028602AE5002840F0038402226D210FF060
:1019600053FC6C2120460FF02DFC28601DE500285B
:1019700040F0F98303226D210FF046FC6C212046D4
:101980000FF020FC286010E5002840F0EF830422CF
:101990006D210FF039FC6C2120460FF013FC2860FC
:1019A00003E5002840F0E58305226D210FF02CFCB3
:1019B0006C2120460FF006FC2860F6E4002840F079
:1019C000DB8306226D210FF01FFC6C2120460FF0F7
:1019D000F9FB2860E9E4002840F0D18307226D215B
:1019E0000FF012FC6C2120460FF0ECFB2860DCE4C9
:1019F00018B90FF06BFC2860D7E4296800200FF0BD
:101A000057FC0024D1E4774B598918B90FF084FCB6
:101A10002860CAE42A6800200FF06CFC0024C4E4AB
:101A2000002840F0AF8301226F210FF0EDFB6E2103
:101A300020460FF0C7FB2860B7E418B90FF0CFFCC1
:101A40002860B2E4296800200FF0BCFC0024ACE45C
:101A5000002840F09A8303226F210FF0D5FB6E21FE
:101A600020460FF0AFFB28609FE4002840F09083F1
:101A700004226F210FF0C8FB6E2120460FF0A2FB5D
:101A8000286092E4002840F0868305226F210FF041
:101A9000BBFB6E2120460FF095FB286085E40028F3
:101AA00040F07C8306226F210FF0AEFB6E212046B2
:101AB0000FF088FB286078E4002840F0728307224A
:101AC0006F210FF0A1FB6E2120460FF07BFB2860F9
:101AD0006BE4002840F0688308226F210FF094FB2C
:101AE00022466E2120460FF0AFFB00B228605CE476
:101AF000002840F05C8308226F210FF085FB012253
:101B00006E2120460FF0A0FB00B228604DE40028B3
:101B100040F0508309226F210FF076FB22466E21A0
:101B200020460FF091FB00B228603EE4002840F010
:101B300044830A226F210FF067FB22466E21204664
:101B40000FF082FB00B228602FE4002840F03883B9
:101B50000A226F210FF058FB01226E2120460FF060
:101B600073FB00B2286020E4002840F02C830B2295
:101B70006F210FF049FB22466E2120460FF064FBD7
:101B800000B2286011E4002840F020830B226F216E
:101B90000FF03AFB01226E2120460FF055FB00B2F8
:101BA000286002E4002840F014830C226F210FF01B
:101BB0002BFB22466E2120460FF046FB00B2286028
:101BC000FFF7F3BB002840F007830C226F210FF0D2
:101BD0001BFB01226E2120460FF036FB00B228606D
:101BE000FFF7E3BB106B0020002840F0F8820D22C5
:101BF0006F210FF009FB22466E2120460FF024FBD7
:101C000000B22860FFF7D1BB002840F0EB820D2224
:101C10006F210FF0F9FA01226E2120460FF014FB1C
:101C200000B22860FFF7C1BB002840F0DE820E2220
:101C30006F210FF0E9FA22466E2120460FF004FBD7
:101C400000B22860FFF7B1BB002840F0D1820E221D
:101C50006F210FF0D9FA01226E2120460FF0F4FA1D
:101C600000B22860FFF7A1BB002840F0C4820F2219
:101C70006F210FF0C9FA22466E2120460FF0E4FAD8
:101C800000B22860FFF791BB002840F0B7820F2216
:101C90006F210FF0B9FA01226E2120460FF0D4FA1D
:101CA00000B22860FFF781BB002840F0AA82102212
:101CB0006F210FF0A9FA22466E2120460FF0C4FAD8
:101CC00000B22860FFF771BB002840F09D8211220E
:101CD0006F210FF099FA22466E2120460FF0B4FAD8
:101CE00000B22860FFF761BB002840F0908211220B
:101CF0006F210FF089FA01226E2120460FF0A4FA1D
:101D000000B22860FFF751BB002840F08382122206
:101D10006F210FF079FA22466E2120460FF094FAD7
:101D200000B22860FFF741BB002840F07682132202
:101D30006F210FF069FA22466E2120460FF084FAD7
:101D40002860FFF732BB002840F06A8213226F211F
:101D50000FF05AFA01226E2120460FF075FA286022
:101D6000FFF723BB002840F05E82C0226F210FF0F6
:101D70004BFA22466E2120460FF066FA00B2286028
:101D8000FFF713BB002840F05182C0226F210FF0F3
:101D90003BFA01226E2120460FF056FA00B228606D
:101DA000FFF703BB002840F04482C1226F210FF0EF
:101DB0002BFA22466E2120460FF046FA00B2286028
:101DC000FFF7F3BA002840F03782C1226F210FF0ED
:101DD0001BFA01226E2120460FF036FA00B228606D
:101DE000FFF7E3BA002840F02A82C2226F210FF0E9
:101DF0000BFA22466E2120460FF026FA00B2286028
:101E0000FFF7D3BA002840F01D82C2226F210FF0E5
:101E1000FBF901226E2120460FF016FA00B228606D
:101E2000FFF7C3BA002840F01082C3226F210FF0E1
:101E3000EBF922466E2120460FF006FA00B2286028
:101E4000FFF7B3BA002840F00382C3226F210FF0DE
:101E5000DBF901226E2120460FF0F6F900B228606E
:101E6000FFF7A3BA002840F0F681C4226F210FF0DB
:101E7000CBF922466E2120460FF0E6F92860FFF7E5
:101E800094BA002840F0EA81C4226F210FF0BCF917
:101E900001226E2120460FF0D7F92860FFF785BA9E
:101EA000002840F0DE81C5226F210FF0ADF92246F7
:101EB0006E2120460FF0C8F92860FFF776BA002897
:101EC00040F0D281C5226F210FF09EF901226E21D0
:101ED00020460FF0B9F92860FFF767BA002840F0F4
:101EE000C681C6226F210FF08FF922466E2120464F
:101EF0000FF0AAF92860FFF758BA002840F0BA811D
:101F0000C6226F210FF080F901226E2120460FF0CA
:101F10009BF92860FFF749BA002840F0AE81C7223C
:101F20006F210FF071F922466E2120460FF08CF9D7
:101F30002860FFF73ABA002840F0A281C7226F213B
:101F40000FF062F901226E2120460FF07DF9286022
:101F5000FFF72BBA002840F09681C8226F210FF0BE
:101F600053F96E2120460FF02DF92860FFF71DBAB6
:101F7000002840F08B81C9226F210FF045F96E21B6
:101F800020460FF01FF92860FFF70FBA002840F035
:101F90008081CA226F210FF037F96E2120460FF0A1
:101FA00011F92860FFF701BA002840F07581CB22B3
:101FB0006F210FF029F96E2120460FF003F92860F8
:101FC000FFF7F3B9B94B18B95B892B60FFF7EDB98F
:101FD0002A6800245A81FFF7E8B920B9B34B5B7A2D
:101FE0002B60FFF7E2B9B24A2878511C0FF024FBAE
:101FF0000024FFF7DAB9002840F05181AB4B1B7A7F
:102000002B60FFF7D2B9002840F04C81A74BDB884A
:102010002B60FFF7CAB90824FFF7C7B90424FFF7FC
:10202000C4B90424FFF7C1B90424FFF7BEB90424DE
:10203000FFF7BBB90424FFF7B8B90424FFF7B5B91B
:102040000424FFF7B2B90424FFF7AFB90424FFF763
:10205000ACB90424FFF7A9B90424FFF7A6B90424F6
:10206000FFF7A3B90424FFF7A0B90424FFF79DB933
:102070000424FFF79AB90424FFF797B90424FFF763
:1020800094B90424FFF791B90424FFF78EB904240E
:10209000FFF78BB90424FFF788B90424FFF785B94B
:1020A0000424FFF782B90424FFF77FB90424FFF763
:1020B0007CB90424FFF779B90424FFF776B9042426
:1020C000FFF773B90424FFF770B90424FFF76DB963
:1020D0000424FFF76AB90424FFF767B90424FFF763
:1020E00064B90424FFF761B90424FFF75EB904243E
:1020F000FFF75BB90424FFF758B90424FFF755B97B
:102100000424FFF752B90424FFF74FB90424FFF762
:102110004CB90424FFF749B90424FFF746B9042455
:10212000FFF743B90424FFF740B90424FFF73DB992
:102130000424FFF73AB90424FFF737B90424FFF762
:1021400034B90424FFF731B90424FFF72EB904246D
:10215000FFF72BB90424FFF728B90424FFF725B9AA
:102160000424FFF722B90424FFF71FB90424FFF762
:102170001CB90424FFF719B90424FFF716B9042485
:10218000FFF713B90424FFF710B90424FFF70DB9C2
:102190000424FFF70AB90424FFF707B90424FFF762
:1021A00004B90424FFF701B90424FFF7FEB804249E
:1021B000FFF7FBB80424FFF7F8B80424FFF7F5B8DD
:1021C0000424FFF7F2B80424FFF7EFB80424FFF764
:1021D000ECB80424FFF7E9B80424FFF7E6B80424B8
:1021E000FFF7E3B80424FFF7E0B80424FFF7DDB8F5
:1021F0000424FFF7DAB80424FFF7D7B80424FFF764
:10220000D4B80424FFF7D1B80424FFF7CEB80424CF
:10221000FFF7CBB80424FFF7C8B80424FFF7C5B80C
:102220000424FFF7C2B80424FFF7BFB80424FFF763
:10223000BCB80424FFF7B9B80424FFF7B6B80424E7
:10224000FFF7B3B80424FFF7B0B80424FFF7ADB824
:102250000424FFF7AAB80424FFF7A7B80424FFF763
:10226000A4B80424FFF7A1B80424FFF79EB80424FF
:10227000FFF79BB80424FFF798B80424FFF795B83C
:102280000424FFF792B80424FFF78FB80424FFF763
:102290008CB80424FFF789B80424FFF786B8042417
:1022A000FFF783B80424FFF780B800BF106B00204D
:1022B000186B002007B5019201AB02460120FEF722
:1022C00068FF03B05DF804FB134602460020FEF7EA
:1022D00060BF022804BF0C4B93F8F00030B90B4BE1
:1022E000DB681B689B690A4A10681847012809D1F6
:1022F000054B93F8F030012B04D1044BDB681B68CD
:102300005B69F0E7704700BF9C64002070A302087F
:10231000882C002010B50020FFF7DBFFBDE810403F
:10232000034B044ADB6810681B689B69184700BFB1
:1023300070A30208882C00201FB5084B33F8081C36
:102340000291991E019133F8041C00915A780146BC
:1023500000200FF067F905B05DF804FB186B002052
:1023600010B5044620B909680FF057F8204610BD93
:102370000820FCE738B50D46044620B90FF03BF8BD
:102380002860204638BD0820FCE70120704710B4C3
:102390000C4630B9044B20465B6811469B6810BC64
:1023A0001847002010BC7047882C002070B5274EBD
:1023B000274DF46860682368CC30DB682860984754
:1023C0000120FFF786FF6368326903F538735360B5
:1023D000204B21496A609A693220C2F804121F49D1
:1023E000C2F80812002111801D4A5A621D4A1A6261
:1023F0001D4ADA611D4A9A621D4A1A651D4ADA634E
:102400001D4A9A631D4ADA621D4A1A631D4ADA643C
:102410001D4A9A641D4A9A651D4A5A651D4A5A66A4
:102420001D4A1A6601221A751C4ADA6540F28A2290
:10243000C3E903204FF47A72194B9A8041F270720B
:102440001A604FF4807259725A8170BD70A30208ED
:10245000882C00209C640020411101088B23010876
:1024600077110108911101088D11010889110108E6
:1024700075230108C9220108B52201086511010868
:10248000612301085F110108511101083923010876
:102490003D110108D3220108451101081523010847
:1024A000106B0020002070470022014B9A6070479B
:1024B0009C64002000200FF0EFB810B500201446F7
:1024C0000FF0C8F8206010BD022804BF0B4B93F832
:1024D000F00030B90A4BDB681B689B69094A106839
:1024E0001847012809D1054B93F8F030012B04D18E
:1024F000034BDB681B685B69F0E770479C64002056
:1025000070A302089C2C002010B50020FFF7DCFF10
:10251000BDE81040034B044ADB6810681B689B69E8
:10252000184700BF70A302089C2C0020002208B5A9
:10253000104617210FF0B0F800221A2110460FF0B4
:10254000ABF8BDE8084041F61912192100200FF040
:10255000A3B808B5FFF7EAFF012008BD08B5FFF7EB
:10256000E5FF012008BD38B50D46044620B90FF03F
:10257000CCF92860204638BD0820FCE7F0B50646B7
:102580003D4B85B033F8062C9C1F0292221D019210
:1025900062883A4D00920146E27900200FF0CCFAB1
:1025A0006B68B34224D105B0F0BD022B15D1344F76
:1025B00020460CF013FC22693B689A4259D06621F0
:1025C00000200FF069F823693B606B2100200FF0B9
:1025D00041F80023A06023624BE0012B49D1F4E7CE
:1025E0006B2138460FF036F82761A060276240E083
:1025F00000200FF08AF90823009301460323E268C4
:1026000004F110000CF0FEFA0122E06069210020C4
:102610000FF062F84FF6FE1200F5F9437F339BB2DC
:1026200093420FD8238901B259434FF0080348BFA2
:10263000FF31B4F9182009120093124804230CF05A
:10264000E1FA2083104C94F82470002FC8D00F4B6F
:102650001B78032BA9D10E4F20460CF0F1FBA2688A
:102660003B689A4205D0682100200FF015F8A36856
:102670003B606E6097E700BF166B00209C2C00202B
:102680003C6B0020306B0020E86A0020386B002093
:10269000406B002070B50E46E0B90F4D95F8244010
:1026A000A4B10E4C2278012A02D10FF02EF9286134
:1026B0000321002021700FF033F86B2100200EF071
:1026C000C9FF336818446860002070BD09680FF0C6
:1026D0002EF9F9E70820F8E7E86A0020386B0020B7
:1026E00070B50E46A8B90C4D95F8244074B10B4C4A
:1026F0002278012A02D10FF008F928610321002075
:1027000021700FF00DF86E60002070BD0FF002F91F
:10271000FAE70820F9E700BFE86A0020386B0020DC
:1027200070B50E46A8B90C4D95F8244074B10B4C09
:102730002278012A02D10FF0E8F828610221002056
:1027400021700EF0EDFFEE60002070BD0FF0CDF8AF
:10275000FAE70820F9E700BFE86A0020386B00209C
:102760000021DDE74942DBE7DAE738B515460C46DC
:1027700000295FD1AC283DD014D80C2836D006D81B
:10278000042825D00B282AD00424204638BD0D2843
:10279000FBD0AB28F8D193B20122642120460EF081
:1027A000A8FFF2E7BE2839D008D8B32825D0BD2825
:1027B000EAD1114620460EF0C3FFE6E7FB2836D0EB
:1027C000FC28E1D11C4AE8B2511C0FF0BFF9DCE74C
:1027D000602120460EF060FF184B1D60D5E75F2199
:1027E00020460EF059FF154B5D61CEE7134B83F881
:1027F0002420CAE793B20A46CFE76B2120460EF0A9
:102800004BFF0F4B1B78032BBFD10C4B2A46C3E960
:102810000155682120460EF03FFFB6E7094B2046E0
:1028200019890EF0BAFF0122054B1A70ADE7054B6E
:102830001A81AAE70824A8E7166B0020E86A00209E
:10284000386B0020106B002038B515460C46002967
:1028500040F08D80B22875D022D8AB2861D014D832
:102860000B284BD004D8042840D00424204638BD7F
:102870000C284BD00D28F8D13E4B93F82420002A89
:1028800049D01B692B600024F0E7AD2853D050D30A
:10289000AE2855D0B028E8D1374BB3F9183038E01E
:1028A000C0285CD013D8BD284FD005D8B328DCD1C0
:1028B00008460FF054F83AE0BE284AD0BF28D4D1D9
:1028C00001226F2120460EF0E7FE6E2134E0FC2845
:1028D00047D004D8FB28C8D1274B1B8919E0FD2815
:1028E00042D0FE28C1D1244B9B8812E060212046B3
:1028F0000EF0B0FE1F4B28601860B7E75F2120463E
:102900000EF0A8FE1B4B28605861AFE7194B93F8F7
:1029100024302B60AAE7662100200EF09BFE286081
:10292000B1E70122642120460EF0D6FE00B22860F5
:102930009CE70A46F6E7662120460EF08BFEF6E796
:102940006821F9E70C4BDB68E3E708460EF006FF69
:10295000EDE7094B204619890EF031FFE7E7022227
:10296000AFE7054BDB79D4E7034B9B79D1E708242C
:102970007CE700BFE86A0020106B002010B40C4612
:1029800030B9054B20469B6811469B6810BC184720
:10299000002010BC704700BF9C2C002070B5444E36
:1029A000444DF46860682368CC30DB682860984741
:1029B0000120FFF789FD6368326903F538735360BE
:1029C0003D4BAA603D499A690024C2F804123C4973
:1029D0000020C2F80812012111803A4A19755A6282
:1029E000394A46211A62394A394DDA61394A9A62BE
:1029F000394A1A65394ADA63394A9A63394ADA62D6
:102A0000394A1A63394ADA64394A9A64394A9A6502
:102A1000394A5A65394A5A66394A1A66394ADA656C
:102A200040F28A22C3E90321374B384A00211A6059
:102A30004FF48072C3E904011A81DC71DC60224624
:102A40001C83C3E90801172120460EF025FE22460B
:102A50001A2120460EF020FE41F6191219212046B7
:102A60000EF01AFE2246062120460EF015FE4FF407
:102A7000FA625F2120460EF00FFE4FF47A62602169
:102A800020460EF009FE28460CF09AF9204B6021F2
:102A90001C70204B20461C601F4B1C600EF0DAFDA2
:102AA0005F21286020460EF0D5FD686170BD00BF33
:102AB00070A302089C2C00209C6400205D25010866
:102AC0005325010821270108692701086527010806
:102AD000E86A0020612701086725010849280108E4
:102AE0006B270108E126010895260108B524010895
:102AF000BB2401087D250108A5240108C92401087B
:102B0000A924010809250108106B00207017E803AB
:102B1000386B0020406B00203C6B002001280BD854
:102B2000064B1A682023834043F0020302EB830321
:102B30005B6800200B60704708207047B42C0020B1
:102B40000022014B9A6070479C64002070B5094ECA
:102B50000546344654F8043B0146224600200FF057
:102B6000EAF8336822462946BDE8704001200FF09C
:102B7000E2B800BFB42C0020014B18680FF03BB93D
:102B8000B42C0020012838B5144613D045B21DB12D
:102B900002281CD0042038BD114B124ADB6824687F
:102BA0001B68D2F8A8021CB15B6998470020F2E7C5
:102BB0009B69FAE70A4B0B4ADB68D2F8A0021B6854
:102BC0005B6A9847003018BF01202060EEE7044B95
:102BD000044ADB68D2F8A4021B685B6AF1E700BF15
:102BE00070A30208B42C0020022804BF0C4B93F8F9
:102BF000F00038B90B4BDB681B685B690A4AD2F8F6
:102C00009C021847012809D1054B93F8F030012B9D
:102C100004D1044BDB681B689B69EFE7704700BF7A
:102C20009C64002070A30208B42C002070B5002022
:102C3000FFF7DAFF134B144CDD68D4F89C022B68C5
:102C40009B6898472B68D4F8A0029B6898472B682C
:102C5000D4F8A4029B6898472B68D4F8B4029B6808
:102C600098472B68D4F8AC029B6898472B68D4F837
:102C7000B0029B6898472B68D4F8A8029B68BDE80F
:102C80007040184770A30208B42C00202DE9F843C7
:102C90000F4691469846194C0021D4F8B83247F0B7
:102CA00080009B689DF820609DF824509847D4F8D8
:102CB000B83200219B6848469847D4F8B8320021C2
:102CC0009B6840469847D4F8B83200219B6830464C
:102CD0009847D4F8B83228469B680121984748EABB
:102CE0000928236846EA082607F07F0703EB8707D1
:102CF00045EA06257D60BDE8F88300BFB42C0020BE
:102D000007B5D3B20193C2F307230093C2F307437D
:102D1000120EFFF7BBFF03B05DF804FB0020FFF7C6
:102D2000EFBF01282DE9F34105460F4628D820269C
:102D3000DFF85480864018F8003074B263B1114B4C
:102D400044F0070103EB8003D3F8BC22C9B2FFF7BC
:102D5000D7FF002308F8053044F00D0100243A465F
:102D6000C9B22846FFF7CCFF2846CDE900442346E8
:102D70002246F1B2FFF78AFF204602B0BDE8F0819B
:102D80000820FAE7B42C00206C000020012873B55D
:102D900005460E461CD82024844044F0070186EAEC
:102DA000E672A2EBE672C9B2FFF7AAFF0123094A55
:102DB000002E5355E1B2B8BF022300242846CDE9C6
:102DC000004322462346FFF761FF204602B070BD54
:102DD0000820FBE76C0000200021D7E74942D5E737
:102DE000D4E738B5274D01F07F042B1993F818323A
:102DF000DB0704D42B6803EB8404606838BDD5F886
:102E0000B83200219B68204698470021D5F8B83297
:102E100008469B6898470021D5F8B83208469B6859
:102E200098470021D5F8B83208469B689847D5F8EE
:102E3000B83201219B6800209847D5F8B8320021AC
:102E40009B68204698470021D5F8B83208469B6811
:102E500098470021D5F8B83204029B680846984785
:102E60000021D5F8B83204439B6808469847D5F846
:102E7000B832240204439B680121002098472402B1
:102E80002043BBE7B42C002010B500201446FFF708
:102E9000A8FF206010BD38B50D462021814041F0CB
:102EA0000101C9B20446FFF79CFF2968014429606B
:102EB0002046BDE8384034E701292DE9F8430446AF
:102EC0000D461E4600F22F861C2A00F0B3825FD802
:102ED0000C2A00F0B3812DD8052A00F0348115D8D2
:102EE000022A00F0E38009D8002A00F0BD80012A00
:102EF00000F0CB8004242046BDE8F883032A00F0CC
:102F0000EC80042A00F0FC800424F4E7082A00F096
:102F1000648107D8062A00F02781072A00F0418142
:102F20000424E8E70A2A00F067810B2A00F0768182
:102F30000424E0E7122A00F0018213D80F2A00F0DF
:102F4000CA8107D80D2A00F097810E2A00F0B281BD
:102F50000424D0E7102A00F0CF81112A00F0DD818F
:102F60000424C8E7152A00F0218207D8132A00F0AC
:102F7000F681142A00F004820424BCE7172A00F02A
:102F80003782C0F02482182A00F043820424B2E77A
:102F9000AC2A00F03A8438D8A52A00F02C8313D844
:102FA000A22A00F0D48207D81D2A00F05F828C2A62
:102FB00000F06B8204249EE7A32A00F0E482A42A96
:102FC00000F0FD82042496E7A82A00F0B58307D814
:102FD000A62A00F05683A72A00F0918304248AE7EA
:102FE000AA2A4FEA011700F0E38340F2C28347F0B8
:102FF0006D07FFB239462846002C40F0F683FFF7F4
:10300000F0FEC0F34110306075E7B62A00F0BE84D0
:1030100013D8B32A00F0598407D8AD2A00F01284DF
:10302000AE2A00F02D84042465E7B42A00F06B84F6
:10303000B52A00F0778404245DE7CE2A00F0F584F9
:1030400007D8B82A00F0B584B92A00F0D084042447
:1030500051E7D22A00F00B85D32A00F01B85D12A34
:1030600000F0F284042446E72021A94041F00D013C
:10307000C9B220B92846FFF7B4FE30603BE71A68B2
:103080002846FFF73DFE002435E72021A94041F006
:103090000101C9B220B92846FFF7A3FE30602AE734
:1030A0001A682846FFF72CFE002424E72021A940B7
:1030B00041F00701C9B220B92846FFF792FE3060FF
:1030C00019E70122B74B28465A5532680024002AD6
:1030D000B8BF5242FFF714FE0DE7002840F02685E6
:1030E0002021A94041F00201C9B22846FFF779FE2C
:1030F00010F4000318BF4FF07F4318433060FAE626
:10310000A94B8A00134418B9D3F8BC323360F2E6F5
:10311000202732688F40002AB8BF5242F9B22846B1
:10312000C3F8BC22FFF75DFE044608B10024E2E6C6
:10313000326847F00701002AB8BF5242C9B2284698
:10314000FFF7DEFDD7E62021A94041F00601C9B214
:1031500020B92846FFF745FE3060CCE61A682846BD
:10316000FFF7CEFD0024C6E620278F4047F010076A
:10317000FFB2394628462CB9FFF733FEC0F30420CE
:103180003060B8E6FFF72DFE336820F4F8521B02DA
:1031900003F4F8531A4339462846FFF7B1FD0024DB
:1031A000A9E620278F4047F01007FFB2394628468E
:1031B0002CB9FFF716FE00F01F0030609BE6FFF70A
:1031C00010FE336820F01F0203F01F031A43394634
:1031D0002846FFF795FD00248DE6002840F0A984DD
:1031E0002021A94041F01501C9B22846FFF7F9FD99
:1031F000C0F3402030607EE6002840F09D8420210E
:10320000A94041F01501C9B22846FFF7EAFD10F0C8
:10321000020F0CBF0123002333606CE6002840F04E
:103220008E842021A94041F01501C9B22846FFF73C
:10323000D8FDC04300F0010030605CE620278F40DD
:1032400047F01407FFB2394628462CB9FFF7C9FDED
:10325000C0F3400030604EE6FFF7C3FD336820F056
:103260000202002B0CBF0223002339461A432846D2
:10327000FFF746FD00243EE620278F4047F0140765
:10328000FFB2394628462CB9FFF7ABFD00F001002C
:10329000306030E6FFF7A5FD326820F00100002A1B
:1032A00014BF024640F0010239462846FFF728FDC8
:1032B000002420E62021A94041F01401C9B220B920
:1032C0002846FFF78EFD306015E61A682846FFF79E
:1032D00017FD00240FE62021A94041F00401C9B2E6
:1032E00020B92846FFF77DFD306004E61A682846BD
:1032F000FFF706FD0024FEE52021A94041F005016D
:10330000C9B220B92846FFF76CFD3060F3E51A68B2
:103310002846FFF7F5FC0024EDE52021A94041F007
:103320000801C9B220B92846FFF75BFD3060E2E52D
:103330001A682846FFF7E4FC0024DCE52021A940B8
:1033400041F00A01C9B220B92846FFF74AFD3060B2
:10335000D1E51A682846FFF7D3FC0024CBE52021ED
:10336000A94041F00301C9B220B92846FFF739FD51
:103370003060C0E51A682846FFF7C2FC0024BAE5B1
:103380002021A94041F00B01C9B220B92846FFF71E
:1033900028FD3060AFE51A682846FFF7B1FC00242D
:1033A000A9E500BF6C000020B42C00202021A9401A
:1033B00041F00C01C9B220B92846FFF712FD306078
:1033C00099E51A682846FFF79BFC002493E5202125
:1033D000A94041F01101C9B220B92846FFF701FD0B
:1033E000306088E51A682846FFF78AFC002482E5E9
:1033F0002021A94041F01201C9B220B92846FFF7A7
:10340000F0FC306077E51A682846FFF779FC002465
:1034100071E52021A94041F01301C9B220B9284625
:10342000FFF7DFFC306066E51A682846FFF768FCA6
:10343000002460E50F0147F06C07FFB239462846CB
:103440002CB9FFF7CEFCC0F38040306053E5FFF7A6
:10345000C8FC336820F480229B0403F480231A43C1
:1034600039462846FFF74CFC002444E5002840F08C
:103470006983C64B1A68202303FA01F545F002055B
:1034800002EB85056B68336035E570B9090141F0E1
:103490006C0101F0FC012846FFF7A3FC4FF4807398
:1034A000C0F303600341336025E51B68102B48D04F
:1034B0000FDC022B41D006DC012B18D04FF0FF337C
:1034C0000024336017E5042B39D0082BF6D10523EF
:1034D0000EE0402B37D003DC202BEFD1032307E095
:1034E000802B32D0B3F5807FE8D1002300E00823A1
:1034F0002C0144F06C04E4B2214633602846FFF707
:1035000070FC336820F070621B0603F070631A438E
:1035100021462846FFF7F4FB21462846FFF761FCC9
:10352000336820F070621B0603F0706321461A4373
:103530002846FFF7E5FB0024DDE40723D8E7062350
:10354000D6E70423D4E70223D2E70123D0E70F0113
:1035500047F06C07FFB2394628462CB9FFF741FC0B
:10356000C0F3C1303060C6E4FFF73BFC336820F4A1
:10357000C032DB0303F4C0331A4339462846FFF751
:10358000BFFB0024B7E40F0147F06C07FFB23946D8
:1035900028462CB9FFF725FCC0F380303060AAE440
:1035A000FFF71FFC336820F480429B0303F4804341
:1035B0001A4339462846FFF7A3FB00249BE40F017A
:1035C00047F06C07FFB2394628462CB9FFF709FCD3
:1035D000C0F3003030608EE4FFF703FC336820F462
:1035E00080521B0303F480531A4339462846FFF7E1
:1035F00087FB00247FE40F0147F06C07FFB23946D8
:103600002846FFF7EEFB3946814600F480482846FD
:10361000B4B9B8F1000F05D0FFF7E3FBC0F3C31056
:10362000306068E4FFF7DDFB19F4006FC0F30210AF
:1036300001D130607AE540F00800306044465AE439
:10364000B8F1000F0ED0FFF7CCFB336820F4F06226
:10365000DB0103F4F0631A4339462846FFF750FBB9
:10366000002448E4FFF7BDFB336820F070021B0123
:1036700003F070031A4339462846FFF741FB4446DE
:1036800039E40F0147F06C07FFB239462846FFF7CF
:10369000A8FB394600F48048284674B9B8F1000FF9
:1036A00005D0FFF79EFBC0F30210306023E4FFF764
:1036B00098FBC0F3C31030601DE4B8F1000F0ED0CA
:1036C000FFF78FFB336820F070021B0103F07003DB
:1036D0001A4339462846FFF713FB00240BE4FFF793
:1036E00080FB336820F4F062DB0103F4F0631A43DB
:1036F00039462846FFF704FB4446FFF7FCBB0F01A1
:1037000047F06C07FFB23946284634B9FFF769FB2A
:1037100000F00F003060FFF7EEBBFFF762FB33688D
:1037200020F00F0203F00F031A4339462846FFF733
:10373000E7FA0024FFF7DFBB0F0147F06D07FFB288
:103740003946284634B9FFF74CFBC0F3C03030602F
:10375000FFF7D1BBFFF745FB336820F40042DB03E2
:103760009BB21A4339462846FFF7CAFA0024FFF7EE
:10377000C2BB47F06D07FFB23946284644B9FFF790
:1037800030FBC0F341303060FFF7B5BBB42C0020F4
:10379000FFF727FB336820F4C0425B0303F4C04308
:1037A0001A4339462846FFF7ABFA0024FFF7A3BBBC
:1037B00047F06D07FFB23946284634B9FFF711FBD1
:1037C000C0F303203060FFF796BBFFF70AFB3368B6
:1037D00020F470621B0203F470631A4339462846D2
:1037E000FFF78EFA0024FFF786BBFFF7FAFA33687B
:1037F00020F060025B0103F060031A43394628465B
:10380000FFF77EFA0024FFF776BB0F0147F06D0744
:10381000FFB23946284634B9FFF7E3FA00F00F004B
:103820003060FFF768BBFFF7DCFA336820F00F0267
:1038300003F00F031A4339462846FFF761FA0024C4
:10384000FFF759BB0F0147F06D07FFB23946284615
:1038500034B9FFF7C6FAC0F300603060FFF74BBB26
:10386000FFF7BFFA336820F080721B0603F0807305
:103870001A4339462846FFF743FA0024FFF73BBBBB
:103880000F0147F06D07FFB2394628466CB9FFF7C4
:10389000A8FA001400F07F0310F0400018BF6FF08A
:1038A0007F0018433060FFF726BBFFF79AFA3368B2
:1038B00020F4FE021B0403F4FE031A433946284693
:1038C000FFF71EFA0024FFF716BB0F0147F06C0745
:1038D000FFB23946284634B9FFF783FAC0F34040B7
:1038E0003060FFF708BBFFF77CFA336820F4003242
:1038F0005B0403F400331A4339462846FFF700FA05
:103900000024FFF7F8BA002840F01F81090141F0B8
:103910006F01C9B22846FFF764FAC0F30440306073
:10392000FFF7E9BA20278F407FB247F014085FFA0B
:1039300088F841462846FFF754FA6CB9410508D586
:1039400047F01101C9B22846FFF74BFA3060FFF784
:10395000D2BA3460FFF7CFBA47F011013268C9B26A
:103960002846FFF7CDF941462846FFF73AFA336873
:1039700020F48062002B18BF4FF4806341461A4345
:103980002846FFF7BDF90024FFF7B5BA2021A9406A
:1039900041F01101C9B228B92846FFF722FA306078
:1039A000FFF7A9BA1A682846FFF7AAF90024FFF71B
:1039B000A2BA0F0147F06C07FFB23946284634B966
:1039C000FFF70FFAC0F340303060FFF794BAFFF70B
:1039D00008FA336820F400525B0303F400531A43DF
:1039E00039462846FFF78CF90024FFF784BA0F0107
:1039F00047F06C07FFB23946284634B9FFF7F1F9B2
:103A0000C0F303503060FFF776BAFFF7EAF9336886
:103A100020F470021B0503F470031A43394628464C
:103A2000FFF76EF90024FFF766BA002840F0908097
:103A3000090141F06F01C9B22846FFF7D2F9C0F37E
:103A400009003060FFF757BA2021A94041F0190161
:103A5000C9B228B92846FFF7C4F93060FFF74BBA5E
:103A60001A682846FFF74CF90024FFF744BA2021D2
:103A7000A94041F01A01C9B228B92846FFF7B1F9A7
:103A80003060FFF738BA1A682846FFF739F9002482
:103A9000FFF731BAC8B9012D01460AD0FFF7A1F9E5
:103AA00000F01800A0F11002504250413060FFF7C2
:103AB00022BA2846FFF795F900F06000A0F1200334
:103AC000584258413060FFF716BA012D4FF00001FF
:103AD00014D00846FFF785F9336853B120F0080287
:103AE00042F0100200210846FFF70AF90024FFF710
:103AF00002BA20F0100242F00802F3E72846FFF76E
:103B000070F9336853B120F0400242F020020021E6
:103B10000120FFF7F5F80024FFF7EDB920F02002AF
:103B200042F04002F3E70824FFF7E5B90424FFF769
:103B3000E2B90424FFF7DFB90424FFF7DCB9042459
:103B4000FFF7D9B90424FFF7D6B90424FFF7D3B996
:103B50000424FFF7D0B907B5019201AB024601205A
:103B6000FFF7AAF903B05DF804FB134602460020F4
:103B7000FFF7A2B908B522210020FFF732F950B9AA
:103B800042210120FFF72DF928B9044B1868BDE840
:103B900008400EF029B9002008BD00BFB42C002059
:103BA00070B5424C424E201D0EF086F8F5686B68E9
:103BB00003F5AC72C4F8A02203F5BA72C4F8A422CB
:103BC00003F57072C4F8A82203F5777203F1CC00F4
:103BD000C4F8AC2203F57E7203F21443C4F8B43285
:103BE0002B68C4F8B022DB68C4F89C0298472B68A5
:103BF000D4F8A802DB6898472B68D4F8A8029B6920
:103C000098472B68D4F8A0021B6998472B68D4F812
:103C1000A4021B6998472B68D4F8B4021B69984723
:103C20002B68D4F8AC021B6998472B68D4F8B00213
:103C30001B69984701206B68326903F5387353603C
:103C40001C4BC4F8B8221C499A69C2F804121B49DB
:103C500010802260C2F80812194A32215A62194AA9
:103C60001A62194ADA61194A9A62194ADA63194AD8
:103C70009A63194ADA62194A1A63194ADA64194AC4
:103C80009A64194A9A65194A5A65194A1A65194A6D
:103C90005A66194A1A6602221A75B622BDE87040A1
:103CA000C3E90321154ADA65FEF79EBFB42C002054
:103CB00070A302089C640020753B0108792B010861
:103CC0008D2D0108E12D0108DD2D0108D92D0108F8
:103CD0006B3B0108573B0108232D0108972E010873
:103CE0001D2D0108892E01084D2B0108852B010887
:103CF0001D2B0108E92B0108412B01082D2C01087F
:103D000001289FBF044B03EB80035B68002094BF36
:103D10000B600820704700BF842F00200022014B59
:103D20009A6070479C640020014601480EF0FAB882
:103D3000842F002010B5034814460EF0A6F820602A
:103D400010BD00BF842F002001480EF090B800BFC6
:103D5000842F00200128F8B50D4625D82024134BC8
:103D600084401F1897F8982266B27AB1D3F89C2243
:103D700044F0070102EB810246F007011846526841
:103D8000C9B20EF074F8002387F8983246F00D019E
:103D90002A46C9B205480EF06AF804480022E1B28A
:103DA0000EF065F80020F8BD0820FCE7842F002005
:103DB00038B50D462021814041F001010446C9B2C9
:103DC00004480EF062F82968014429602046BDE8E5
:103DD0003840BFE7842F00200129F8B504460D467E
:103DE0001E4600F2F6851C2A00F0C5825ED80C2A19
:103DF00000F0A7812CD8052A00F0268114D8022AC9
:103E000000F0D58008D8002A00F0AF80012A00F029
:103E1000BD8004242046F8BD032A00F0DF80042A78
:103E200000F0EF800424F5E7082A00F0598107D854
:103E3000062A00F01A81072A00F035810424E9E7F8
:103E40000A2A00F05C810B2A00F06B810424E1E770
:103E5000122A00F0198213D80F2A00F0E08107D847
:103E60000D2A00F09C810E2A00F0C8810424D1E7BD
:103E7000102A00F0E781112A00F0F5810424C9E737
:103E8000152A00F0348207D8132A00F00E82142A73
:103E900000F01C820424BDE7172A00F04A82C0F01B
:103EA0003782182A00F056820424B3E7AB2A00F0C8
:103EB00037842BD8A52A00F02D8313D8A22A00F02E
:103EC000D28207D81D2A00F072828C2A00F07882F4
:103ED00004249FE7A32A00F0E282A42A00F0FE82D5
:103EE000042497E7A82A00F0C28307D8A62A00F086
:103EF0006183A72A00F0A48304248BE7A92A00F099
:103F0000D383AA2A00F0EE83042483E7B52A00F0C5
:103F1000B58413D8AE2A00F05F8407D8AC2A00F02D
:103F20001D84AD2A00F03784042473E7B32A00F01F
:103F30007884B42A00F0938404246BE7CE2A00F03E
:103F4000F68407D8B62A00F0C184B82A00F0D184DC
:103F500004245FE7D12AC0F03F85D22A40F23F8592
:103F6000D32A00F0F284042454E72021A94041F030
:103F70000D01C9B220B9AF480DF087FF306049E7A5
:103F80001A68AC480DF073FF002443E72021A940D4
:103F900041F00101C9B220B9A6480DF076FF3060AA
:103FA00038E71A68A3480DF062FF002432E72021A9
:103FB000A94041F00701C9B29E481CB90DF065FF48
:103FC000306027E7012332680544002AB8BF524217
:103FD00085F8983200240DF04AFF1BE7002840F0D6
:103FE00001852021A94041F00201C9B291480DF09C
:103FF0004CFF10F4000318BF4FF07F4318433060AC
:1040000008E720218B4FA940D7F89C3241F00705E3
:10401000AA00134410B95B683360FBE63268C9B28A
:10402000002AB8BF52425A6038460DF02EFF0446AF
:1040300008B10024EEE63268E9B2002AB8BF524265
:1040400038460DF014FFE5E62021A94041F00601B5
:10405000C9B220B977480DF018FF3060DAE61A6867
:1040600074480DF004FF0024D4E6202101FA05F580
:1040700045F01005EDB229466E482CB90DF005FF4C
:10408000C0F304203060C5E60DF0FFFE336820F475
:10409000F8521B0203F4F8531A43294665480DF001
:1040A000E6FE0024B6E6202101FA05F545F01005EC
:1040B000EDB229465F482CB90DF0E7FE00F01F0075
:1040C0003060A7E60DF0E1FE336820F01F0203F038
:1040D0001F031A43294657480DF0C9FE002499E6EC
:1040E000002840F082842021A94041F01501C9B286
:1040F00050480DF0CAFEC0F3402030608AE6002828
:1041000040F076842021A94041F01501C9B2494808
:104110000DF0BBFE10F0020F0CBF01230023336033
:1041200078E6002840F067842021A94041F015017D
:10413000C9B240480DF0A9FEC04300F00100306054
:1041400068E6202101FA05F545F01405EDB229468F
:1041500038482CB90DF099FEC0F34000306059E6A4
:104160000DF093FE336820F00202002B18BF0223EB
:1041700029461A432F480DF07AFE29462D480DF0A6
:1041800084FE336820F00802022B0CBF08230023B2
:1041900029461A4327480DF06AFE00243AE62021FA
:1041A00001FA05F545F01405EDB2294621482CB970
:1041B0000DF06BFE00F0010030602BE60DF065FEA7
:1041C000326820F00100002A0CBF024640F00102D4
:1041D000294618480DF04BFE294616480DF055FEAD
:1041E000336820F00402022B0CBF0423002329466D
:1041F0001A4310480DF03BFE00240BE62021A94095
:1042000041F01401C9B220B90A480DF03EFE3060F9
:1042100000E61A6807480DF02AFE0024FAE520217E
:10422000A94041F00401C9B230B902480DF02DFE99
:104230003060EFE5842F00201A68A7480DF017FEC4
:104240000024E7E52021A94041F00501C9B220B9C9
:10425000A1480DF01AFE3060DCE51A689E480DF0AA
:1042600006FE0024D6E52021A94041F00801C9B28C
:1042700020B999480DF009FE3060CBE51A689648E0
:104280000DF0F5FD0024C5E52021A94041F00A010B
:10429000C9B220B990480DF0F8FD3060BAE51A684F
:1042A0008D480DF0E4FD0024B4E52021A94041F043
:1042B0000301C9B220B988480DF0E7FD3060A9E5D7
:1042C0001A6885480DF0D3FD0024A3E52021A940FC
:1042D00041F00B01C9B220B97F480DF0D6FD306026
:1042E00098E51A687C480DF0C2FD002492E5202173
:1042F000A94041F00C01C9B220B977480DF0C5FDC5
:10430000306087E51A6874480DF0B1FD002481E53E
:104310002021A94041F01101C9B220B96E480DF029
:10432000B4FD306076E51A686B480DF0A0FD0024FE
:1043300070E52021A94041F01201C9B220B96648B8
:104340000DF0A3FD306065E51A6863480DF08FFD40
:1043500000245FE52021A94041F01301C9B220B932
:104360005D480DF092FD306054E51A685A480DF032
:104370007EFD00244EE50D0145F06C05EDB22946A9
:1043800055482CB90DF081FDC0F38040306041E507
:104390000DF07BFD336820F480229B0403F480231E
:1043A0001A4329464C480DF062FD002432E50028EE
:1043B00040F02483484901EB85014B68336029E5CF
:1043C00070B9090141F06C0101F0FC0142480DF0A7
:1043D0005CFD4FF48073C0F303600341336019E563
:1043E0001B68102B39D00FDC022B32D006DC012BDE
:1043F00018D04FF0FF33002433600BE5042B2AD094
:10440000082BF6D105230EE0402B28D003DC202B0F
:10441000EFD1032307E0802B23D0B3F5807FE8D1D1
:10442000002300E008232D0145F06C05EDB2336058
:10443000294629480DF029FD336820F070621B06DB
:1044400003F070631A43294623480DF010FD002441
:10445000E0E40723E7E70623E5E70423E3E7022395
:10446000E1E70123DFE70D0145F06C05EDB22946D8
:1044700019482CB90DF009FDC0F3C1303060C9E412
:104480000DF003FD336820F4C032DB0303F4C033C6
:104490001A43294610480DF0EAFC0024BAE40D0145
:1044A00045F06C05EDB229460B482CB90DF0EDFC3A
:1044B000C0F380303060ADE40DF0E7FC336820F4E9
:1044C00080429B0303F480431A43294602480DF0BF
:1044D000CEFC00249EE400BF842F00200D0145F097
:1044E0006C05EDB22946BB482CB90DF0CEFCC0F3EB
:1044F000003030608EE40DF0C8FC336820F4805248
:104500001B0303F480531A432946B2480DF0AFFC55
:1045100000247FE40D0145F06C05EDB22946AD485D
:104520000DF0B3FC00F48047A4B93FB12946A94877
:104530000DF0ABFCC0F3C31030606BE40311020557
:1045400003F0700301D4336073E543F00803336074
:104550003C465FE429469F4877B10DF096FC3368EE
:1045600020F4F062DB0103F4F0631A432946994812
:104570000DF07DFC00244DE40DF087FC326820F442
:104580000060120202F400620243294691480DF0D5
:104590006EFC29468F480DF078FC336820F07002DD
:1045A0001B0103F070031A4329468A480DF05FFC93
:1045B0003C462FE40D0145F06C05EDB229468548D7
:1045C0000DF063FC2946074682489CB97D0405D559
:1045D0000DF05BFCC0F3021030601BE40DF055FCE5
:1045E0003905C0F3C31001D4306022E540F0080063
:1045F00030600FE40DF049FC10F480442946754802
:104600000FD00DF042FC336820F070021B0103F064
:1046100070031A4329466F480DF029FC0024FFF768
:10462000F9BB0DF032FC336820F4F062DB0103F4D7
:10463000F0631A43294667480DF019FCFFF7EABBFF
:104640000D0145F06C05EDB22946624824B90DF024
:104650001CFC3460FFF7DEBB0DF017FC294620F090
:104660000F025C480DF003FC0024FFF7D3BB0D01E3
:1046700045F06D05EDB22946564834B90DF005FCFC
:10468000C0F3C0303060FFF7C5BB0DF0FEFB3368F0
:1046900020F40042DB039BB21A4329464D480DF03B
:1046A000E6FB0024FFF7B6BB0D0145F06D05EDB24A
:1046B0002946484834B90DF0E8FBC0F3413030607A
:1046C000FFF7A8BB0DF0E1FB336820F4C0425B03A9
:1046D00003F4C0431A4329463E480DF0C8FB0024AA
:1046E000FFF798BB0D0145F06D05EDB2294639483D
:1046F00034B90DF0CAFBC0F303203060FFF78ABB6A
:104700000DF0C3FB336820F470621B0203F4706386
:104710001A4329462F480DF0AAFB0024FFF77ABB65
:104720000D0145F06D05EDB229462A4834B90DF06A
:10473000ACFBC0F341103060FFF76CBB0DF0A5FB84
:10474000336820F060025B0103F060031A432946DE
:1047500020480DF08CFB0024FFF75CBB0D0145F0F9
:104760006D05EDB229461B4834B90DF08EFB00F003
:104770000F003060FFF74EBB0DF087FB336820F071
:104780000F0203F00F031A43294612480DF06FFB86
:104790000024FFF73FBB0D0145F06D05EDB2294642
:1047A0000C4834B90DF071FBC0F300603060FFF7C6
:1047B00031BB0DF06AFB336820F080721B0603F0FA
:1047C00080731A43294603480DF051FB0024FFF77C
:1047D00021BB00BF842F00200D0145F06D05EDB217
:1047E00029468B486CB90DF050FB001400F07F0394
:1047F00010F0400018BF6FF07F0018433060FFF7E3
:1048000009BB0DF042FB336820F4FE021B0403F4E5
:10481000FE031A4329467E480DF029FB0024FFF7CA
:10482000F9BA0D0145F06C05EDB22946784834B966
:104830000DF02BFBC0F340403060FFF7EBBA0DF0FA
:1048400024FB336820F400325B0403F400331A4382
:1048500029466F480DF00BFB0024FFF7DBBA002858
:1048600040F0CF80090141F06F01C9B268480DF0F6
:104870000CFBC0F304403060FFF7CCBA202101FAF2
:1048800005F56DB245F01101C9B228B960480DF0C7
:10489000FCFA3060FFF7BEBA45F014051A685C48B0
:1048A000EDB20DF0E4FA294659480DF0EEFA3368FE
:1048B00020F48062002B18BF4FF4806329461A430E
:1048C00053480DF0D4FA0024FFF7A4BA2021A940E0
:1048D00041F01101C9B228B94D480DF0D6FA306047
:1048E000FFF798BA1A684A480DF0C1FA0024FFF79A
:1048F00091BA0D0145F06C05EDB22946444834B932
:104900000DF0C3FAC0F340303060FFF783BA0DF00A
:10491000BCFA336820F400525B0303F400531A43DB
:1049200029463B480DF0A3FA0024FFF773BA00288C
:104930006AD1090141F06F01C9B235480DF0A5FAFD
:10494000C0F309003060FFF765BAC8B9012D014610
:104950002F480AD00DF099FA00F01800A0F11002CB
:10496000504250413060FFF755BA0DF08EFA00F01A
:104970006000A0F12003584258413060FFF74ABA66
:10498000012D4FF00001224811D00DF07EFA33685E
:1049900020F0180243B142F0100200211C480DF033
:1049A00066FA0024FFF736BA42F00802F5E70DF088
:1049B0006CFA336820F0600243B142F0200200211B
:1049C00013480DF054FA0024FFF724BA42F04002D5
:1049D000F5E70824FFF71EBA0424FFF71BBA0024EA
:1049E000FFF718BA0424FFF715BA0424FFF712BA28
:1049F0000424FFF70FBA0424FFF70CBA0424FFF7CE
:104A000009BA0424FFF706BA0424FFF703BA00BF6B
:104A1000842F002007B5019201AB02460120FFF769
:104A2000DBF903B05DF804FB134602460020FFF7F4
:104A3000D3B901480DF0E0BA842F0020012810B549
:104A4000144603D002280FD0042010BD0A4B0B4A95
:104A5000DB68D2F8A4021B685B6A9847003018BF75
:104A6000012020600020F0E7034B044ADB68D2F805
:104A7000A8021B685B6AF0E770A30208842F00207D
:104A8000022804BF0C4B93F8F00038B90B4BDB68DD
:104A90001B685B690A4AD2F8A0021847012809D1AD
:104AA000054B93F8F030012B04D1044BDB681B68F5
:104AB0009B69EFE7704700BF9C64002070A3020869
:104AC000842F002070B50020FFF7DAFF094B0A4C55
:104AD000DD68D4F8A0022B689B6898472B68D4F84F
:104AE000A4029B6898472B68D4F8A8029B68BDE88D
:104AF0007040184770A30208842F00200128F8B5E1
:104B000004460F461AD820250D4E854045F0070172
:104B100087EAE772A2EBE772C9B230460DF0A7F957
:104B20000123002F30463444ACBF1A460222E9B2BA
:104B300084F898320DF09BF90020F8BD0820FCE7BE
:104B4000842F00200021D9E74942D7E7D6E708B5EE
:104B5000222108480DF099F948B9422105480DF085
:104B600094F920B9BDE8084002480DF03DBA002094
:104B700008BD00BF842F0020034B0846D3F8AC3299
:104B80001146DB68184700BF842F0020F8B5304C71
:104B9000304D314F0021A2692846304B0DF09DF970
:104BA000FE68736803F5AC7203F1CC0003F5BA73C9
:104BB000C5F8A8323368C5F8A422DB68C5F8A0029E
:104BC00098473368D5F8A4021B6998473368D5F82D
:104BD000A8021B69984773683A6903F538735360F4
:104BE000C5F8AC22A3691E4AC5F89C32C3F804225A
:104BF0001C4A0220C3F8082201221A801A4B3222D2
:104C000063621A4B20752362194BE361194BA3624F
:104C1000194BE363194BA363194BE362194B2363ED
:104C2000194BE364194BA364194BA365194B6365D6
:104C3000194B2365194B6366194B23664FF48C732C
:104C4000C4E90332174BE365BDE8F84018E700BF3D
:104C50009C640020842F002070A302086899020839
:104C60004F4B0108334A0108FD4A01084D4B01082A
:104C7000494B0108454B0108294A0108154A01081A
:104C8000553D0108B13D0108493D0108353D010888
:104C9000293D01083D4A0108013D0108814A0108FA
:104CA0001D3D0108C54A010801289FBF044B03EBC5
:104CB0008003DB69002094BF0B600820704700BFB1
:104CC000403200200022014B9A6070479C64002013
:104CD000014601480DF025BB403200200A4601463E
:104CE00001480DF0BFB900BF4032002010B50020D0
:104CF0001446FFF7F3FF206010BD38B514460A468E
:104D0000014603481D460DF0ADF92040E84038BD8E
:104D10004032002013460A46014601480DF09EB974
:104D2000403200200020F5E701282DE9F04104463B
:104D300088461FD82025104F854007EB8007D7F8FD
:104D4000A4226EB23AB146F00701C9B2FFF7E2FF02
:104D50000023C7F8A43246F00D014246C9B22046EE
:104D6000FFF7D8FF20460022E9B2FFF7D3FF00206B
:104D7000BDE8F0810820FBE74032002038B50D4641
:104D80002021814041F00101C9B20446FFF7A6FF8E
:104D90002968014429602046BDE83840C4E701285D
:104DA0002DE9F0410446884623D82025124F85403E
:104DB00007EB8007D7F8A43245F00706F6B223B90F
:104DC0003146FFF78BFFC7F8A40288EAE872A2EB2E
:104DD000E87231462046FFF79DFFB8F1000F2046EC
:104DE000ACBF01220222E9B2FFF794FF0020BDE828
:104DF000F0810820FBE700BF403200200021CEE711
:104E00004942CCE7CBE72DE9F0470C4D99460646E1
:104E10000F4690460A4601462846089C0DF022F9A6
:104E200004FA09F2424002EA080282EA000331462B
:104E30003A462846BDE8F0470DF010B94032002050
:104E400001292DE9F34104460D461E4600F2B085C6
:104E50001C2A00F0958260D80C2A00F0A8812ED878
:104E6000052A00F0318116D8022A00F0E3800AD822
:104E7000002A00F0BD80012A00F0CB8004242046E7
:104E800002B0BDE8F081032A00F0E880042A00F0B7
:104E9000F8800424F3E7082A00F0558107D8062A91
:104EA00000F02381072A00F038810424E7E70A2A6A
:104EB00000F059810B2A00F068810424DFE7122AF0
:104EC00000F0E58113D80F2A00F0AE8107D80D2A33
:104ED00000F083810E2A00F096810424CFE7102A87
:104EE00000F0B381112A00F0C1810424C7E7152A1C
:104EF00000F0008207D8132A00F0DA81142A00F0AB
:104F0000E8810424BBE7172A00F01882C0F003826E
:104F1000182A00F024820424B1E7AC2A00F0E283CE
:104F200037D8A52A00F0E18213D8A22A00F098828F
:104F300007D81D2A00F03B828C2A00F0418204240D
:104F40009DE7A32A00F0A382A42A00F0B7820424DC
:104F500095E7A82A00F0728307D8A62A00F01883E4
:104F6000A72A00F05683042489E7AA2A4FEA0111F0
:104F700000F0968340F2798341F06D01C9B20028B8
:104F800040F0A683052360222846FFF7B6FE306076
:104F900075E7B62A00F04C8413D8B32A00F0F183E9
:104FA00007D8AD2A00F0B583AE2A00F0CB830424E5
:104FB00065E7B42A00F0FE83B52A00F00B840424D0
:104FC0005DE7CE2A00F0798407D8B82A00F0438440
:104FD000B92A00F05984042451E7D22A00F09084C1
:104FE000D32A00F0A084D12A00F07784042446E775
:104FF0002021A94041F00D01C9B220B92846FFF790
:105000006DFE30603BE71A682846FFF783FE0024F8
:1050100035E72021A94041F00101C9B220B9284655
:10502000FFF75CFE30602AE71A682846FFF772FE39
:10503000002424E72021A94041F00701C9B220B98A
:105040002846FFF74BFE306019E71A682846002A09
:10505000B8BF5242FFF75EFE002410E7002840F080
:10506000AA842021A94041F00201C9B22846FFF7D5
:1050700035FE10F4000318BF4FF07F431843306033
:10508000FDE62021AC4BA940D3F8AC3241F0070734
:10509000BA00134410B95B683360F0E63268C9B2F5
:1050A000002AB8BF52425A602846FFF717FE04464E
:1050B00008B10024E3E63268F9B2002AB8BF5242D0
:1050C0002846FFF727FEDAE62021A94041F0060135
:1050D000C9B220B92846FFF701FE3060CFE61A6852
:1050E0002846FFF717FE0024C9E62021A94041F019
:1050F0001001C9B238B908234FF4F8522846FFF717
:10510000FCFD3060BBE61B684FF4F8520093284664
:105110000823FFF778FE0024B1E62021A94041F0E2
:105120001001C9B230B903461F222846FFF7E5FD3A
:105130003060A4E61B681F22009328460023FFF777
:1051400062FE00249BE6002840F038842021A9401C
:1051500041F0150109234FF40072C9B22846FFF748
:10516000CCFD30608BE6002840F02B842021A94044
:1051700041F0150101230222C9B22846FFF7BDFD07
:10518000B0FA80F04009306079E6002840F01C84D5
:105190002021A94041F0150103460122C9B2284649
:1051A000FFF7ABFDB0FA80F04009306067E62021E0
:1051B000A94041F01401C9B230B9012302222846A6
:1051C000FFF79BFD30605AE61B68022200932846D9
:1051D0000123FFF718FE002451E62021A94041F0E9
:1051E0001401C9B230B9034601222846FFF785FDF4
:1051F000306044E61B680122009328460023FFF735
:1052000002FE00243BE62021A94041F01401C9B26E
:1052100020B92846FFF762FD306030E61A6828465C
:10522000FFF778FD00242AE62021A94041F004017F
:10523000C9B220B92846FFF751FD30601FE61A6851
:105240002846FFF767FD002419E62021A94041F018
:105250000501C9B220B92846FFF740FD30600EE6CF
:105260001A682846FFF756FD002408E62021A940C9
:1052700041F00801C9B220B92846FFF72FFD306080
:10528000FDE51A682846FFF745FD0024F7E52021D3
:10529000A94041F00A01C9B220B92846FFF71EFD16
:1052A0003060ECE51A682846FFF734FD0024E6E597
:1052B0002021A94041F00301C9B220B92846FFF7D7
:1052C0000DFD3060DBE51A682846FFF723FD00245A
:1052D000D5E52021A94041F00B01C9B220B92846EB
:1052E000FFF7FCFC3060CAE51A682846FFF712FD9C
:1052F0000024C4E52021A94041F00C01C9B220B925
:105300002846FFF7EBFC3060B9E51A682846FFF73E
:1053100001FD0024B3E52021A94041F01101C9B2EB
:1053200020B92846FFF7DAFC3060A8E51A6828465D
:10533000FFF7F0FC0024A2E5403200202021A94024
:1053400041F01201C9B220B92846FFF7C7FC30600E
:1053500095E51A682846FFF7DDFC00248FE520213B
:10536000A94041F01301C9B220B92846FFF7B6FCA5
:10537000306084E51A682846FFF7CCFC00247EE5FF
:10538000090141F06C01C9B238B912234FF48022EF
:105390002846FFF7B2FC306071E51B684FF48022AD
:1053A000009328461223FFF72EFD002467E500280E
:1053B00040F00D83B94B03EB8105EB6933605EE58B
:1053C00080B9090141F06C0118234FF0706201F0BF
:1053D000FC012846FFF791FC4FF4807343FA00F07C
:1053E00030604CE51B68102B34D00DDC022B2DD027
:1053F00004DC012B16D04FF0FF3314E0042B27D030
:10540000082BF8D105230EE0402B25D003DC202B00
:10541000F1D1032307E0802B20D0B3F5807FEAD1C0
:10542000002300E00823336033685C1C3FF441AE86
:10543000290141F06C0100934FF07062182301F0D4
:10544000FC012846FFF7DFFC002418E50723EAE704
:105450000623E8E70423E6E70223E4E70123E2E783
:10546000090141F06C01C9B238B90F234FF4C032C1
:105470002846FFF742FC306001E51B684FF4C0325C
:10548000009328460F23FFF7BEFC0024F7E4090130
:1054900041F06C01C9B238B90E234FF4804228465E
:1054A000FFF72BFC3060EAE41B684FF48042009366
:1054B00028460E23FFF7A7FC0024E0E4090141F091
:1054C0006C01C9B238B90C234FF480522846FFF75B
:1054D00014FC3060D3E41B684FF4805200932846DC
:1054E0000C23FFF790FC0024C9E40F0147F06C0780
:1054F000FFB240BB0E234FF4804239462846FFF7E7
:10550000FCFB804640B107234FF4F0623946284641
:10551000FFF7F3FB3060B2E40423702239462846DB
:10552000FFF7EBFB0B2330604FF40062394628464F
:10553000FFF7E3FB00283FF4BCAD3368444643F07B
:10554000080333609BE439462846FFF7C7FB10F495
:105550008044336809D000934FF4F0620723394642
:105560002846FFF750FC002489E4C3F3C0030093EE
:10557000394628460B234FF40062FFF744FC33689A
:1055800070220093394604232846FFF73CFC76E45A
:105590000F0147F06C07FFB23946284614BBFFF7EE
:1055A0009DFB400407D50423702239462846FFF7A7
:1055B000A4FB306063E407234FF4F06239462846C9
:1055C000FFF79BFB0B2330604FF4006239462846FF
:1055D000FFF793FB00283FF46CAD336843F00803FA
:1055E00033604CE4FFF77AFB336810F48044009397
:1055F00007D00423702239462846FFF704FC002414
:105600003DE407234FF4F06239462846FFF7FBFBE1
:1056100035E4090141F06C01C9B230B903460F22EB
:105620002846FFF76AFB306029E41B680F220093CD
:1056300028460023FFF7E7FB002420E4090141F09E
:105640006D01C9B238B90F234FF400422846FFF765
:1056500054FB306013E41B684FF40042009328466B
:105660000F23FFF7D0FB002409E441F06D01C9B21C
:1056700040B90D234FF4C0422846FFF73EFB30608F
:10568000FFF7FDBB1B684FF4C042009328460D2373
:10569000FFF7B9FB0024FFF7F2BB00BF4032002048
:1056A00041F06D01C9B240B908234FF47062284639
:1056B000FFF723FB3060FFF7E2BB1B684FF470621B
:1056C000009328460823FFF79EFB0024FFF7D7BB73
:1056D0001B686022009328460523FFF794FB0024F3
:1056E000FFF7CDBB090141F06D01C9B238B90346DE
:1056F0000F222846FFF701FB3060FFF7C0BB1B6895
:105700000F22009328460023FFF77DFB0024FFF7BC
:10571000B6BB090141F06D01C9B240B918234FF081
:1057200080722846FFF7E9FA3060FFF7A8BB1B68D4
:105730004FF08072009328461823FFF764FB002483
:10574000FFF79DBB090141F06D01C9B270B910238B
:105750004FF4FE022846FFF7D0FA10F0400318BFBE
:105760006FF07F0318433060FFF789BB1B684FF46D
:10577000FE02009328461023FFF745FB0024FFF7A5
:105780007EBB090141F06C01C9B240B911234FF44D
:1057900000322846FFF7B1FA3060FFF770BB1B6894
:1057A0004FF40032009328461123FFF72CFB00240E
:1057B000FFF765BB002840F00D81090141F06F0142
:1057C00010234FF4F812C9B22846FFF796FA30605A
:1057D000FFF755BB20278F407FB247F014085FFAD0
:1057E00088F878B941462846FFF778FA41057FF5F1
:1057F00060AC47F01101C9B22846FFF76FFA30607C
:10580000FFF73DBB47F011011A68C9B22846FFF700
:1058100081FA33684FF48062003318BF0123414698
:10582000009328460A23FFF7EEFA0024FFF727BB70
:105830002021A94041F01101C9B228B92846FFF73B
:105840004DFA3060FFF71BBB1A682846FFF762FA73
:105850000024FFF714BB090141F06C01C9B240B943
:105860000D234FF400522846FFF747FA3060FFF748
:1058700006BB1B684FF40052009328460D23FFF728
:10588000C2FA0024FFF7FBBA090141F06C01C9B26A
:1058900040B914234FF470022846FFF72EFA306007
:1058A000FFF7EDBA1B684FF47002009328461423EB
:1058B000FFF7A9FA0024FFF7E2BA002840F08D8034
:1058C000090141F06F01034640F2FF32C9B2284698
:1058D000FFF713FA3060FFF7D2BA2021A94041F058
:1058E0001901C9B228B92846FFF7F8F93060FFF767
:1058F000C6BA1A682846FFF70DFA0024FFF7BFBAA8
:105900002021A94041F01A01C9B228B92846FFF761
:10591000E5F93060FFF7B3BA1A682846FFF7FAF9DD
:105920000024FFF7ACBAC8B9012D01460AD0FFF731
:10593000D5F900F01800A0F110025042504130603B
:10594000FFF79DBA2846FFF7C9F900F06000A0F103
:105950002003584258413060FFF791BA012D4FF0B3
:10596000000112D00846FFF7B9F9336820F0180299
:1059700043B142F0100200210846FFF7CBF90024A2
:10598000FFF77DBA42F00802F5E72846FFF7A6F9CF
:10599000336820F0600243B142F020020021012070
:1059A000FFF7B8F90024FFF76ABA42F04002F5E7C2
:1059B0000824FFF764BA0424FFF761BA0424FFF750
:1059C0005EBA0424FFF75BBA0424FFF758BA042434
:1059D000FFF755BA0424FFF752BA0424FFF74FBA71
:1059E00007B5019201AB02460120FFF729FA03B087
:1059F0005DF804FB134602460020FFF721BA014878
:105A00000CF0F0BB40320020012838B5144613D00A
:105A100045B21DB102281CD0042038BD114B124ADA
:105A2000DB6824681B68D2F8BC021CB15B6998472C
:105A30000020F2E79B69FAE70A4B0B4ADB68D2F8D1
:105A4000B4021B685B6A9847003018BF01202060D1
:105A5000EEE7044B044ADB68D2F8B8021B685B6AC5
:105A6000F1E700BF70A3020840320020022804BF03
:105A70000C4B93F8F00038B90B4BDB681B685B6983
:105A80000A4AD2F8B0021847012809D1054B93F809
:105A9000F030012B04D1044BDB681B689B69EFE7F6
:105AA000704700BF9C64002070A3020840320020B1
:105AB00070B50020FFF7DAFF134B144CDD68D4F803
:105AC000B0022B689B6898472B68D4F8B4029B6897
:105AD00098472B68D4F8B8029B6898472B68D4F88D
:105AE000C8029B6898472B68D4F8C0029B68984707
:105AF0002B68D4F8C4029B6898472B68D4F8BC0282
:105B00009B68BDE87040184770A30208403200202F
:105B100008B522210020FFF7E1F848B94221012011
:105B2000FFF7DCF820B9BDE8084002480CF043BBA1
:105B3000002008BD40320020012938B505460C463A
:105B40000FD1084B102200210CF088FA2846054B93
:105B5000214618220CF082FABDE8384002480CF0C9
:105B6000F7BA38BDC804050040320020012810B43F
:105B70000C4607D8054B2046D3F8CC3211469B681B
:105B800010BC1847002010BC704700BF40320020F6
:105B90002DE9F04101275F4C5F4DA1695F4B8CB04F
:105BA000C5F8AC125E4ACDE9007328460023DFF841
:105BB000D8810CF0A3FA5B4928460CF0F8FAD8F823
:105BC0000C60736803F5AC72C5F8B42203F5BA72C1
:105BD000C5F8B82203F57072C5F8BC2203F57772D8
:105BE00003F1CC00C5F8C02203F57E7203F2144322
:105BF000C5F8C8323368C5F8C422DB68C5F8B002FE
:105C000098473368D5F8BC02DB6898473368D5F805
:105C1000BC029B6998473368D5F8B4021B69984762
:105C20003368D5F8B8021B6998473368D5F8C802BD
:105C30001B6998473368D5F8C0021B6998473368D9
:105C4000D5F8C4021B6998476FF080617368D8F873
:105C5000102003F538735360334BC5F8CC22029300
:105C600003F19F2303F56A03563303932F4A304B06
:105C70003048CDE90423304B02AACDE90613A3F145
:105C8000D943A3F59113A3F2272308932B4B0021AB
:105C9000CDE909034FF477432846ADF82C300CF0DA
:105CA000DAFB02AA394628460CF0D5FBA369244A40
:105CB0001F80C3F80422234A3225C3F80822224B4E
:105CC00038466362214B2362214BE361214BA3627F
:105CD000214BE363214BA363214BE362214B2363FD
:105CE000214BE364214BA364214BA365214B6365E6
:105CF000214B2365214B6366214B236602232375C9
:105D0000DE23C4E903351F4BE365FFF7AFFE0CB09C
:105D1000BDE8F0819C640020403200200024F400A3
:105D2000689B0208395B010854B5AAAA29294924AD
:105D300022421010224240007D77BBB580FFFF5603
:105D4000115B0108FF5901089F4D0108054E01082C
:105D5000014E0108FD4D0108F5590108E1590108FE
:105D6000294D01087D4D0108254D0108ED4C010824
:105D7000D14C0108095A0108A94C01086D5A0108C3
:105D8000C54C0108B15A010870A3020801289FBF41
:105D9000044B03EB8003DB68002094BF0B600820FA
:105DA000704700BF1C3500200022014B9A607047ED
:105DB0009C64002038B50546054C014620460CF091
:105DC000E3FC29462046BDE838400CF0DDBC00BFAE
:105DD0001C35002010B5034814460CF066FC20600A
:105DE00010BD00BF1C35002001480CF050BC00BFA6
:105DF0001C3500200129F8B504461E4600F25386E2
:105E00001C2A00F0CD825ED80C2A00F0A4812CD888
:105E1000052A00F0258114D8022A00F0D78008D87E
:105E2000002A00F0AF80012A00F0BE800424204642
:105E3000F8BD032A00F0DF80042A00F0F08004247B
:105E4000F5E7082A00F0578107D8062A00F01A81E2
:105E5000072A00F034810424E9E70A2A00F05B8174
:105E60000B2A00F068810424E1E7122A00F01A826C
:105E700013D80F2A00F0DD8107D80D2A00F0998190
:105E80000E2A00F0C4810424D1E7102A00F0E68134
:105E9000112A00F0F5810424C9E7152A00F03882A0
:105EA00007D8132A00F01082142A00F01F8204245D
:105EB000BDE7172A00F05082C0F03C82182A00F09B
:105EC0005D820424B3E7AB2A00F03D842BD8A52AD9
:105ED00000F0358313D8A22A00F0DA8207D81D2AF1
:105EE00000F07A828C2A00F0808204249FE7A32AA3
:105EF00000F0EA82A42A00F00383042497E7A82A8A
:105F000000F0C88307D8A62A00F06283A72A00F011
:105F1000A48304248BE7A92A00F0D983AA2A00F0DD
:105F2000F483042483E7B52A00F0BB8413D8AE2A97
:105F300000F0628407D8AC2A00F02384AD2A00F078
:105F40003D84042473E7B32A00F07E84B42A00F071
:105F5000998404246BE7CE2A00F00B8507D8B62A73
:105F600000F0D584B82A00F0E68404245FE7D22A42
:105F700000F02585D32A00F03685D12A00F0088567
:105F8000042454E7202303FA01F141F00D01C9B2C2
:105F900020B9B1480CF089FB306048E73268AE4860
:105FA0000CF075FB002442E7202303FA01F141F0D5
:105FB0000101C9B220B9A8480CF077FB306036E780
:105FC0003268A5480CF063FB002430E7202303FA75
:105FD00001F141F00701C9B220B99F480CF065FBFF
:105FE000306024E732689C48002AB8BF52420CF067
:105FF0004EFB00241BE7002840F05885202303FABD
:1060000001F141F00201C9B293480CF04EFB10F4CB
:10601000000318BF4FF07F431843306007E78E4FEF
:106020008D003D4418B9D5F898323360FFE620263C
:106030001B688E40002BB8BF5B42F1B23846C5F8F2
:1060400098320CF032FB0446002840F0328546F0CE
:106050000701D5F89822C9B238460CF018FBE6E6DD
:10606000202303FA01F141F00601C9B220B97A48B0
:106070000CF01BFB3060DAE6326877480CF007FB67
:106080000024D4E620258D4045F01005EDB22946C8
:1060900071482CB90CF009FBC0F304203060C6E64F
:1060A0000CF003FB336820F4F8521B0203F4F8539E
:1060B0001A43294668480CF0EAFA0024B7E620257E
:1060C0008D4045F01005EDB2294663482CB90CF01F
:1060D000ECFA00F01F003060A9E60CF0E6FA336835
:1060E00020F01F0203F01F031A4329465A480CF000
:1060F000CEFA00249BE6002840F0DE84202303FA39
:1061000001F141F01501C9B253480CF0CEFAC0F3C9
:10611000402030608BE6002840F0D184202303FA31
:1061200001F141F01501C9B24B480CF0BEFAC0F3C1
:10613000400030607BE6002840F0C484202303FA4E
:1061400001F141F01501C9B243480CF0AEFA00F07C
:10615000010030606BE620258D4045F01405EDB25E
:1061600029463D482CB90CF0A0FAC0F3400030603D
:106170005DE60CF09AFA336820F00202002BCCBFE7
:106180000223002329461A4333480CF080FA29469B
:1061900031480CF08AFA336820F00802022B0CBF59
:1061A0000823002329461A432B480CF070FA0024D8
:1061B0003DE620258D4045F01405EDB229462648E0
:1061C0002CB90CF072FA00F0010030602FE60CF0F0
:1061D0006CFA326820F00100002AD4BF024640F079
:1061E000010229461C480CF052FA29461A480CF0C4
:1061F0005CFA336820F00402022B0CBF0423002356
:1062000029461A4314480CF042FA00240FE62023D2
:1062100003FA01F141F01401C9B220B90E480CF0A3
:1062200044FA306003E632680B480CF030FA002480
:10623000FDE5202303FA01F141F00401C9B220B9C0
:1062400005480CF032FA3060F1E5326802480CF093
:106250001EFA0024EBE500BF1C350020202303FAC2
:1062600001F141F00501C9B220B9AC480CF01DFAAA
:106270003060DCE53268A9480CF009FA0024D6E564
:10628000202303FA01F141F00801C9B220B9A34863
:106290000CF00BFA3060CAE53268A0480CF0F7F950
:1062A0000024C4E5202303FA01F141F00A01C9B238
:1062B00020B99A480CF0F9F93060B8E5326897488F
:1062C0000CF0E5F90024B2E5202303FA01F141F0D6
:1062D0000301C9B220B991480CF0E7F93060A6E596
:1062E00032688E480CF0D3F90024A0E5202303FA8D
:1062F00001F141F00B01C9B220B988480CF0D5F981
:10630000306094E5326885480CF0C1F900248EE5D0
:10631000202303FA01F141F00C01C9B220B97F48F2
:106320000CF0C3F9306082E532687C480CF0AFF9BC
:1063300000247CE5202303FA01F141F01101C9B2E8
:1063400020B976480CF0B1F9306070E532687348D6
:106350000CF09DF900246AE5202303FA01F141F0D5
:106360001201C9B220B96D480CF09FF930605EE5AA
:1063700032686A480CF08BF9002458E5202303FAB0
:1063800001F141F01301C9B220B964480CF08DF954
:1063900030604CE5326861480CF079F9002446E53C
:1063A000090141F06C05EDB229465C482CB90CF0AE
:1063B0007CF9C0F38040306039E50CF076F9336841
:1063C00020F480229B0403F480231A432946534877
:1063D0000CF05DF900242AE5002840F076834F4B4D
:1063E00003EB8101CB68336021E570B9090141F00D
:1063F0006C0101F0FC0149480CF057F94FF480732F
:1064000000F00F000341336011E51B68102B39D0F9
:106410000FDC022B32D006DC012B18D04FF0FF33FB
:106420000024336003E5042B2AD0082BF6D1052382
:106430000EE0402B28D003DC202BEFD1032307E014
:10644000802B23D0B3F5807FE8D1002300E0082320
:10645000090141F06C04E4B2214633602F480CF08E
:1064600024F9336820F070621B0603F07063214644
:106470001A432A480CF00BF90024D8E40723E7E775
:106480000623E5E70423E3E70223E1E70123DFE74F
:10649000090141F06C05EDB2294620482CB90CF0F9
:1064A00004F9C0F3C1303060C1E40CF0FEF8336889
:1064B00020F4C032DB0303F4C0331A4329461748E3
:1064C0000CF0E5F80024B2E4090141F06C05EDB2EE
:1064D000294612482CB90CF0E8F8C0F3403030607F
:1064E000A5E40CF0E2F8336820F400525B0303F4F7
:1064F00000531A43294609480CF0C9F8002496E4D1
:10650000090141F06C05EDB22946044844B90CF08C
:10651000CCF8C0F30030306089E400BF1C350020A7
:106520000CF0C3F8336820F480521B0303F480534B
:106530001A432946C3480CF0AAF8002477E409015D
:1065400041F06C05EDB22946BE480CF0AEF8294684
:10655000C0F38037BB486CB92FB10CF0A6F8C0F37C
:10656000C310306063E40CF0A0F8C0F30210306098
:106570003C465CE477B10CF098F8336820F4F062A4
:10658000DB0103F4F0631A432946AE480CF07FF8B0
:1065900000244CE40CF089F8326820F40060120208
:1065A00002F4006202432946A6480CF070F829461E
:1065B000A4480CF07AF8336820F070021B0103F055
:1065C00070031A4329469F480CF061F83C462EE4BC
:1065D000090141F06C05EDB229469A480CF065F8C6
:1065E0002946C0F380379748B4B92FB10CF05DF855
:1065F000C0F3021030601AE40CF057F8C0F3C31077
:10660000306029468F480CF050F83368000A00F0DB
:106610000800034333600AE47FB10CF046F83368A6
:1066200020F070021B0103F070031A4329468548CD
:106630000CF02DF80024FFF7FABB0CF036F83368A5
:1066400020F4F062DB0103F4F0631A4329467D482D
:106650000CF01DF83C46FFF7EABB090141F06C0560
:10666000EDB22946774834B90CF01FF800F00F005E
:106670003060FFF7DCBB0CF018F8336820F00F0235
:1066800003F00F031A4329466E480CF000F800246B
:10669000FFF7CDBB090141F06D05EDB22946694810
:1066A00034B90CF002F8C0F3C0303060FFF7BFBB64
:1066B0000BF0FBFF336820F40042DB039BB21A436C
:1066C000294660480BF0E3FF0024FFF7B0BB090147
:1066D00041F06D05EDB229465A4834B90BF0E5FF9B
:1066E000C0F341303060FFF7A2BB0BF0DEFF336830
:1066F00020F4C0425B0303F4C0431A4329465148C7
:106700000BF0C5FF0024FFF792BB090141F06D05B6
:10671000EDB229464B4834B90BF0C7FFC0F3032054
:106720003060FFF784BB0BF0C0FF336820F4706269
:106730001B0203F470631A43294642480BF0A7FF7B
:106740000024FFF774BB090141F06D05EDB2294645
:106750003C4834B90BF0A9FFC0F341103060FFF79B
:1067600066BB0BF0A2FF336820F060025B0103F010
:1067700060031A43294633480BF089FF0024FFF7D2
:1067800056BB090141F06D05EDB229462D4834B9DB
:106790000BF08BFF00F00F003060FFF748BB0BF0F1
:1067A00084FF336820F00F0203F00F031A432946D9
:1067B00024480BF06CFF0024FFF739BB090141F0BE
:1067C0006D05EDB229461F4834B90BF06EFFC0F3DA
:1067D00000603060FFF72BBB0BF067FF336820F0E1
:1067E00080721B0603F080731A43294615480BF08C
:1067F0004EFF0024FFF71BBB090141F06D05EDB210
:10680000294610486CB90BF050FF001400F07F03CC
:1068100010F0400018BF6FF07F0018433060FFF7A2
:1068200006BB0BF042FF336820F4FE021B0403F4A6
:10683000FE031A43294603480BF029FF0024FFF703
:10684000F6BA00BF1C350020090141F06C05EDB21D
:106850002946A24834B90BF028FFC0F3404030600D
:10686000FFF7E5BA0BF021FF336820F400325B0438
:1068700003F400331A43294698480BF008FF00241C
:10688000FFF7D5BA002840F02381090141F06F01DC
:10689000C9B292480BF009FFC0F304403060FFF723
:1068A000C6BA202505FA01F14DB245F01407FFB232
:1068B00098B9394689480BF0F8FE10F4806008D08A
:1068C00045F01101C9B285480BF0EFFE3060FFF7CB
:1068D000AEBA30600446FFF7AABA45F011011A6853
:1068E000C9B27E480BF0D3FE39467C480BF0DDFE82
:1068F000336820F48062002B18BF4FF48063394660
:106900001A4376480BF0C3FE0024FFF790BA202309
:1069100003FA01F141F01101C9B228B96F480BF037
:10692000C4FE3060FFF783BA32686C480BF0AFFEEC
:106930000024FFF77CBA090141F06C05EDB229464D
:10694000664834B90BF0B1FEC0F340303060FFF759
:106950006EBA0BF0AAFE336820F400525B0303F416
:1069600000531A4329465D480BF091FE0024FFF7BF
:106970005EBA002840F0AF80090141F06F01C9B252
:1069800056480BF092FEC0F309003060FFF74FBA93
:1069900020258D4045F01905EDB229464F4824B910
:1069A0000BF083FE3060FFF742BA0BF07EFE3268D8
:1069B00029464A480BF06BFE0024FFF738BA202323
:1069C00003FA01F141F01A01C9B228B943480BF0AA
:1069D0006CFE3060FFF72BBA326840480BF057FE70
:1069E0000024FFF724BAC8B9012901463B480AD060
:1069F0000BF05BFE00F01800A0F110025042504175
:106A00003060FFF714BA0BF050FE00F06000A0F108
:106A10002003584258413060FFF709BA01292F4836
:106A20004FF000011FD00BF040FE336820F0080249
:106A3000002B0CBF0823002300211A4327480BF02A
:106A400026FE002125480BF030FE336820F01002AE
:106A5000002B18BF102300211A4320480BF017FE0B
:106A60000024FFF7E4B90BF020FE336820F0200289
:106A7000002B18BF202300211A4318480BF007FEF3
:106A8000002116480BF011FE336820F04002002B65
:106A90000CBF4023002300211A4310480BF0F7FDE0
:106AA0000024FFF7C4B90824FFF7C1B90424FFF795
:106AB000BEB90024FFF7BBB90424FFF7B8B904241A
:106AC000FFF7B5B90424FFF7B2B90424FFF7AFB953
:106AD0000424FFF7ACB90424FFF7A9B91C35002042
:106AE00007B5019201AB02460120FFF783F903B01D
:106AF0005DF804FB134602460020FFF77BB910B592
:106B0000044605480B4600EB8402D2F89822214641
:106B10000BF027FF002010BD1C35002010B50446E7
:106B200005480A4600EB8403D3F8983221460BF05F
:106B3000FAFE002010BD00BF1C35002008B501463C
:106B400002480BF0EDFE002008BD00BF1C35002000
:106B500008B50A46014602480BF0DFFE002008BDDA
:106B60001C35002008B50A46014602480BF0D3FE4A
:106B7000002008BD1C35002008B50A460146024821
:106B80000BF0ABFE002008BD1C35002001480BF0C7
:106B90008CBE00BF1C350020012838B5144613D028
:106BA00045B21DB102281CD0042038BD114B124A39
:106BB000DB6824681B68D2F8AC021CB15B6998479B
:106BC0000020F2E79B69FAE70A4B0B4ADB68D2F830
:106BD000A4021B685B6A9847003018BF0120206040
:106BE000EEE7044B044ADB68D2F8A8021B685B6A34
:106BF000F1E700BF70A302081C350020022804BF83
:106C00000C4B93F8F00038B90B4BDB681B685B69E1
:106C10000A4AD2F8A0021847012809D1054B93F877
:106C2000F030012B04D1044BDB681B689B69EFE754
:106C3000704700BF9C64002070A302081C35002030
:106C400070B50020FFF7DAFF134B144CDD68D4F861
:106C5000A0022B689B6898472B68D4F8A4029B6815
:106C600098472B68D4F8A8029B6898472B68D4F8FB
:106C7000B8029B6898472B68D4F8B0029B68984785
:106C80002B68D4F8B4029B6898472B68D4F8AC0200
:106C90009B68BDE87040184770A302081C350020AF
:106CA00008B5222107480BF000FD48B942210548EC
:106CB0000BF0FBFC20B9BDE8084002480BF0DEBD3C
:106CC000002008BD1C350020012910B504460DD157
:106CD000074A10210BF0DBFC2046054A18210BF077
:106CE000D6FCBDE8104003480BF02ABD10BD00BF24
:106CF000C80405001C350020034B0846D3F8BC32FD
:106D00001146DB68184700BF1C350020F8B54A4C17
:106D10004A4DA2694A4B28464A4F00210BF0EDFC30
:106D2000494928460BF0D5FDFE68736803F5AC723F
:106D3000C5F8A42203F5BA72C5F8A82203F570724B
:106D4000C5F8AC2203F5777203F1CC00C5F8B02288
:106D500003F57E7203F21443C5F8B8323368C5F800
:106D6000B422DB68C5F8A00298473368D5F8AC02B6
:106D7000DB6898473368D5F8AC029B69984733685D
:106D8000D5F8A4021B6998473368D5F8A8021B6997
:106D900098473368D5F8B8021B6998473368D5F827
:106DA000B0021B6998473368D5F8B4021B6998474D
:106DB00073683A6903F538735360C5F8BC22A36958
:106DC000224A0220C3F80422214AC3F808220122E1
:106DD0001A80204B322263621F4B207523621F4BA7
:106DE000E3611F4BA3621F4BE3631F4BA3631F4B66
:106DF000E3621F4B23631F4BE3641F4BA3641F4BD2
:106E0000A3651F4B63651F4B23651F4B63661F4BB9
:106E100023664FF48C73C4E903321D4BE3652B6882
:106E2000D3F8A020D3F82031C5F89822C5F89C32B9
:106E3000BDE8F840E2E600BF9C6400201C3500205D
:106E4000689D020870A30208C96C0108A16C0108C2
:106E50008D6B0108796B0108656B0108516B0108A6
:106E60003D6B0108F56A0108E16A01081D6B010824
:106E7000FF6A0108E95D0108D55D0108B55D0108FB
:106E8000996B01088D5D0108FD6B0108A95D010882
:106E9000416C010818B9034B5B680B607047082010
:106EA000704700BFE83700200022014B9A6070470E
:106EB0009C6400200428F8B5144672D00AD8012832
:106EC0003DD0A0B102285AD003280CBF00240424CE
:106ED0002046F8BD062800F09180C0F08380072886
:106EE00000F09480FC2800F09D800424F0E71268F4
:106EF00032F0030340F0A780544B554DDE68D207B3
:106F0000D5F8940233680BD51B699847246832681A
:106F100014F00204D5F8900209D0136998472CE0C8
:106F2000DB6898473368D5F894029B69EDE7D3682E
:106F300098473368D5F890029B699847C8E744F6AC
:106F4000206312689A427EDC42F21071404B8A4202
:106F5000D3F8B4023D4BDB681B68CCBF5B699B690F
:106F6000984742F211732268002092FBF3F103FB71
:106F70001121384B89B29B6898470024A8E7334B0E
:106F80001468DD68D5E9003000F507703CB1DB68B6
:106F90009847D5E900309B6900F50770BEE79B680C
:106FA000CBE72A4B2A4EDF6815683B68D6F8A0026B
:106FB0004DB1012D11D01B6998473B68D6F8A0024E
:106FC0005B6A984707E0DB6898473B689B69D6F89F
:106FD000A002984728462060CFE7DB6898473B68C7
:106FE0005B69F4E7194B1A4ADB68D2F8AC021B68FC
:106FF0005B6A9847003018BF0120ECE7134B144A36
:10700000DB68D2F8B0021B685B6AF2E7104B1268CB
:10701000D3F8A8020D4B012ADB681B680CBF5B6923
:107020009B697BE7094B0A4DDE6814683368D5F825
:10703000A00234B1DB6898473368D5F8A0029B6999
:107040006CE71B6979E7102442E700BF70A30208D0
:10705000E8370020800A0020224B70B5DD68224C02
:107060002B68D4F898029B6998472B68D4F8B8022B
:107070009B6898472B68D4F8B4029B6898472B68A4
:10708000D4F89C029B6898472B68D4F8A0029B68B0
:1070900098472B68D4F8A4029B6898472B68D4F8CB
:1070A00090029B6898472B68D4F894029B68984795
:1070B0002B68D4F8AC029B6898472B68D4F8B002D0
:1070C0009B6898472B68D4F8A8029B6898472B6860
:1070D000D4F898029B689847BDE87040034B5B6802
:1070E000184700BF70A30208E8370020800A00207C
:1070F00001480BF080BC00BFE83700200146014882
:107100000BF029BDE837002010B5034814460BF0FA
:1071100080FC206010BD00BFE8370020F8B50646AF
:107120001D460C46002940F081868C2A00F0E18241
:1071300079D80E2A00F0D0813CD8062A00F041818F
:107140001BD8022A00F0FC8008D8002A00F0DA8060
:10715000012A00F0E68004242046F8BD042A00F04D
:107160000D8140F2FB80002840F024812621C14897
:107170000BF04FFC34462860EEE70A2A00F05D81F0
:1071800007D8072A00F03581082A00F04A81042434
:10719000E2E70C2A00F0708140F25E813421B548AC
:1071A000002E40F086810BF034FC00F001002860D6
:1071B0003446D1E7152A00F0EE811AD8112A00F0E2
:1071C000B78107D80F2A00F09581102A00F0A1811D
:1071D0000424C1E7132A00F0C88140F2B7810028D7
:1071E00040F0D2812B21A3480BF013FC34462860D9
:1071F000B2E71C2A00F028820AD8182A00F0FC8185
:107200001B2A00F00882172A00F0D3810424A3E788
:10721000212A00F03982222A00F050821D2A00F033
:107220002B82042498E7B32A00F04D8436D8A82A8C
:1072300000F087831CD8A42A00F0DD8207D8A22A98
:1072400000F0A782A32A00F0BD82042484E7A62AC6
:1072500000F0278340F2E7826C218648002E40F040
:1072600062830BF0D6FB00F00F002860344673E712
:10727000AB2A00F0B48307D8A92A00F07A83AA2A9F
:1072800000F09283042467E7AD2A00F0DF83C0F0AA
:10729000C083AE2A00F0F58304245DE7BB2A00F02A
:1072A000F98415D8B62A00F0738407D8B42A00F000
:1072B0002484B52A00F02E8404244DE7B92A00F076
:1072C000A98400F2C284B82A00F08984042443E728
:1072D000CC2A00F063850AD8BF2A00F01A85C02A9C
:1072E00000F03C85BC2A00F0FD84042434E7D12A58
:1072F00000F07A85D22A00F08885CE2A00F06885D1
:10730000042429E730B92D215A480BF082FB34467A
:10731000286021E71A682D2156480BF06CFB0024E9
:107320001AE730B9212153480BF073FB344628602B
:1073300012E71A6821214F480BF05DFB00240BE790
:1073400030B927214B480BF064FB3446286003E733
:107350001A68272147480BF04EFBFDE6002840F055
:107360006885222143480BF054FB10F4000318BF3A
:107370004FF07F43184328603446EDE63D4F20B977
:10738000D7F8BC3204462B60E6E61B682021002BB0
:10739000B8BF5B423846C7F8BC320BF03AFB044634
:1073A000002840F04985D7F8BC22272138460BF049
:1073B00022FBD1E61A6826212E480BF01CFB002484
:1073C000CAE610212B4836B90BF023FBC0F304208A
:1073D00028603446C0E60BF01CFB2B6820F4F85202
:1073E0001B0203F4F8531A43102122480BF003FB4D
:1073F000B2E610211F4836B90BF00BFB00F01F005E
:1074000028603446A8E60BF004FB2B6820F01F022E
:1074100003F01F031A43102116480BF0ECFA002466
:107420009AE6002840F00B85352112480BF0F1FA5E
:10743000C0F34020286034468EE6002840F00285E4
:1074400035210C480BF0E5FA10F0020F0CBF0123B8
:10745000002334462B607FE6002840F0F684352177
:1074600004480BF0D6FAC04300F00100286034460F
:1074700072E600BFE83700203421A44836B90BF08B
:10748000C8FAC0F340002860344665E60BF0C1FA44
:107490002C6834B940F0020234219C480BF0ABFA5E
:1074A0005AE620F00202342198480BF0A4FA002496
:1074B00052E60BF0AEFA2C6834B940F001023421E8
:1074C00092480BF098FA47E620F0010234218F48E9
:1074D0000BF091FA00243FE630B934218B480BF0D1
:1074E00098FA3446286037E61A68342187480BF04A
:1074F00082FA31E630B9242184480BF08AFA344606
:10750000286029E61A68242180480BF074FA0024C8
:1075100022E630B925217D480BF07BFA34462860FD
:107520001AE61A68252179480BF065FA002413E65B
:1075300030B9282175480BF06CFA344628600BE608
:107540001A68282171480BF056FA05E630B92A214D
:107550006E480BF05EFA34462860FDE51A682A2171
:107560006A480BF048FA0024F6E530B92321674851
:107570000BF04FFA34462860EEE51A682321634881
:107580000BF039FA0024E7E51A682B215F480BF06D
:1075900032FA0024E0E530B92C215C480BF039FACE
:1075A00034462860D8E51A682C2158480BF023FA95
:1075B000D2E5574C70B9152154480BF02AFA30B176
:1075C0004FF08073B3FBF0F39C4228BF1C462C6045
:1075D0000024C1E51B686BB14FF0807292FBF3F29F
:1075E000A242A8BF22462A60152148480BF003FAA0
:1075F0000024B1E52246F6E730B9332143480BF0C9
:1076000008FA34462860A7E51A6833213F480BF092
:10761000F2F90024A0E56C213C4836B90BF0F9F9E9
:10762000C0F3C0402860344696E50BF0F2F92B68B1
:1076300020F40022DB0403F400231A436C213348B6
:107640000BF0D9F9002487E56C21304836B90BF0EE
:10765000E0F9C0F38040286034467DE50BF0D9F9AD
:107660002B6820F480229B0403F480231A436C21AE
:1076700026480BF0C0F96FE5002840F0E983234B62
:1076800004465B682B6067E540B901461F480BF074
:10769000C0F900F00100286034465DE500211B4878
:1076A0000BF0B7F92B6820F0010203F001031A4335
:1076B000002116480BF09FF900244DE540B9014622
:1076C00012480BF0A6F9C0F340002860344643E5A9
:1076D00000210E480BF09DF92B6820F002025B00A0
:1076E00003F002031A43002108480BF084F9002438
:1076F00032E578B96C2105480BF08BF94FF48073B3
:10770000C0F3036003412B60344625E5E8370020D1
:10771000FFFF0F001B68102B35D00FDC022B2ED083
:1077200006DC012B18D04FF0FF3310242B6013E53B
:10773000042B26D0082BF6D105230EE0402B24D0B5
:1077400003DC202BEFD1032307E0802B1FD0B3F500
:10775000807FE8D1296001E008232B606C21BA48C2
:107760000BF057F92B6820F070621B0603F0706372
:107770001A436C21B4480BF03EF90024ECE40723D3
:10778000EBE70623E9E70423E7E70223E5E7012324
:10779000E3E76C21AC4836B90BF03BF9C0F3C130DC
:1077A00028603446D8E40BF034F92B6820F4C0325A
:1077B000DB0303F4C0331A436C21A3480BF01BF91D
:1077C0000024C9E46C21A04836B90BF022F9C0F3BB
:1077D000803028603446BFE40BF01BF92B6820F49E
:1077E00080429B0303F480431A436C2196480BF0BC
:1077F00002F90024B0E46C21934836B90BF009F982
:10780000C0F3003028603446A6E40BF002F92B6880
:1078100020F480521B0303F480531A436C218A48DE
:107820000BF0E9F898E46C2187480BF0F2F800F4CB
:1078300080449EB944B16C2183480BF0EAF8C0F350
:10784000C3102860344687E4C0F3021300F40060DC
:10785000034314BF082300232B607DE484B16C2113
:1078600079480BF0D6F82B6820F4F062DB0103F4C2
:10787000F0631A436C2174480BF0BDF800246BE4EC
:107880002A6811074CBF40F4006020F40060120128
:1078900020F07000D2B202436C216B480BF0ABF8C1
:1078A0005AE46C2168480BF0B4F8AEB910F4804487
:1078B00008D06C2164480BF0ACF8C0F302102860CB
:1078C000344649E4C0F3C31300F40060034314BF1B
:1078D000082300232B603FE46C215B480BF099F8F0
:1078E00010F480444FF06C0157480ED00BF091F823
:1078F0002B6820F070021B0103F070031A436C2107
:1079000051480BF078F8002426E40BF082F82B683D
:1079100020F4F062DB0103F4F0631A436C214A485F
:107920000BF069F818E40BF074F82B6820F00F02E4
:1079300003F00F031A436C2143480BF05CF800245A
:107940000AE46D21404836B90BF063F8C0F3C0304B
:107950002860344600E40BF05CF82B6820F4004209
:10796000DB039BB21A436D2137480BF044F8FFF755
:10797000F3BB6D2134483EB90BF04BF8C0F34130F6
:1079800028603446FFF7E8BB0BF043F82B6820F47F
:10799000C0425B0303F4C0431A436D212A480BF035
:1079A0002AF80024FFF7D8BB6D2127483EB90BF019
:1079B00030F8C0F3032028603446FFF7CDBB0BF04E
:1079C00028F82B6820F470621B0203F470631A43DA
:1079D0006D211D480BF00FF80024FFF7BDBB6D2192
:1079E00019483EB90BF015F8C0F341102860344631
:1079F000FFF7B2BB0BF00DF82B6820F060025B01C3
:107A000003F060031A436D210F480AF0F4FFFFF7FB
:107A1000A3BB6D210C483EB90AF0FBFF00F00F003C
:107A200028603446FFF798BB0AF0F3FF2B6820F07C
:107A30000F0203F00F031A436D2103480AF0DBFF26
:107A40000024FFF789BB00BFE83700206D21B6484E
:107A50003EB90AF0DEFFC0F3006028603446FFF74D
:107A60007BBB0AF0D6FF2B6820F080721B0603F068
:107A700080731A436D21AC480AF0BDFF0024FFF764
:107A80006BBB6D21A84876B90AF0C3FF001400F063
:107A90007F0310F0400018BF6FF07F00184328608C
:107AA0003446FFF759BB0AF0B4FF2B6820F4FE02FE
:107AB0001B0403F4FE031A436D219B480AF09BFF4D
:107AC0000024FFF749BB6C2197483EB90AF0A1FF9B
:107AD000C0F3404028603446FFF73EBB0AF099FFF0
:107AE0002B6820F400325B0403F400331A436C214A
:107AF0008D480AF080FFFFF72FBB002840F0AB81D4
:107B00006F2189480AF085FFC0F30440286034469D
:107B1000FFF722BB34218448C6B90AF07AFF430537
:107B200010D5142180480AF074FF804B30B14FF01B
:107B30008072B2FBF0F2934228BF13462B60002400
:107B4000FFF70ABB2E603446FFF706BB0AF061FF61
:107B50002B6820F48062002B18BF4FF4806334211F
:107B60001A4371480AF047FF2968704B71B14FF012
:107B7000807292FBF1F29A42A8BF1A462A60142141
:107B800069480AF038FF0024FFF7E6BA1A46F5E71D
:107B900090B9142164480AF03CFF58B14FF080734B
:107BA000B3FBF0F0614B984228BF184628600024D0
:107BB000FFF7D2BA5D48F9E71B6873B14FF08072E6
:107BC00092FBF3F259498A42C8BF0A46142156482B
:107BD0000AF011FF0024FFF7BFBA544AF6E76C2100
:107BE00051483EB90AF015FFC0F3403028603446D2
:107BF000FFF7B2BA0AF00DFF2B6820F400525B03C6
:107C000003F400531A436C2147480AF0F4FE0024A1
:107C1000FFF7A2BA6C2144483EB90AF0FAFEC0F35D
:107C2000035028603446FFF797BA0AF0F2FE2B683B
:107C300020F470021B0503F470031A436C213A48C8
:107C40000AF0D9FE0024FFF787BA384C78B913211F
:107C500035480AF0DEFE30B14FF08073B3FBF0F32D
:107C60009C4228BF1C462C600024FFF775BA1B6895
:107C700073B14FF0807292FBF3F2A242A8BF22468A
:107C80002A60132128480AF0B6FE0024FFF764BAE0
:107C90002246F5E7702124483EB90AF0BAFEC0F347
:107CA000072028603446FFF757BA0AF0B2FE2A6868
:107CB00020F47F40120292B2024370211A480AF067
:107CC0009AFE214618480AF0A4FE2B6820F0040210
:107CD000002B18BF042321461A4313480AF08BFED9
:107CE000FFF73ABA7021104836B90AF092FEC0B2D6
:107CF00028603446FFF730BA0AF08BFE2A7820F06D
:107D0000FF000243702108480AF075FE0024FFF7C7
:107D100023BA68B9702104480AF07BFEC0F3014021
:107D200028603446FFF718BAE8370020FFFF0F003D
:107D30001B68032B00F2928070214D480AF069FE07
:107D40002B6820F440321B0403F440331A437021A3
:107D500047480AF050FE0024FFF7FEB948B97021E9
:107D600043480AF056FEC0F3804028603446FFF7CF
:107D7000F3B91B68012B74D870213D480AF049FE05
:107D80002B6820F480229B0403F480231A43702183
:107D900037480AF030FE0024FFF7DEB9702134487E
:107DA0003EB90AF036FEC0F3015028603446FFF7B2
:107DB000D3B90AF02EFE2B6820F440121B0503F401
:107DC00040131A4370212A480AF015FEFFF7C4B980
:107DD000002849D16F2126480AF01BFEC0F3090094
:107DE00028603446FFF7B8B938B9392120480AF07D
:107DF00010FE34462860FFF7AFB91A6839211C48D5
:107E00000AF0F9FD0024FFF7A7B938B93A2118485C
:107E10000AF0FFFD34462860FFF79EB91A683A2140
:107E200013480AF0E8FD0024FFF796B90824FFF78D
:107E300093B90424FFF790B90024FFF78DB9042407
:107E4000FFF78AB90424FFF787B90424FFF784B940
:107E50000424FFF781B90424FFF77EB91024FFF74B
:107E60007BB91024FFF778B90424FFF775B900BF78
:107E7000E837002007B5019201AB02460120FFF769
:107E80004DF903B05DF804FB134602460020FFF7EE
:107E900045B908B50348D0F8BC220AF0EBFE002033
:107EA00008BD00BFE837002008B50348D0F8BC2261
:107EB0000AF0CCFE002008BDE837002008B50248D3
:107EC0000AF0C1FE002008BDE837002008B50248CE
:107ED0000AF0B6FE002008BDE837002008B50248C9
:107EE0000AF0ACFE002008BDE837002008B50248C3
:107EF0000AF090FE002008BDE837002001480AF093
:107F000012BE00BFE837002038B522210D480AF024
:107F100080FD0C4C10B920460AF0EEFD0A4BD4F857
:107F2000B402DD682B689B6998472B68D4F89002EF
:107F30001B6998472B68D4F894021B699847012065
:107F400038BD00BFE837002070A30208022804BF34
:107F50000C4B93F8F00038B90B4BDB681B685B697E
:107F60000A4AD2F898021847012809D1054B93F81C
:107F7000F030012B04D1044BDB681B689B69EFE7F1
:107F8000704700BF9C64002070A30208E8370020FF
:107F9000012908B508D1054A70210AF02CFDBDE879
:107FA000084003480AF07EBD08BD00BFC8040500B4
:107FB000E8370020034B0846D3F8C0321146DB688F
:107FC000184700BFE837002070B5644E644CF56870
:107FD0006B6803F1CC02C4F8982203F58272C4F8EE
:107FE0009C2203F59072C4F8A02203F5BA72C4F87B
:107FF000902203F5C872C4F8942203F5F272C4F813
:10800000B42203F50072C4F8B82203F5627203F1DA
:10801000E800C4F8A82203F5697203F57073C4F888
:10802000AC322B68C4F8B0221B69C4F8A40298478C
:108030002B68D4F8A0021B6998472B68D4F89C02DF
:108040001B6998472B68D4F8AC021B6998472B68CA
:10805000D4F8B0021B6998472B68D4F8A802DB68F3
:1080600098472B68D4F890021B6998472B68D4F87E
:1080700094021B6998472B68D4F89802DB689847EC
:108080002B68D4F8B402DB6898472B68D4F8B802A0
:10809000DB6898472B68D4F8A8029B699847326937
:1080A00001266B68C4F8C02203F5387353602D4B6A
:1080B0002D499A693220C2F804122C491680C2F860
:1080C00008122B491E7559622A4919622A49D96139
:1080D0002A4999622A49D9632A4999632A49D96266
:1080E0002A4919632A49D9642A4999642A49996510
:1080F0002A4959652A4919652A4959662A4919663A
:108100004FF4F071C3E9031028492046D965284B84
:1081100000210AF0A6FC274920460AF018FD236832
:108120000220D3F8A030C4F8BC32FFF70FFF0222C0
:10813000D4F8B832197C5A74186832460CF07DF9BC
:108140002B68D4F8B8021C4C1B68984723689847E2
:108150000021A3680846BDE87040184770A30208D4
:10816000E83700209C640020097F0108FD7E01089B
:10817000ED7E0108DD7E0108CD7E0108BD7E01088F
:10818000897E0108757E0108A97E0108937E010899
:10819000F170010809710108FD700108B56E010850
:1081A000956E01084D7F0108A96E010859700108FC
:1081B000689F0208917F0108800A002018B9034BCC
:1081C0001B680B6070470820704700BFB83A00205A
:1081D0000022014B9A6070479C640020234B70B5CD
:1081E000DD68234C2B68D4F898029B6998472B686C
:1081F000D4F8A8029B6998472B68D4F8AC029B6915
:1082000098472B68D4F89C029B6898472B68D4F851
:10821000A0029B6898472B68D4F8A4029B689847F3
:108220002B68D4F890029B6898472B68D4F8940286
:108230009B6898472B68D4F8B0029B6898472B68D6
:10824000D4F8B4029B6898472B68D4F898029B68CE
:1082500098472B68D4F8A8029B6898472B68D4F8F5
:10826000AC029B68BDE87040184700BF70A30208CD
:10827000B83A0020024BD3F8B8020AF07FBD00BF25
:10828000B83A002038B5284D00F07F042B1993F838
:108290000C32DB0705D4D5F8B83203EB84046068F0
:1082A00038BDD5F8BC3200219B6820469847002194
:1082B000D5F8BC3208469B6898470021D5F8BC32F7
:1082C00008469B6898470021D5F8BC3208469B6851
:1082D0009847D5F8BC3201219B6800209847D5F813
:1082E000BC3200219B68204698470021D5F8BC325B
:1082F00008469B6898470021D5F8BC3204029B6869
:10830000084698470021D5F8BC3204439B680846CC
:108310009847D5F8BC32240204439B680121002011
:10832000984724022043BBE7B83A0020022804BF44
:108330000C4B93F8F00038B90B4BDB681B685B699A
:108340000A4AD2F898021847012809D1054B93F838
:10835000F030012B04D1044BDB681B689B69EFE70D
:10836000704700BF9C64002070A30208B83A002048
:10837000012870B506460F4D0F4C07D1EB6AC4F8C3
:10838000C0325B68984784F8C46270BD94F8C43208
:10839000012B03D1D4F8C0329B689847EB682A6957
:1083A0005B68C4F8BC2203F538735360002384F87B
:1083B000C432EAE770A30208B83A00200528F8B5ED
:1083C0000C46154600F0A5801FD8022869D004D8B5
:1083D00000283ED004242046F8BD032873D004288A
:1083E000F8D1604B604EDF6814683B68D6F8A00295
:1083F000002C7ED0012C00F087801B6998473B68D9
:10840000D6F8A0025B6A98477BE0082800F08D80D0
:1084100009D80628DED1534B534ADB68D2F8B402A0
:108420001B685B6A7CE0092800F08880FC28D1D1B9
:108430004C4B4D4EDF6814683B68D6F8A002002C08
:1084400000F08C80DB6898473B68D6F8A0029B69F7
:1084500016E0126832F0030340F08280414B424E36
:10846000DF68D207D6F894023B680BD51B699847A2
:108470002C683B6814F00204D6F8900209D01B69FE
:1084800098473FE0DB6898473B68D6F894029B69C1
:10849000EDE7DB6898473B68D6F890029B69984700
:1084A00099E7304B1468DE68D6E9003000F50770B4
:1084B0003CB1DB689847D6E900309B6900F507704E
:1084C000DEE79B68EBE7284BD3F8A802254BDB6877
:1084D0001B6839B1146814F0010401D05B69CFE75F
:1084E0009B69DCE75B6A9847003018BF0120286071
:1084F00071E7DB6898473B689B69D6F8A00298470C
:1085000020462860002466E7DB6898473B685B6983
:10851000F3E7144B144ADB68D2F8B0021B685B6ABD
:108520009847003018BF0120EBE710680E4B00F0B1
:10853000010083F8C502FFF71BFFE3E7094B126850
:10854000DC68012AD4E9003000F5077004D1DB684B
:108550009847D4E90030B0E79B6891E71B699EE734
:10856000102438E770A30208B83A00207FB52C4BDE
:1085700000F07F041A1992F80C221D4612F0010F28
:1085800006D1D3F8B83203EB8404606804B070BD40
:1085900005230122032101A8ADF804308DF806401F
:1085A00006F0C2FBD5F8C0328DF80700DB699847AA
:1085B0000421D5F8C0320DEB01005B69984703F048
:1085C000A5F80646D5F8C0321B6A984707281FD978
:1085D0000821D5F8C0320DEB01009B6998470122B4
:1085E000072102A89DF80F5006F09EFB854214D18A
:1085F0009DF80830052B10D19DF80930FF2B0CD1C8
:108600009DF80A30A34208D1DDF80B0000BABDE79F
:10861000304603F08BF83228D4D94FF0FF30B5E75D
:10862000B83A0020034A0146D2F8B83200200AF0D6
:108630006CBB00BFB83A0020024B93F8C53203B1BF
:1086400094E71FE6B83A002038B52220FFF7F4FF80
:10865000094C18B9D4F8B8020AF088FB074BD4F8D3
:108660009002DD682B681B6998472B68D4F8940248
:108670001B699847012038BDB83A002070A3020852
:1086800010B508461446FFF7D7FF206010BD2DE94E
:10869000F74F364D01F07F0995F8C56290469A462E
:1086A0009DF830409DF8347049F08000AB46A6B389
:1086B00005238DF802008DF803200721012268466A
:1086C000ADF800308DF804A08DF805408DF80670E7
:1086D00006F02AFBD5F8C0328DF80700DB69984711
:1086E0006D460026DBF8C03215F8010BDB68013659
:1086F0009847082EF6D1022003F00EF847EA04242A
:10870000DBF8B83244EA0A4403EB890944EA086416
:10871000C9F8044003B0BDE8F08FD5F8BC3231464B
:108720009B689847D5F8BC3231469B6840469847CD
:10873000D5F8BC3231469B6850469847D5F8BC32D4
:1087400031469B6820469847D5F8BC3201219B688A
:10875000384698474AEA082344EA0324D5F8B83251
:1087600047EA042403EB8909D2E700BFB83A0020A6
:1087700007B5D3B20193C2F307230093C2F30743B3
:10878000120EFFF784FF03B05DF804FB0020FFF733
:10879000EFBF73B50D460646E8B9104C94F8C632E3
:1087A00043B1D4F8B8322721D3F8A020FFF7E0FF77
:1087B00084F8C66200242A462D210020FFF7D8FF46
:1087C0002046CDE90044234622462021FFF75FFFE3
:1087D000204602B070BD0820FBE700BFB83A002079
:1087E00038B50C4605462120FFF726FF2368C1183F
:1087F00021602846BDE83840CBE737B50D46044632
:10880000C8B901220D4B83F8C62281EAE172A2EBBE
:10881000E1722721FFF7ACFF002DACBF012302233B
:108820002046CDE90043224623462021FFF72FFFB3
:10883000204603B030BD0820FBE700BFB83A002057
:108840000021DAE74942D8E7D7E7F8B506461D46E2
:108850000C46002940F01B86222A00F0B38272D811
:108860000E2A00F0C7813AD8062A00F04A811AD8A9
:10887000022A00F0FE8008D8002A00F0DE80012ADB
:1088800000F0E98004242046F8BD042A00F0148199
:1088900040F20381002840F02D812620FFF7CCFE16
:1088A00034462860EFE70A2A00F0648107D8072AD7
:1088B00000F03E81082A00F052810424E3E70C2AEC
:1088C00000F0728140F264813420002E40F08481F7
:1088D000FFF7B2FE00F0010028603446D3E7152A06
:1088E00000F0E18119D8112A00F0AD8107D80F2AD4
:1088F00000F08D81102A00F098810424C3E7132A28
:1089000000F0BC8140F2AC81002840F0C5812B20F2
:10891000FFF792FE34462860B5E71B2A00F000827C
:1089200007D8172A00F0CC81182A00F0EB81042424
:10893000A9E71D2A00F02782C0F00982212A00F051
:108940002A8204249FE7AE2A00F0FE8341D8A72A9A
:1089500000F0568321D8A32A00F0AD8207D88C2AD4
:1089600000F04782A22A00F08E8204248BE7A52A19
:1089700000F0D08240F2B6826C20FFF75DFE00F47A
:108980008044002E40F01D83002C00F00F8300096E
:1089900000F070002860344675E7AA2A00F078835A
:1089A00007D8A82A00F04283A92A00F0568304249D
:1089B00069E7AC2A00F09F8340F283836D20002E8C
:1089C00040F0B283FFF738FEC0F300602860344601
:1089D00059E7BB2A00F09E8415D8B62A00F01C8403
:1089E00007D8B42A00F0D083B52A00F0D983042434
:1089F00049E7B92A00F0508400F26884B82A00F0F0
:108A0000318404243FE7CC2A00F0FD840AD8BF2A31
:108A100000F0BC84C02A00F0D884BC2A00F0A084F6
:108A2000042430E7D12A00F01285D22A00F01F85F5
:108A3000CE2A00F00185042425E728B92D20FFF770
:108A4000FBFD344628601EE71A682D210020FFF741
:108A50008FFE002417E728B92120FFF7EDFD3446EB
:108A6000286010E71A6821210020FFF781FE00240A
:108A700009E728B92720FFF7DFFD3446286002E721
:108A80001A682721002AB8BF52422046FFF770FE1D
:108A90000122B34B83F8C622F5E6002840F0FA84A1
:108AA0002220FFF7C9FD10F4000318BF4FF07F43E9
:108AB000184328603446E6E6A94BD3F8B82220B91B
:108AC000D2F8A03004462B60DDE62B682020002B76
:108AD000B8BF5B42C2F8A030FFF7AEFD044608B154
:108AE0000024D0E62A682721002AB8BF5242FFF7A7
:108AF0003FFEC8E61A6826210020FFF739FE002451
:108B0000C1E6102036B9FFF797FDC0F304202860B6
:108B10003446B8E6FFF790FD2B6820F4F8521B02AC
:108B200003F4F8531A4310212046FFF721FEAAE66A
:108B3000102036B9FFF780FD00F01F002860344692
:108B4000A1E6FFF779FD2B6820F01F0203F01F0359
:108B50001A4310210020FFF70BFE002493E60028A3
:108B600040F09B843520FFF767FDC0F3402028606C
:108B7000344688E6002840F093843520FFF75CFDFA
:108B800010F0020F0CBF0123002334462B607AE65D
:108B9000002840F088843520FFF74EFDC04300F0E8
:108BA0000100286034466EE6342036B9FFF744FDF4
:108BB000C0F340002860344665E6FFF73DFD2B68B2
:108BC00020F002025B0003F002031A43342100206C
:108BD000FFF7CEFD002456E6FFF72EFD2B6820F0B0
:108BE000010203F001031A4334210020FFF7C0FD06
:108BF000002448E628B93420FFF71EFD34462860DB
:108C000041E61A6834212046FFF7B2FD3BE628B959
:108C10002420FFF711FD3446286034E61A68242129
:108C20000020FFF7A5FD00242DE628B92520FFF739
:108C300003FD3446286026E61A6825210020FFF748
:108C400097FD00241FE628B92820FFF7F5FC3446DD
:108C5000286018E61A6828212046FFF789FD12E6E9
:108C600028B92A20FFF7E8FC344628600BE61A688A
:108C70002A210020FFF77CFD002404E628B92320E8
:108C8000FFF7DAFC34462860FDE51A68232100204E
:108C9000FFF76EFD0024F6E51A682B210020FFF790
:108CA00067FD0024EFE528B92C20FFF7C5FC34460A
:108CB0002860E8E51A682C212046FFF759FDE2E517
:108CC000284C68B91520FFF7B7FC30B14FF080731E
:108CD000B3FBF0F39C4228BF1C462C600024D2E575
:108CE0001B686BB14FF0807292FBF3F2A242A8BFF7
:108CF00022462A6015210020FFF73AFD0024C2E534
:108D00002246F6E728B93320FFF796FC3446286060
:108D1000B9E51A6833210020FFF72AFD0024B2E5E7
:108D20006C2036B9FFF788FCC0F3C0402860344699
:108D3000A9E5FFF781FC2B6820F40022DB0403F493
:108D400000231A436C212046FFF712FD9BE56C209F
:108D500056B9FFF771FCC0F380402860344692E5B5
:108D6000B83A0020FFFF0F00FFF766FC2B6820F4E5
:108D700080229B0403F480231A436C210020FFF718
:108D8000F7FC00247FE5002840F09083BF4B0446A9
:108D90001B682B6077E530B9FFF74EFC00F001004F
:108DA000286034466FE50020FFF746FC00212B6861
:108DB00020F0010203F001031A430846FFF7D8FC34
:108DC000002460E530B9FFF737FCC0F340002860AD
:108DD000344658E50846FFF72FFC2B6820F00202C6
:108DE0005B0003F002031A4321462046FFF7C0FC54
:108DF00049E550B96C20FFF71FFC4FF48073C0F3B6
:108E0000036003412B6034463DE51B68102B34D0D2
:108E10000FDC022B2DD006DC012B18D04FF0FF33D6
:108E200010242B602FE5042B25D0082BF6D1052329
:108E30000EE0402B23D003DC202BEFD1032307E0EF
:108E4000802B1ED0B3F5807FE8D1002300E00823FB
:108E50002B606C20FFF7F0FB2B6820F070621B0684
:108E600003F070631A436C210020FFF781FC00249B
:108E700009E50723ECE70623EAE70423E8E70223F2
:108E8000E6E70123E4E76C2036B9FFF7D5FBC0F332
:108E9000C13028603446F6E4FFF7CEFB2B6820F49F
:108EA000C032DB0303F4C0331A436C210020FFF708
:108EB0005FFC0024E7E46C2036B9FFF7BDFBC0F38C
:108EC000803028603446DEE4FFF7B6FB2B6820F4E0
:108ED00080429B0303F480431A436C212046FFF732
:108EE00047FCD0E46C2036B9FFF7A6FBC0F3003096
:108EF00028603446C7E4FFF79FFB2B6820F48052BC
:108F00001B0303F480531A436C210020FFF730FC4D
:108F10000024B8E46C20FFF78FFB0746C6B910F4B5
:108F2000804405D0C70907F4F0672F603446AAE4EF
:108F30006C20FFF781FB17F00B0F4FEA201000F0B9
:108F4000700001D12860CBE540F0080028609AE469
:108F50006C20FFF771FB10F480444FF06C000ED0D2
:108F6000FFF76AFB2B6820F4F062DB0103F4F06387
:108F70001A436C210020FFF7FBFB002483E4FFF77A
:108F80005BFB6C2120F400622046FFF7F1FB6C20B4
:108F9000FFF752FB2B6820F070021B0103F07003F7
:108FA0001A436C212046FFF7E3FB6CE4C30902057A
:108FB00003F4F06301D42B6092E543F008032B60C7
:108FC00061E46C2074B1FFF737FB2B6820F070026E
:108FD0001B0103F070031A436C210020FFF7C8FB4C
:108FE000002450E4FFF728FB2B6820F4F062DB013B
:108FF00003F4F0631A436C212046FFF7B9FB42E407
:109000006C2036B9FFF718FB00F00F0028603446DB
:1090100039E4FFF711FB2B6820F00F0203F00F0378
:109020001A436C212046FFF7A3FB2CE46D2036B9D0
:10903000FFF702FBC0F3C0302860344623E4FFF79B
:10904000FBFA2B6820F40042DB039BB21A436D212C
:109050000020FFF78DFB002415E46D2036B9FFF7E3
:10906000EBFAC0F34130286034460CE4FFF7E4FA31
:109070002B6820F4C0425B0303F4C0431A436D2104
:109080000020FFF775FB0024FFF7FDBBB83A002076
:109090006D203EB9FFF7D0FAC0F3032028603446B4
:1090A000FFF7F1BBFFF7C8FA2B6820F470621B02D0
:1090B00003F470631A436D212046FFF759FBFFF755
:1090C000E2BB6D203EB9FFF7B7FAC0F3411028604C
:1090D0003446FFF7D8BBFFF7AFFA2B6820F06002E9
:1090E0005B0103F060031A436D210020FFF740FB92
:1090F0000024FFF7C8BB6D203EB9FFF79DFA00F0D2
:109100000F0028603446FFF7BEBBFFF795FA2B68C7
:1091100020F00F0203F00F031A436D210020FFF728
:1091200027FB0024FFF7AFBBFFF786FA2B6820F080
:1091300080721B0603F080731A436D210020FFF735
:1091400017FB0024FFF79FBB6D2076B9FFF774FA79
:10915000001400F07F0310F0400018BF6FF07F0094
:10916000184328603446FFF78EBBFFF765FA2B687B
:1091700020F4FE021B0403F4FE031A436D21204673
:10918000FFF7F6FAFFF77FBB002840F092816F20CF
:10919000FFF752FAC0F3044028603446FFF773BB70
:1091A0003420BEB9FFF748FA43050FD51420FFF766
:1091B00043FAC64B30B14FF08072B2FBF0F29342EB
:1091C00028BF13462B600024FFF75DBB2E6034469A
:1091D000FFF759BBFFF730FA2B6820F48062002BB1
:1091E00018BF4FF4806334211A430020FFF7C0FA00
:1091F0002968B64B71B14FF0807292FBF1F29A423E
:10920000A8BF1A462A6014210020FFF7B1FA0024F3
:10921000FFF739BB1A46F5E7AC4C80B91420FFF7CD
:109220000BFA50B14FF08073B3FBF0F0A04288BF4F
:10923000204628600024FFF726BBA448F9E71B68F6
:1092400073B14FF0807292FBF3F2A242A8BF2246A4
:109250002A6014210020FFF78BFA0024FFF713BBCC
:109260009A4AF5E76C203EB9FFF7E6F9C0F34030C3
:1092700028603446FFF707BBFFF7DEF92B6820F4C0
:1092800000525B0303F400531A436C210020FFF7E4
:109290006FFA0024FFF7F7BA6C203EB9FFF7CCF95C
:1092A000C0F3035028603446FFF7EDBAFFF7C4F966
:1092B0002B6820F470021B0503F470031A436C2121
:1092C0000020FFF755FA0024FFF7DDBA7F4C70B994
:1092D0001320FFF7B1F930B14FF08073B3FBF0F317
:1092E0009C4228BF1C462C600024FFF7CCBA1B68A8
:1092F00073B14FF0807292FBF3F2A242A8BF2246F4
:109300002A6013210020FFF733FA0024FFF7BBBACD
:109310002246F5E770203EB9FFF78EF9C0F307202B
:1093200028603446FFF7AFBAFFF786F92A6820F4C1
:109330007F40120292B2024370212046FFF718FAD2
:109340002046FFF779F92B6820F00402002B18BFA4
:10935000042321461A432046FFF70AFAFFF793BA7F
:10936000702036B9FFF768F9C0B228603446FFF7BD
:109370008ABAFFF761F92A7820F0FF0002437021D2
:109380000020FFF7F5F90024FFF77DBA40B97020FF
:10939000FFF752F9C0F3014028603446FFF773BA73
:1093A0001B68032B00F288807020FFF745F92B68BB
:1093B00020F440321B0403F440331A437021002090
:1093C000FFF7D6F90024FFF75EBA40B97020FFF727
:1093D00033F9C0F3804028603446FFF754BA1B6865
:1093E000012B6CD87020FFF727F92B6820F480221E
:1093F0009B0403F480231A4370210020FFF7B8F97F
:109400000024FFF740BA70203EB9FFF715F9C0F30A
:10941000015028603446FFF736BAFFF70DF92B6884
:1094200020F440121B0503F440131A437021204618
:10943000FFF79EF9FFF727BA002843D16F20FFF707
:10944000FBF8C0F3090028603446FFF71CBA30B9B6
:109450003920FFF7F1F834462860FFF714BA1A688C
:1094600039210020FFF784F90024FFF70CBA30B946
:109470003A20FFF7E1F834462860FFF704BA1A688B
:109480003A210020FFF774F90024FFF7FCB9082403
:10949000FFF7F9B90424FFF7F6B90424FFF7F3B98D
:1094A0000424FFF7F0B90424FFF7EDB90424FFF713
:1094B000EAB90424FFF7E7B91024FFF7E4B9102450
:1094C000FFF7E1B90424FFF7DEB900BFFFFF0F008B
:1094D00007B5019201AB02460120FFF7B6F903B0D0
:1094E0005DF804FB134602460020FFF7AEB9044BBB
:1094F000084693F8C5320BB1FFF738B8FEF7C2BE85
:10950000B83A002038B5544C204609F0C3FB534B01
:10951000DD686B6803F1E802C4F8A42203F58272E7
:10952000C4F89C2203F59072C4F8A02203F5BA7225
:10953000C4F8902203F5C872C4F8942203F5E472CB
:10954000C4F8A82203F5007203F1CC00C4F8AC22E1
:1095500003F5697203F57073C4F8B0322B68C4F870
:10956000B422DB68C4F8980298472B68D4F8A802A4
:10957000DB6898472B68D4F8AC02DB6898472B6807
:10958000D4F898025B6998472B68D4F8A8029B69C5
:1095900098472B68D4F8AC025B6998472B68D4F8DD
:1095A000A4021B6998472B68D4F8A0021B6998474E
:1095B0002B68D4F89C021B6998472B68D4F8B0023A
:1095C0001B6998472B68D4F8B4021B6998472B682D
:1095D000D4F890021B6998472B68D4F894021B6951
:1095E000984794F8C502FEF7C3FE1D4B1D499A69C2
:1095F0000220C2F804121C49C4F8B822C2F80812AA
:1096000001211180194A19755A62194A32211A62C8
:10961000184ADA61184A9A62184ADA63184A9A6351
:10962000184ADA62184A1A63184ADA64184A9A64BD
:10963000184A9A65184A5A65184A1A65184A5A66A5
:10964000184A1A664FF42572C3E90321164ADA65EF
:10965000BDE83840FEF76ABEB83A002070A30208A1
:109660009C6400204986010875820108FB87010877
:10967000498801084588010841880108E5940108E6
:10968000D194010893870108E18701088D870108BB
:109690008186010825860108BD830108BD81010876
:1096A0002D830108D1810108DD81010818B9034B20
:1096B0005B680B6070470820704700BF8C3D00203E
:1096C0000022014B9A6070479C6400200428F8B582
:1096D0000C4615466FD006D8022844D055D8D0B1D4
:1096E00004242046F8BD062800F09380C0F0858051
:1096F000FC28F5D14D4B4E4EDF6814683B68D6F818
:10970000A002002C00F08D80DB6898473B68D6F8FB
:10971000A0029B6916E0126832F0030340F08380D8
:10972000424B434EDF68D207D6F894023B680BD514
:109730001B6998472C683B6814F00204D6F8900225
:1097400009D01B69984751E0DB6898473B68D6F819
:1097500094029B69EDE7DB6898473B68D6F8900276
:109760009B699847BDE7314B1468DE68D6E9003045
:1097700000F507703CB1DB689847D6E900309B697B
:1097800000F50770DEE79B68EBE7294BD3F8A802EA
:10979000264BDB681B6839B1146814F0010401D052
:1097A0005B69CFE79B69DCE75B6A9847003018BFCD
:1097B0000120286095E71D4B1D4EDF6814683B684B
:1097C000D6F8A0024CB1012C12D01B6998473B6817
:1097D000D6F8A0025B6A984707E0DB6898473B68C9
:1097E0009B69D6F8A002984720462860002478E7B5
:1097F000DB6898473B685B69F3E70C4B0C4ADB6816
:10980000D2F8B0021B685B6A9847003018BF01208D
:10981000EBE7064B064ADB68D2F8B4021B685B6ACA
:10982000F2E71B699DE710245BE700BF70A3020805
:109830008C3D0020234B70B5DD68234C2B68D4F899
:1098400098029B6998472B68D4F8A8029B699847AF
:109850002B68D4F8AC029B6998472B68D4F89C021B
:109860009B6898472B68D4F8A0029B6898472B68A0
:10987000D4F8A4029B6898472B68D4F890029B68A0
:1098800098472B68D4F894029B6898472B68D4F8C3
:10989000B0029B6898472B68D4F8B4029B6898473D
:1098A0002B68D4F898029B6898472B68D4F8A802D4
:1098B0009B6898472B68D4F8AC029B68BDE8704061
:1098C000184700BF70A302088C3D002001460148E4
:1098D00009F0E2BA8C3D002010B50348144609F0A7
:1098E00096FA206010BD00BF8C3D0020014809F0B1
:1098F00080BA00BF8C3D0020F8B506461D460C46D8
:10990000002940F06186222A00F0C88275D80E2A0C
:1099100000F0D2813CD8062A00F04D811BD8022AE3
:1099200000F0058108D8002A00F0E380012A00F049
:10993000EF8004242046F8BD042A00F0198140F28B
:109940000781002840F030812621C04809F05FFAE5
:1099500034462860EEE70A2A00F0698107D8072A12
:1099600000F04181082A00F056810424E2E70C2A25
:1099700000F07B8140F26C813421B448002E40F02D
:109980008D8109F044FA00F0010028603446D1E7E7
:10999000152A00F0F0811AD8112A00F0B98107D8F1
:1099A0000F2A00F09781102A00F0A3810424C1E758
:1099B000132A00F0CA8140F2B981002840F0D48116
:1099C0002B21A24809F023FA34462860B2E71B2A6B
:1099D00000F0118207D8172A00F0DB81182A00F066
:1099E000FB810424A6E71D2A00F03682C0F01B820A
:1099F000212A00F0398204249CE7AE2A00F0288452
:109A000043D8A72A00F0778322D8A32A00F0C68281
:109A100007D88C2A00F05982A22A00F0A6820424DA
:109A200088E7A52A00F0EB8240F2D0826C218748BB
:109A300009F0EDF900F48044002E40F03C83002C46
:109A400000F02E83000900F070002860344671E7B2
:109A5000AA2A00F09C8307D8A82A00F06383A92AC9
:109A600000F07A83042465E7AC2A00F0C58340F255
:109A7000A8836D217548002E40F0DA8309F0C7F9FC
:109A8000C0F300602860344654E7BB2A00F0CF845E
:109A900015D8B62A00F0488407D8B42A00F0F98314
:109AA000B52A00F00384042444E7B92A00F07F8437
:109AB00000F29884B82A00F05F8404243AE7CC2AA4
:109AC00000F03A850AD8BF2A00F0F084C02A00F0DE
:109AD0000E85BC2A00F0D38404242BE7D12A00F0A1
:109AE0005185D22A00F05F85CE2A00F03F850424FC
:109AF00020E730B92D21554809F089F9344628600E
:109B000018E71A682D21514809F073F9002411E76C
:109B100030B921214D4809F07AF93446286009E727
:109B20001A682121494809F064F9002402E730B994
:109B30002721464809F06BF934462860FAE61A688E
:109B40002721002AB8BF5242404809F052F9F1E6F5
:109B5000002840F03C8522213C4809F058F910F4D7
:109B6000000318BF4FF07F43184328603446E1E6F6
:109B7000364F20B9D7F8B83204462B60DAE61B68B6
:109B80002021002BB8BF5B423846C7F8B83209F035
:109B90003EF9044608B10024CCE6D7F8B8222721C4
:109BA000384609F026F9C5E61A682621274809F043
:109BB00020F90024BEE61021244836B909F027F91F
:109BC000C0F3042028603446B4E609F020F92B687D
:109BD00020F4F8521B0203F4F8531A4310211B48D7
:109BE00009F007F9A6E61021184836B909F00FF96F
:109BF00000F01F00286034469CE609F008F92B6845
